:020000040000FA
:103000002BEF1BF091EF1BF0A5EF1BF0ADEF1BF0CA
:10301000CBEF1BF0F9EF1BF04EEF1CF053EF1CF061
:103020003BEF1CF040EF1CF056EF1CF006EF1CF0DD
:1030300004EF1CF001EF1CF003EF1CF080EF1AF01E
:10304000E9EF1AF0F7EF1AF0FBEF1AF013EF1CF0AC
:1030500012EF1CF0A8EF1AF0B3EF1AF0FCEF1AF021
:103060001200000012000000120000001200000018
:103070001200000012000000120000001200000008
:10308000FFFF0C4590000845910004459200004563
:103090009300FC449400C844A300CC45A000224502
:1030A0008B0026458A002A4589002E458800444623
:1030B0008000824881008A48820002468300504690
:1030C000BA000647BF00BE46B900E246BB00FC4757
:1030D000BD001448BE002C4897004E4795006C4731
:1030E0009E008E47BC00EA4796002E469D009E48F3
:1030F000B000A248B100A648B200AA48B300AE484A
:10310000B400B248B500B648B600BA48B700304976
:10311000A8003449A9003849AA003C49AB004049FD
:10312000AC004449AD004849AE004C49AF0092485C
:10313000B8000000000044000088440001894400F9
:10314000028A4400038B2B0001822B0004810A00B9
:103150000680480000B5480001B6480002B70600E6
:1031600000BB060001BA060002B9060004AC060066
:1031700005AD060006AE060007AF070000A7070072
:1031800001A60800009F0800019E0800029D08009B
:1031900003940800049508000596080006970700A8
:1031A00004A4070005A5070006B30A0007B207003C
:1031B00007B1090006AB090007AA0900009309003E
:1031C000019209000291090003900900049B090083
:1031D000059A0A0000980A0001990A0002A30A0051
:1031E00003A20A0004A10A0005A0070003BF07000C
:0631F00002BE0000000019
:1032800006811C811081148108810C8100810481D8
:103290001A811E81128116810A810E810281FFFF2F
:10330000060103510F0BD8B41200DAEC16F039D0D5
:103310000400A8D848E106011FEE60F0E7BE19D00E
:103320001FEE50F0E7BE15D01EEE20F0E7BE11D024
:103330001EEE30F0E7BE0DD01EEE40F0E7BE09D025
:103340001EEE50F0E7BE05D01EEE60F0E7BE01D0E5
:10335000DFD7E1CF01F6E2CF02F6050EE3500F0B07
:1033600006010D6F020EE330700B046F0439001973
:10337000070B09E1020EE350030B17E0FE0F23E0F9
:1033800004D0000E05D0020E03D0030E01D0FF0EB4
:1033900001C6E1FF02C6E2FFE79E010F03E0FF0F57
:1033A00015EC1AF0B5D7D2EF16F0040EE350FF0F6C
:1033B00001E0EBD7000E15EC1AF054D8F4E10F0140
:1033C00030B7FBD7F0D7080E0D632ED0040EE3CF35
:1033D000F6FF030EE3CFF7FFF86A030ED890F63638
:1033E000F736F836FF0FFAE1060EE12607EE00F099
:1033F000F650380BE926080EE6CFEEFFFF0FFCE192
:10340000F6503F0B380A0FE1F85005E1F750330A48
:103410000AE0070A08E0C00EF61617EE00F0B6EC58
:1034200016F0010A01E0ADD7B0D70601066F1AD831
:103430000DE10F0130B7FBD71FEE31F00601065149
:1034400007D80F01356B3087060112000601120004
:1034500004C6E7FFE68E030B0809E66EE66A05C6BA
:10346000E6FF1200060100BB08D07450380B07E0DD
:103470006F886F501F0B20096F6EFF091200000B41
:02348000120038
:103500000096F90E96160501856B640ECEEC16F04A
:103510008C9C8C9A380E8A6E4ED854D8320ECEECD3
:1035200016F049D84FD8320ECEEC16F044D84AD80F
:10353000080E19D80C0E17D8060E15D8010EB3ECCC
:103540001AF0849F380E0FD80C0E0DD8000E4FD0F5
:103550008A6EE8408D6EE84411D885B512008C8AD9
:103560008C9C29D82FD08A6EE8408D6EE84406D80E
:1035700085B512008C9A8C9C1ED824D085B512007B
:10358000F30E9312060E96128C9A836B846B8C8CBE
:1035900019D8832BD8B4842B09E00DD881BEF8D775
:1035A00011D80C0E9316F90E9616120085A7858178
:1035B00085B78583F6D78C8E0000000000000000E0
:1035C00000001200000000000000000000008C9EBF
:1035D0001200010EB3EC1AF08BBF03D08CBF01D0E8
:1035E00012007A8F010EB3EC1AF07A9F12000501D7
:1035F0007A518009B8D7ACD7E83AE830380B40099F
:10360000B2DF0501876B0900F550A2DF872B87A782
:10361000FAD7F7EF1AF001030703010000000000DA
:103620000010181C18101B131B1B1B1B111F110E45
:103630001E1D1B17001F001D1B1D1E0E111F1D1917
:10364000150D001D1D1F0206021A020207000103CC
:103650000713191C1810106AF29EFE0EF66EFF0E6C
:10366000F76E3F0EF86E0900F550066E0900F55032
:10367000076E270A11E0F86AF28EEE0E24EC16F0BF
:103680000638070B24EC16F007507F0B24EC16F0DD
:103690001EEC16F0F29EFFD7F86AF28E01010E6B57
:1036A000010EE8CF6DF01568090ECB6E240ECA6EC0
:1036B0000F0EBD6E040EBE6EB7EC5FF004EC16F09C
:1036C000126E0101420E0C6F0D6F0F0EE8CF18F352
:1036D000E8CF58F3136A146A3BEC54F03AEC52F01A
:1036E0003DEC51F0125009E10A0E78EC16F0010E93
:1036F00080EC16F0000E7CEC16F07DEC1CF0000E59
:1037000014EC16F0AEEC1DF0D3ECA0F01082100E0D
:10371000036E270E046E000EBCEC16F0E7EC29F0E9
:10372000120010921FEC63F010B405D050EC5DF065
:10373000E2EC5FF005D0F29E109644B01086F28E57
:1037400030EC1EF0E2EC26F0120010A431EC63F035
:10375000125002E1DBEC27F01200120000144D4978
:103760004449626F785349442056322E30524332D6
:10377000302040104C61756E6368696E672043535A
:103780002020202040104353206E6F7420656E610E
:10379000626C6564212082EC16F05C0EF66E370ECA
:1037A000F76E000EF86E31501CE09EEC16F0720EB3
:1037B000F66E370EF76E000EF86E125006E0840EAD
:1037C000F66E370EF76E000EF86E9EEC16F000B631
:1037D00008D0160EF66E360EF76E000EF86EE6EC9A
:1037E00016F01C8210A404D044A002D0F5ECA0F086
:1037F00012001250D8A4120010B61200F3EC29F0F7
:103800001200EFEF7FF0120024EF87F0125208E170
:10381000E8CF04F11BECA1F010B4120004C1E8FFE2
:1038200003EF87F012000B6E0101F80E0B620BD054
:103830003D513C6F3D6B3F5104083B273F6B3C3192
:10384000E8303F0B3E6FFA0E0B620CD01E89C2C0EF
:10385000E8FFE8B210883D29800ED8B43D6B3B6B81
:10386000030E3F6FFB0E0B6201D01E8BFC0E0B6232
:1038700001D01E8D1200125002E12FEF22F0120033
:103880001250D8A4120003C057F0000E036203D0F8
:10389000045059EF27F003067FEF27F0125002E1A2
:1038A00062EC26F01200CAEC26F012001200050E9F
:1038B00003601200125005E0035004C003F037EF1C
:1038C0008CF0336A3350C6EC16F044140FE003500A
:1038D000BEEC8CF0E150020FE96EE250040FEA6E8C
:1038E00004C0EFFF03C056F0B5EC3EF0332A33A41A
:1038F000E9D712001200120012000301EE6B036AF6
:1039000013EEF0F0E66AE66A032A03A6FBD701D8B5
:10391000F3D7F0DF0301EF6912000301EE6F12002D
:103920000301EE511200056E13EEF0F0E834FE0BC9
:10393000E126E750031804E1010EE350041809E002
:1039400003C0E6FF04C0E5FF0550C6EC16F0030116
:10395000EF13120003C004F0D8900436036AE3D7D3
:103960000F0EC16E036ED00E921603500F0B921005
:1039700003B8928AF80E96160338E830070B9612B1
:103980001200036E8950D00B046E03500F0B04100D
:1039900003B82009896E8D50F80B046E0338E830A7
:1039A000070B04108D6E1200E8B41AD0E8B20CD0E8
:1039B000E8B005D003B0898003A08990120003B05D
:1039C000898203A089921200E8B005D003B08984EF
:1039D00003A08994120003B0898603A0899612007F
:1039E000E8B20CD0E8B005D003B0898A03A0899A68
:1039F000120003B08D8003A08D901200E8B005D0B6
:103A000003B08D8203A08D92120003B08D8403A0B9
:103A10008D94120016511803F4CF1BF1F3CF1AF155
:103A200017511903F4CF1DF1F3CF1CF116511903EF
:103A3000F3501B27F4501C23E86A1D231751180369
:103A4000F3501B27F4501C23E86A1D231200E2DF09
:103A500019AF04D016511C5F17511D5B17AF04D06E
:103A600018511C5F19511D5B1200180E086E096A6F
:103A70000A6A180E086EF334F436F5360A3609363B
:103A8000F33607500A5E0650D8A0063C095ED8B04F
:103A9000F380F3B003D0092607500A26082EEBD78F
:103AA00012003E0EC06E0301E06BE16BF36A13EE91
:103AB000E3F0E66AF32AF3A6FCD7010EC26EC282D7
:103AC000120013EEE3F00301E051E126E750C45C7D
:103AD00002E2FF0A010F08E0FF0F06E0C4CFE7FF94
:103AE000E051C6EC16F0E113E029070BE06FE0357A
:103AF000E8341C0B0109C26EC28212000301F29E5F
:103B0000E151E16BE26FFF0BF28E27E0000EE2B1B4
:103B10001DD8010E0301E2B319D8020E0301E2B56C
:103B200015D8030E0301E2B711D8040E0301E2B960
:103B30000DD8050E0301E2BB09D8060E0301E2BD54
:103B400005D8070E0301E2BF01D807D0036E13EEBC
:103B5000E3F0E3CF04F057EF1CF012000601006B16
:103B6000010E096F0A6BF29EFF0EF66EFF0EF76EE6
:103B70003F0EF86E0900F550270A01E0008BF86A45
:103B8000F28E00BB120004EC16F00601036F12E186
:103B900016EE20F0010EE66E530EE66E490EE66E4E
:103BA000440EE66E200EE66E020EE66E000EE66E27
:103BB000000EE66E09690A6B0E6B16EE10F00F6BC5
:103BC000E66A0F2B0FA7FCD70F6B0601100E00172C
:103BD000800EB3D9400E776E000E706EC50E716EFA
:103BE000010E726E200E736E000E0F01606F506F2B
:103BF0000D01000EF86F0E01206B306B406B506BA7
:103C0000606B706B0D01030ED46FD56B0D01D86B1B
:103C10000D01700EE06FE16BE26BE36BE46BE56B43
:103C2000E66BE76B0D01F06BF16BF26BF36B03C6A8
:103C300005F60601046B076B086B000E1FEE00F023
:103C400062D903C604F61FEE04F0000E6CD90F0112
:103C5000FF0E186F080E196F1A6B1B6B000E6DD1DB
:103C600034EC1EF067EF1EF0060103512EE10E0545
:103C70003F0B0E6F2AE10F29070BD8B4010F0F6F0E
:103C800016EE10F00F51E35220E0E306ECD91DE1EF
:103C900006010F51C6EC16F009130FC605F6076BA7
:103CA000086B030E54D911E1000EE66E008DCCECCA
:103CB0001FF0009D0AE116EE10F00F51E36A0F515C
:103CC000036EDBEC41F0FF091200000B1200040050
:103CD000CAD9D8A412001FEE60F0E7BE1CD01FEEB8
:103CE00050F0E7BE18D01EEE20F0E7BE14D01EEE56
:103CF00030F0E7BE10D01EEE40F0E7BE0CD01EEE56
:103D000050F0E7BE08D01EEE60F0E7BE04D006011A
:103D100000B7DDD71200E1CF01F6E2CF02F6050EC3
:103D2000E3500F0B06010D6F020EE330700B046FB2
:103D300000A704D004390019070B0BE1020EE35071
:103D4000030B2FE0FF0F14E0FF0F22E026D0000E40
:103D500005D0020E03D0030E01D0FF0E01C6E1FF15
:103D600002C6E2FFE79E010F02E0FF0F96D8AFD731
:103D70007AD9F3E10F0130B7FBD72FEE35F0DCEC49
:103D80008BF01FEE31F0010ECED80F013087E5D752
:103D90002FEE35F002EC8CF0E1D7E79E000E90D8C4
:103DA000DCD7040EE350F00B16E1040EE35018E0EC
:103DB000FF0F1DE0FD0F1DE0FF0F1EE0FF0F2CE0C9
:103DC000FF0F38E0FF0F40E0FF0F4AE0FF0F54E025
:103DD000FB0F60E0C0D7040EE35055EC8BF0BED76C
:103DE0000087F80B00170439070B0013B0D70097B2
:103DF000AED72BEC1BF0ABD7040E0D63ACD7060E81
:103E0000E126E6CFE8FFE6CF03F0E6CF04F0E6CF09
:103E100005F0ADEC1BF09BD7030E0D639CD7060E8F
:103E2000E126E6CF03F0E6CF04F0E6CF05F001ECA3
:103E30001CF08DD7010E0D638ED7060EE126E650DD
:103E4000036E06EC1CF083D7020E0D6384D7060EBA
:103E5000E126E650036EE6CF04F03BEC1CF077D78A
:103E6000020E0D6378D7060EE126E650036EE6CF0C
:103E700004F040EC1CF06BD7030E0D636CD7060EFC
:103E8000E126E650036EE6CF04F0E6CF05F056ECEF
:103E90001CF05DD780EC19F05ED70601066FE3D801
:103EA0000DE10F0130B7FBD71FEE31F006010651CF
:103EB0003AD80F01356B3087060112000601120057
:103EC000D2D81FE10F0130B7FBD71FEE31F0000E43
:103ED0002AD81FEE35F0080EE66E010EE66E530E80
:103EE000E66E490EE66E440EE66E200EE66E020E9B
:103EF000E66E000EE66E000EE66E0F0130870601DC
:103F000012000601120005C6E7FFE69E030B080932
:103F1000E76E04C6E8FFE834E00BE61208C6E6FFE9
:103F200007C6E6FF120004C6E7FFE68E030B08098A
:103F3000E66EE66A05C6E6FF1200F36E6F501F0BD1
:103F4000F3106F6E6E50E00BF318FCE112000601E7
:103F5000066F0551C6EC16F0091511E084D80FE183
:103F60000F0140B7FBD70601065103C604F61FEE4A
:103F700041F0C9DF1FEE45F0000B06011200FF09FA
:103F8000060112000E01709F0F01408740A703D069
:103F90007450300BFBE01200F5DF05D0F3DF0E01AB
:103FA00070AFFDD70CD006010B6B0C6B06010B2B11
:103FB000D8B40C2B0CBB4ED00E0170AFF7D7060156
:103FC000009974CEE8FF056345D072CEE8FF030B7D
:103FD00005E0FF0F03E0FF0F37E03CD000AD35D028
:103FE00016EE20F00535E834E834380BE1260E01F2
:103FF00076CEE6FF77CEE6FF78CEE6FF79CEE6FF17
:104000007ACEE6FF7BCEE6FF7CCEE6FF7DCEE6FFF6
:104010007551080A13E1010E766310D0530E7763D1
:104020000DD0490E78630AD0440E796307D0200E74
:104030007A6304D0020E7B6301D007D006010551DC
:10404000C6EC16F00A1306D0A7D70E01709F000B1E
:10405000060112000E01709F06010551C4EC16F016
:104060000917FF091200060100BB0FD07450380B6E
:104070000EE06F880601008974AA06D0008B010E3D
:104080000917200E5ADF01D0A0DDFF091200000B36
:104090001200F36E16EE10F0E126080EE76EF350F4
:1040A000C4EC16F0060109171200000E436C6F6E87
:1040B000696E6720536C61766573400A416464726F
:1040C0006573733A20307800401157616974696EE6
:1040D0006720666F7220526573657400401021215D
:1040E0002121204641494C4544202121212106011E
:1040F0000351700BD8A4120082EC16F0AA0EF66ED3
:10410000400EF76E000EF86E9EEC16F0080EF36E81
:10411000FF0ECEEC16F0F32EFBD70400A5DD16EE55
:1041200011F0E650FAE1E650F8E1E650F6E1010E52
:104130000601056F0D0E88EC16F0200E94EC16F0BB
:1041400005C6E8FF98EC16F0BA0EF66E400EF76E54
:10415000000EF86E9EEC16F00601000E67D85BE1CB
:104160000F0E64D858E1000EF66E300EF76E000E9A
:10417000F86EF6500FE14A0E88EC16F0F85098EC05
:1041800016F0F75098EC16F0F65098EC16F0200E5A
:1041900094EC16F00400F6CF07F6F7CF08F6F830E7
:1041A00008330733D89008330733D89008330733E0
:1041B000020ECDDE30E1080EE66E0900F5CFE6FF17
:1041C000F650070BFAE1EADE26E1F850D2E0F650AD
:1041D000D0E1F750800ACDE1010E28D8C80EF66E66
:1041E000400EF76E000EF86E9AEC16F006010551BF
:1041F000066E040006504DDF37DD06010650056FE0
:10420000C6EC16F006010915F4E00601052B030EB5
:10421000056590D71200010E09D8DC0EF66E400E2F
:10422000F76E000EF86E9AEC16F0EFD7076F086B7A
:10423000000E8DDE03E1000EE66EAEDE120001031D
:10424000030001030400010305000103060001034C
:1042500007000109090001090A0001090B00010911
:104260000C0001090D000B0000000B0001000B0009
:1042700002000B0003000B00040003020200030213
:104280000400020001000200020004010100040217
:104290000300040608000409090004090A00FF00DD
:1042A0000000FF010000FF020000FF030000FF0408
:1042B000000004000200040D0D00040D0E000409AE
:1042C0000900040D0F0003030300030304000303AC
:1042D000050003030600030307000309090003099F
:1042E0000A0003090B0003090C0003090D00090073
:1042F0000000090001000900020009000300090094
:104300000400050303000503060004000100040087
:10431000020006000300060404000604050006046B
:10432000060006040700FF000000FF010000FF0276
:104330000000FF030000FF04000006000300060465
:104340000400060405000604060006040700030135
:104350000100030102000301030003010400030143
:10436000050003060600030607000306080003060F
:10437000090003060A00060000000600010006000E
:104380000200060003000600040000000000000018
:104390000000040001000400020000000000000012
:1043A0000000000000000000000000000000FF000E
:1043B0000000FF010000FF020000FF030000FF04F7
:1043C00000000000000000000000000000000000ED
:1043D00000000000000001030300010304000103CA
:1043E0000500010306000103070001090900010996
:1043F0000A0001090B0001090C0001090D00090068
:104400000000090001000900020009000300090082
:10441000040003030300030305000200010002007F
:104420000200040002000404040004040500040463
:10443000060004040700FF000000FF010000FF0267
:104440000000FF030000FF04000004000200040459
:10445000040004040500040406000404070004A08A
:10446000FCEC16F05DEC3EF0820EF66E300EF76E50
:10447000000EF86E0900F550066E0900F5CF07F042
:10448000F5100DE00900F55009000318F3E1F29E64
:1044900005000650FD6E0750FE6EF28E12001200EF
:1044A00004B0120010B6B2D20350DEEC16F0FF0ECC
:1044B00059EF27F004B0120010B6A8D20350DEEC7A
:1044C00016F0010E59EF27F0315004E004B012004D
:1044D00077EF20F02B9E04A02B8E04B0120010B6B4
:1044E000E5EFA0F02AEF2DF0090E11D0080E0FD045
:1044F000070E0DD0060E0BD0050E09D0040E07D006
:10450000030E05D0020E03D0010E01D0000E04B040
:10451000120010B67BD21EB480EF40F022240CEFC4
:104520002DF0010E05D0020E03D0040E01D0080EAE
:10453000066E1C8204B043D04450F00BF00A03E036
:104540000650441A04D0F00E44160650441237D8D0
:104550005DEC3EF02FEC3FF0E7507F0B2F6E36EC1A
:104560003FF0E750070B306E1F50C00B08E110EE14
:1045700068F010CBE8FF030B536E1FC0E3FFD0ECD5
:1045800041F06AEC3EF01F50C00B0CE110CBE8FF8D
:104590005318030B07E010EE68F010CBE8FF030B95
:1045A000E3501EDAF4EC2CF023DA44A007D010A478
:1045B00005D0F5ECA0F0108608EC25F012000638C6
:1045C000FF0A4416063804B04412120010B61ED278
:1045D0002B9004A02B801E9404A01E841C82120029
:1045E00004B0120010B612D22B7202D204B0120024
:1045F00010B60CD22B742B982BB42B880A0E266E77
:10460000F7D104B0120010B601D2000E44B0D5ECC0
:104610003FF0010E44B2D5EC3FF0020E44B4D5ECAD
:104620003FF0030E44B6D5EC3FF01C84120004B0FA
:10463000120010B6EBD14528030BD8B4010F456E1C
:104640001C84120004B0120010B6E0D1420EC5D195
:1046500004B0120010B6DAD110CBE8FFE8B223D0D4
:10466000E8B00FD0010E48B0020E48B2040E486EFA
:10467000000E48B2010E48B4020E476E4EEC2FF009
:10468000ACD14528030BD8B4010F456E010E486E1E
:10469000495003E0FF0F01E003D04EEC2FF09DD115
:1046A00058EC2FF09AD1E8B005D0010E486E4EECD0
:1046B0002FF093D1010E486E4EEC2FF08ED104B046
:1046C000120010B6A3D110CBE8FF030B020AD8B436
:1046D0001200010E036E000E046E4EEC2FF046EF3A
:1046E0002EF004B0120010B691D110CBE8FF030BEE
:1046F000020AD8B41200020E036E000E046E4EECD5
:104700002FF046EF2EF004B0120010B67FD1492AE8
:10471000030E4960496A49A24EEC2FF049B258ECA9
:104720002FF05BD9495002E1030E0CD049B209D0F9
:1047300010CBE8FF030B020A02E1060E03D0090EBC
:1047400001D0000E226E236E1C88C8EF29F004B041
:10475000120010CBE8FF030B000ED8A4010E036E6D
:10476000000E046E52EC2FF046EF2EF004B0120053
:1047700010B64CD110CBE8FF030B010ED8A4020EEB
:10478000036E000E046E52EC2FF046EF2EF004B0D4
:10479000120010B63BD110CBE8FFE8B212D0E8B05F
:1047A00008D0000E036E000E046E54EC2FF046EF9E
:1047B0002EF04528030BD8B4010F456E54EC2FF0B2
:1047C0000CD1E8B003D054EC2FF007D154EC2FF00B
:1047D00004D104B0120010B619D1070E036E030EF7
:1047E000046E54EC2FF046EF2EF004B0120010B619
:1047F0000DD14C06020E4CB24C6EFAD004B0120031
:1048000010B604D1000E036E000E046E50EC2FF0B3
:1048100046EF2EF004B0120010B6F8D0030E036E6F
:10482000000E046E50EC2FF046EF2EF004B0120094
:1048300010B6ECD010CBE8FF030B010A040ED8B47D
:10484000050E036E000ED8B4010E046E50EC2FF06E
:1048500046EF2EF010B6DAD004A009D01FAE02D079
:104860001C8212001C9C1C94266A1C961200010ECD
:10487000A8EF2EF010B6CAD004B0F0D7FF0EA8EF04
:104880002EF02BB0F0EF22F0E5D72BB0F6EF22F0B0
:10489000F1D704B0120010B6B9D02B7AA9D0000E0F
:1048A0000DD0010E0BD0020E09D0030E07D0040E5E
:1048B00005D0050E03D0060E01D0070E4F6E10B6C0
:1048C000A5D004A005D04F50C4EC16F05E1619D048
:1048D0005E5003E02B7AF8EC24F04F50C6EC16F053
:1048E0005E1210CBE8FFE8B216D0E8B00BD05C6ADD
:1048F0004E50C6EC16F05D1404E04EC04DF04F5023
:1049000079D812000BEE8CF04FC0EFFF94EC3EF024
:104910004FC02DF06DD0E8B00AD00BEE51F04FC073
:10492000EFFF94EC3EF04FC02DF062D01200120069
:10493000000E0DD0010E0BD0020E09D0030E07D0D1
:10494000040E05D0050E03D0060E01D0070E04A0FC
:1049500004D0C4EC16F05D1612004E6E4D6E10B60B
:1049600055D010CBE8FFE8B22CD0E8B021D04D50A4
:10497000C6EC16F05D125C6A4F50C6EC16F05E1481
:1049800002E04F5037D82BB003D056EC2FF025D093
:104990001E944E50FE0B01E005D04E504B6E54EC71
:1049A0002FF01BD04E50FE0F4A6E52EC2FF015D058
:1049B0000BEEDCF04EC0EFFF94EC3EF04EC02DF05D
:1049C00017D0E8B009D04DC050F0010E06D8020E45
:1049D000236E226AC3EF29F012001F6201D008D0B3
:1049E0001F6E236A226AD4EC2AF01C88C8EC29F0D6
:1049F0001C8412001C84566E0BEE00F025EC37F080
:104A00004550181A0BEE00F010EF37F010EFA1F040
:104A10005DEC3EF08FD810CBE8FF030B010A01E0FC
:104A200002D04550486E4950C6EC16F0070B066E92
:104A300010CBE8FF030B020A0CE0010E566E4DECA2
:104A400030F0EF38F00BEFB8000E0612EF38E83018
:104A5000030B2BAA08092BBA0409076E10CBE8FF39
:104A6000030B04E0030A02E0453804D04B50C6ECC7
:104A700016F0E838300B07124C50C6EC16F0E83A46
:104A8000E836E834C00B0712000E566E7EEC30F0AC
:104A9000EFCF08F04A50C6EC16F03F0B096E4550B8
:104AA000E83AE836E834C00B091210CBE8FFE8B268
:104AB00006D0E8B002D0000E07D0140E05D0E8B042
:104AC00002D0000E09D0140E566E91EC30F0EF3883
:104AD0000F0BDAD8EFA0000E0A6E0A503F0B1DB87C
:104AE00040091DBA40091DBC40091DBE40090A6E9F
:104AF0004CB20A8E360EF66E310EF76E000EF86E60
:104B00000900F550E96E0900F5CFEAFFF51011E054
:104B10000900F550C6EC16F0EF14D8A4010E036E90
:104B20000900F550F5AE60EC16F0F5BEB1EC26F0DC
:104B3000E7D7120010B6120010EE60F010CBE8FFBD
:104B4000E8B24BD0E8B027D01D962BBC120045B080
:104B500011D005CCE6FF0DCCE6FF15CCE6FF1DCC51
:104B6000E6FF25CCE6FF2DCCE6FF35CCE6FF3DCCBD
:104B7000E6FF120004CCE6FF0CCCE6FF14CCE6FF07
:104B80001CCCE6FF24CCE6FF2CCCE6FF34CCE6FFC1
:104B90003CCCE6FF120044B012001D966AD80B010F
:104BA00070A30FD08C51F80B0CE18C51C6EC16F0B1
:104BB000076E10EE60F0080E066E07C0E6FF062EC8
:104BC000FCD7C0A309D0DC51F80B06E110EE60F071
:104BD000DC51070BE126E7681200E8B017D044B0BB
:104BE00012001D9646D80B0150AD0FD05151F80B55
:104BF0000CE15151C6EC16F0076E10EE60F0080E95
:104C0000066E07C0E6FF062EFCD7120044A003D0B4
:104C100030D82BBC12001D964650080D420EF324CE
:104C2000F66E4C0EF420F76EF86A000EF82210EEC5
:104C300060F0080EF36E0900F5CFE6FFF32EFBD708
:104C400012000040447F7F40400000627351494F92
:104C5000460000226349497F360000181814167F69
:104C60007F1000276745457D3900003E7F49497325
:104C7000320010EE60F020EEE8F0F36AE66ADE6AD9
:104C8000F32AF3A6FBD712000F0BC8EC16F0010CA9
:104C9000020C040C080C100C210C220C240C280C07
:104CA0001F0C1F0C1F0C1F0C1F0C1F0C1F0C00EEE9
:104CB000D0F010EED8F0F36AEE68E66AF32AF3A6B5
:104CC000FBD712005B28070B5B6ED8B45C2A5B50E5
:104CD000C6EC16F0036E020E68EC16F010B602D0A9
:104CE0001DA61CD010EEE8F05B500708E126E75047
:104CF000D8A4E706E75011E0AA0EF66E4E0EF76E46
:104D0000000EF86EE730E830E830070BF626000EAC
:104D1000F722000EF8220900F5500AD02BBC03D070
:104D200010EE60F002D010EEE8F05B500708E350A0
:104D3000036E5C50380B09E15E50031A5B500708A4
:104D4000C6EC16F05D14D8A4031E000E68EC16F035
:104D500020EEE0F05B50DBCF03F0010E68EC16F0C4
:104D6000120010EEE0F003B001D00AD0036EE83676
:104D7000E838070BE1260350C6EC16F0E7121200E4
:104D8000036EE836E838070BE1260350C4EC16F052
:104D9000E71612005B04070B0B6E040E5CEC16F0BA
:104DA000100EE126E76A10EED0F00B50E3CF0CF0C6
:104DB00003C0E3FF10EED8F00B50E1260C500318AF
:104DC000E712120000016C6B10EED8F06C51E12676
:104DD000E75010E0E7B013D8E7B214D8E7B415D81D
:104DE000E7B616D8E7B817D8E7BA18D8E7BC19D885
:104DF000E7BE1AD86C2B070E6C65E6D71200E79059
:104E0000000E14D0E792010E11D0E794020E0ED0DE
:104E1000E796030E0BD0E798040E08D0E79A050E2C
:104E200005D0E79C060E02D0E79E070E036E6C3994
:104E3000E830380B8009031210EED0F06C51E126F7
:104E40000350C6EC16F0E714D8A4010E046E2FEC44
:104E500022F010EED8F000016C51E126120010EEA5
:104E6000E8F0E126800E03260350F00B800A02E1F1
:104E7000E76A12000338E8A604D0E8B4070E040974
:104E800003D0E8A4000E030B070BA20FF66EF76A1F
:104E90004E0EF722F86A000EF8220900F5CFE7FF60
:104EA000120078381808080C0E0F80C0E0F0F8FCEB
:104EB000FEFF586E10B610EFA1F01CBCA6EF2EF04E
:104EC0001EB41C821E941FBE01EC2DF010EE18F0D3
:104ED0001AC003F01BC004F05850DCEC16F003A01D
:104EE00012001FAE07D02BAE37EF2DF018C011F017
:104EF00035EF2DF01CA87BEF2DF083EF2DF0045043
:104F0000586E056E10B610EFA1F01EB41C821E94F0
:104F10005DEC3EF0040E036407D0060E03640AD075
:104F2000080E03640AD00CD0035049B0050F49B2F3
:104F30000A0F0CD003500A0F09D003500A0F06D0F5
:104F400003500A0F4CB0050F4CB20A0FF56E10CB90
:104F5000E8FF030B880D3E0EF324F66E420EF4209C
:104F6000F76EF86A000EF822F534E834FC0BF626EA
:104F7000000EF722000EF8220900F550066E1AE026
:104F80000900F5CF04F00900F5CF03F0062803E08F
:104F9000065089EF2EF01F507F0B0CE004500F0BD2
:104FA0002224036E2450036005D022C004F01F5059
:104FB00089EF2EF01200252E12007A0E256E275052
:104FC000D8A42706D8A41200262A40507F0BD8A4C4
:104FD000400641507F0BD8A4410642507F0BD8A415
:104FE000420643507F0BD8A44306315003E03104FE
:104FF00001E031062BB402D01FBE12002B982BB457
:105000002B882650040A04E02650140A04E01200FB
:105010001C861C841200266A1C962BA402D02BB678
:105020002B981C841200EF0FD8B0EF0E110FC8ECB4
:1050300016F010D010D017D029D00FD1FCD001D14C
:1050400006D121D12BD12FD13FD178D19CD12FD0D6
:1050500076D0C1D012001CA8236A1CA8226AE9508D
:105060007F0B96D112001CA8236A1CA8226A5DEC53
:105070003EF02FEC3FF0E7507F0B2F6E36EC3FF009
:10508000E750070B306E5AEC2FF082D11CA8236A30
:105090001CA8226A11C02EF0460E7AD140102D2D88
:1050A0002D2D2D20434F5059202D2D2D2D2D1D847C
:1050B00010CBE8FF030B020A1AE013EE80F00CEEAF
:1050C00000F02D38700BE912566A5650EBCFE3FF13
:1050D000100EE126800EE9265650EBCFE3FFF00ECE
:1050E000E126800EE926562A56A8EFD70ED013EEF9
:1050F00080F00CEE00F02D50200DF350E926566A9A
:10510000EECFE6FF562A56AAFBD79C0EF66E500E3F
:10511000F76E000EF86E0AD1120040102D20427575
:105120006666657220456D707479202D40102D2DB6
:105130002D2D205041535445202D2D2D2D201DA4C3
:105140003AD010CBE8FF030B020A1CE00CEE00F093
:105150002D38700BE912566A13EE80F05650E3CFEB
:10516000EFFF94EC3EF0800EE92613EE90F05650DF
:10517000E3CFEFFF94EC3EF0810EE926562A56A8C5
:10518000EBD712D00CEE00F02D50200DF350E92695
:10519000566A13EE80F05650E3CFEFFF94EC3EF0EA
:1051A000EE50562A56AAF5D72C0EF66E510EF76E13
:1051B000000EF86EBBD01A0EF66E510EF76E000E92
:1051C000F86EB4D040102D2D2D2D20436C656172EA
:1051D000202D2D2D2D2010CBE8FF030B020A16E009
:1051E0000CEE00F02D38700BE912566A800EEF6E4F
:1051F00094EC3EF0800EE926400EEF6E94EC3EF00B
:10520000810EE926562A56A8F1D70ED00CEE00F0F2
:105210002D50200DF350E926566AEF6A94EC3EF0CB
:10522000EE50562A56AAF9D7C40EF66E510EF76EF6
:10523000000EF86E7BD011D824502360120066EF68
:105240002BF00BD82450236012007FEF2BF005D8F1
:1052500024502360120086EF2BF0245023601200AC
:105260001C88266A1C961C84D3EC2DF0040EA9EC35
:105270002DF00900F5CF1AF00900F5CF1BF0000E54
:1052800073DBF4EF2CF0245023601200E6DF182AC1
:105290001A281860186A83EC2DF07CD056503EEC2A
:1052A0005AF079EF3FF04650F2EC5AF00BEE60F016
:1052B00046500A0DF350E9260A0E066E94EC3EF0B5
:1052C000EE50062EFBD712002FC013F030C014F0A2
:1052D000145013100AE0ACEC5EF007E01A0EF66E04
:1052E000530EF76E000EF86E21D0326A1C8A2DEF35
:1052F00029F0080EF66E530EF76E000EF86E16D8F3
:1053000015EC2EF01C98AFD640102D2D2053617651
:1053100065205061746368202D2D40102D206E6F24
:105320007420706F737369626C65202D9AEC16F0AF
:10533000180E53EC4FF0400EFAEF16F02E5004E02A
:1053400007EC5FF001E0CAD7600EF66E530EF76E01
:10535000000EF86E10D82EC011F0F6EC2DF096D697
:1053600040132D2D205361766520456E73656D6267
:105370006C65202D2D009AEC16F0150E53EC4FF0B5
:10538000400EFAEF16F0326A1E801E922DEF29F0C1
:105390001CA80BD01C981C9A1E901C9E1C84266A6C
:1053A0001C96000EE1DA20DB0FD31F6E1C82000E6C
:1053B000DBD2800EEDD71CA8236A1CA8226A000E3F
:1053C000E7D71CA8236A1CA8226A400EE1D7800EEA
:1053D0001F6E180E316EF10E446E030E456E2B9A41
:1053E00057EC26F0120050EC41F03150D8A41200D6
:1053F0005DEC3EF0D0EC42F0D8A412001DA203D028
:105400001D926AEF3EF0C5EC3FF0F29E2B9C2BBA4A
:105410002B8C5E50D8A42B9CF28E1CA21FD01C9209
:105420001C84266A1C961C9C1C9ECFDB1EB408D0D4
:10543000BBD85DEC3EF0000E97DAD6DAC5DA286A02
:105440001C808DEC41F01CA012001EB407D01FAED2
:1054500005D0450E88EC16F085EC4FF01CA008EF47
:1054600025F02750D8A41200285005E11CA41200F2
:105470001C9408EC25F01EB4A8D01FAE8BD01CBC29
:1054800088D05DEC3EF0285007E0FF0F19E0FF0FD9
:1054900021E0FF0F2BE044D0050E88EC16F036EC2F
:1054A0003FF0146E2FEC3FF0136E66EC4FF0ACEC57
:1054B0005EF0200ED8A42A0E94EC16F0282A69D0AB
:1054C000000E88EC16F057EC4FF07C0E94EC16F0C2
:1054D000282A5FD00A0E88EC16F010CBE8FF73EC98
:1054E0004FF0020E53EC4FF0282A53D00E0E88ECEA
:1054F00016F0430E94EC16F0680E94EC16F06E0E57
:1055000094EC16F02E0E94EC16F010EE3CF03350A6
:10551000030BE126E7287F0B90EC16F0282A39D000
:10552000400E88EC16F009C6F3FF2D0E1DB8500E84
:1055300044A003D0310E1DB8020EF3A02A0E94EC45
:1055400016F02D0E1DBA500E44A203D0320E1DBA15
:10555000030EF3A22A0E94EC16F02D0E1DBC500E75
:1055600044A403D0330E1DBC040EF3A42A0E94EC05
:1055700016F02D0E1DBE500E44A603D0340E1DBED7
:10558000050EF3A62A0E94EC16F07C0E94EC16F0A1
:10559000286A12000C0E00A684EC16F00400020E1D
:1055A0006BEC2FF0CCEF16F01FBE1200000E6BEC70
:1055B0002FF0C2EC16F0F86A0900F5CF24F00900CC
:1055C000F6CF20F0F7CF21F0FFD1285003E10BEC0C
:1055D00040F002D023EC40F0282A010E286412008B
:1055E000286A1200000A456E73656D626C653A2088
:1055F000285028E11CBC26D01FAC15D0E40EF66E56
:10560000550EF76E000EF86E9EEC16F057EC4FF04C
:1056100007EC5FF0200ED8A42A0E94EC16F0050ECD
:1056200053EC4FF00FD0000E88EC16F05DEC3EF01E
:1056300085EC4FF036EC3FF0146E2FEC3FF0136E1C
:1056400066EC4FF0400E1FEC2CF0282A2850050A7B
:10565000D8A41200400E0ED9286A12001CBA75D0C8
:105660001EB0A1D01CBC05D01CBE03D0000E1FEC88
:105670002CF01CBE03D0400E5CEC2CF0282A2850E5
:10568000050AD8A41200000EF5D8286A00B6120048
:105690001CA812002450236012001CBE12002250CD
:1056A000235C040DF350420F88EC16F00E0E00A69A
:1056B00084EC16F012000014506172616D6574651F
:1056C000722041737369676E2E3A20201C8EB60ECD
:1056D000F66E560EF76E000EF86E9EEC16F0400E4B
:1056E00088EC16F01850EDEF4FF00007506174632E
:1056F000683A2000000742616E6B3A202000F40EE9
:10570000F66E560EF76E000EF86E07D0EA0EF66EC5
:10571000560EF76E000EF86E00D01C8E9EEC16F042
:105720005DEC3EF036EC3FF0146E2FEC3FF0136E64
:1057300066EC4FF0090E53EC4FF0400E88EC16F07B
:10574000D4EC4FF0040E53EF4FF01CBC07D0000E0A
:1057500088EC16F085EC4FF0180E30DA1CB606D047
:10576000325088EC16F0200E94EC16F0900EF66E87
:10577000570EF76E000EF86E9EEC16F000B6120093
:10578000325088EC16F00E0E00A684EC16F01200D3
:1057900040145341564520203C2020203E202044E8
:1057A000656C20436C721CBC21D0000E88EC16F096
:1057B000DCEC3CF0200E94EC16F01EB20CD02D2840
:1057C0008EEC16F05F0E94EC16F05050070B010FA4
:1057D0008EEC16F009D0520E94EC16F06F0E94EC8D
:1057E00016F0740E94EC16F0140EE8D91EB208D020
:1057F0001CB606D0325088EC16F0200E94EC16F051
:10580000280EF66E580EF76E000EF86E9EEC16F02F
:1058100000B612001EB21200325088EC16F00E0EC6
:1058200000A684EC16F01200401447415320526F3A
:105830007420526E6420436C722044524D20066ED8
:105840002850040DF350061088EC16F0A1D928500A
:105850000A0DF3502926F4502A2222502824010F41
:10586000246003D0040EAAD904D050D8200E94ECA2
:1058700016F01200130F88EC16F01CB81AD0060EA2
:10588000246002D0200E16D0225009E02450FB0FD5
:1058900022620AD000A6000E00B6080E0BD000A6A9
:1058A000010E00B6090E06D000A6070E00B6090EBE
:1058B00001D0200E94EF16F0066E2850040DF35020
:1058C000061088EC16F064D928500A0DF3502926EA
:1058D000F4502A2222502824010F246007D05AECC9
:1058E0002FF01F1812E0040E69D90FD0225028247F
:1058F000236207D01CB605D01CA803D0040E5ED9C5
:1059000004D02ED8200E94EC16F01200010E21D9EE
:105910000800240EF5621BD0240E1DA094EC16F096
:1059200022042824566EFDEC30F00AE13C0E94EC83
:1059300016F02D0E1DB094EC16F03E0E94EF16F0FE
:10594000E950800F1DB092EF16F098EF16F0030E9D
:10595000066E0900F55094EC16F0062EFAD71200E8
:10596000FFD80350C4EF37F0F36EFF0B12E11FBEF8
:1059700007D01CB80ED0010E036EF35074EF16F072
:10598000020E046E020E2BB0010E036EF35074EF84
:1059900016F01A50066EE00B1B1007E1000E056EA4
:1059A000010E036EF35074EF16F01B50076E0636AF
:1059B0000736050E076407502BA0020F046E020E77
:1059C000036EF35074EF16F01CB812001FBE08D01F
:1059D00024042450FB0FD8A0000E1A6E1B6A12007C
:1059E0007F0E1A6E1B6A12001CA805D0DCD8B8D82E
:1059F000055061EF31F01FBE04D02250186E196AB5
:105A000012002BAE02D0115004D05DEC3EF02FEC12
:105A10003FF0186E196A12001CA012001CBE120082
:105A20001CBA75D21EB0CFD21FAE06D0FF0BD8B4B1
:105A3000E1EF29F0DBEF29F0236E186E276A1C8452
:105A4000266A1C96245023601200ADD889D80450D1
:105A500013EF28F01CA01200276A286A1FBE12004C
:105A6000040E6BEC2FF0CCEF16F03DEF51F032D876
:105A70005DEC3EF036EC3FF0146E18507F0B136E69
:105A8000336A3350C6EC16F0441416E02FEC3FF0A6
:105A900013C0E7FF36EC3FF014C0E7FFBEEC3FF069
:105AA00000EE81F013C0EFFFABEC3EF000EE80F0B3
:105AB00014C0EFFFABEC3EF0332A33A4E2D75DEC29
:105AC0003EF0120007D82FEC3FF018507F0BE76E26
:105AD000BEEF3FF02BA412002BA612002B965DEC1C
:105AE0003EF02FEC3FF0E7507F0B2F6E36EC3FF08F
:105AF000E750306E9AD018503F0B236E226E1C84F4
:105B0000266A1C9612004FD82B86336A3350C6EC97
:105B100016F0441404E026D805505FEC31F0332A27
:105B200033A4F4D71DD80350550A09E00C0A07E046
:105B3000690A05E0380A07E00F0A03E005D0C6DD70
:105B400003D0DDDD01D0E2DD1C840A0E266E1C864A
:105B500012002924F66E000E2A20F76EF86A120051
:105B60005DEC3EF00BEE00F029C0F6FF2AC0F7FF17
:105B70000900F550566EE926060EEBDF0900F5CF59
:105B800003F00900F5CF04F00900F5CF05F012008D
:105B900020C029F021C02AF022500A0DF3502926F6
:105BA000000E2A22120020C029F021C02AF0235022
:105BB0000A0DF3502926000E2A221200066E200E2E
:105BC00094EC16F0062EFBD71200475002D8486E10
:105BD0001200F90FD8B0F90E070FC8EC16F0010C3F
:105BE000020C040C030C050C060C070C07EC5FF010
:105BF0001BE12EC011F0336A335003E1FCEC51F08D
:105C000009D01CEC43F009C6F3FF3350C6EC16F084
:105C1000F31403E03350CBEC51F0332A33A4ECD728
:105C200033EC52F08DEC3EF012005DEC3EF02FC0F4
:105C300013F030C014F0ACEC5EF024E1A96AAA6A5B
:105C400004001BEE00F0A950E126AA50E222C2ECAB
:105C50005EF0A950F5E1010EAA64F2D72FEC3FF0F7
:105C600013C0E7FF36EC3FF014C0E7FF00EE81F011
:105C700013C0EFFFABEC3EF000EE80F014C0EFFF7E
:105C8000ABEC3EF012002B861C8412001CA012000C
:105C90000A6E1FC053F023C055F022C054F01F6E8F
:105CA00083DC03C023F004C022F02DEC29F018504F
:105CB0001A64FF0E010F186E26DFC8EC29F053504E
:105CC0000A1807E153C01FF06FDC54C022F055C022
:105CD00023F01C8412001CA012000A6E1FC053F097
:105CE00023C055F022C054F01F6E5EDC03C023F0C9
:105CF00004C022F02DEC29F0187005DFC8EC29F063
:105D000053C01FF051DC54C022F055C023F01C8456
:105D100012001CA0120005C00AF01F6E45DC03C073
:105D200023F004C022F02DEC29F010EE18F01AC078
:105D300003F01BC004F00A50DCEC16F003B0E3DE05
:105D4000575012DECAEC29F01C841200039001D0D7
:105D50000380066A062AE8BE06681FAE04D0130E4A
:105D60002BBE110E07D0090E6BEC2FF00900F55079
:105D7000D8B486D0E96EEA6A130A03E12FEC3FF04B
:105D8000136E0900F5501FBE7F0E076E03B00CD0D6
:105D90000650EF2606BE04D00750EF60EF6E10D01D
:105DA0000750EFBEEF6A0CD00650EF2606BE05D0B6
:105DB0000750010FEF60EF6A03D00750EFBEEF6EA0
:105DC0001FBE1AD00B0E6BEC2FF00900F5500D0A18
:105DD00003E01F0A06E010D0E5EC2DF000EE48F0DD
:105DE0000BD006BE04D0EF50D8B4EF2A05D0EF5048
:105DF000D8B4EF04030BEF6E1EB04BD0E950130A7A
:105E000003E0020A05E006D013C018F030DE41D0EE
:105E10002CDE3FD0000E88EC16F05B0E94EC16F0F2
:105E2000060E6BEC2FF0030E9CEC16F00B0E6BECD9
:105E30002FF00900F550100A0BE1080EEF6404D0B2
:105E4000EF2890EC16F00AD0EF288EEC16F006D072
:105E5000200E94EC16F0F550C4EC37F05D0E94EC87
:105E600016F0200E94EC16F00C0E00A684EC16F042
:105E70000FD0000C5B4E6F742068657265215D2049
:105E8000720EF66E5E0EF76E000EF86E9EEC16F059
:105E90001C8C1C841CA812002DEF29F0000E0BD0C6
:105EA000040E09D0080E07D00C0E05D0100E03D03A
:105EB000140E01D0180EF36E10CBE8FF030BF32481
:105EC000900FF66EF76A880EF722F86A000EF82235
:105ED0000900F5501200E16E10CBE8FF030B1FBC68
:105EE000040E020DAC0EF324F66E880EF420F76E4D
:105EF000F86A000EF822C2EC16F0F86A1F503F0B49
:105F00000C0DF350E124F626F450F72212001CA0E9
:105F10001200066E2250065E276A1C84266A1C96B2
:105F20005DEC3EF00650FA0FD8B0FA0E060FC8EC42
:105F300016F005D008D00BD00ED039D022D0CAEC44
:105F400029F079EF29F032040F0B326E39D0322864
:105F50000F0B326E35D00BEE00F0000EE9263250FA
:105F6000066E0F0E06600AD00628EBCF07F006502B
:105F700007C0EBFF062A0E0E0664F6D70F0EEB6A7B
:105F80001FD00BEE00F0000EE9260E0E066E065036
:105F9000EBCF07F0062807C0EBFF0606062803E054
:105FA00032500660F4D73250EB6AEB8A09D00BEE20
:105FB00000F0000EE926066AEE6A062A06A8FCD75B
:105FC000CFDD05507ED1066E2250065E276A1C8406
:105FD000266A1C965DEC3EF00650FB0FD8B0FB0E17
:105FE000050FC8EC16F004D029D02CD03ED048D0F4
:105FF000FDEC30F0020E32B6E9263250C6EC16F057
:10600000066E076AEE500614D8A40780ED500614F9
:10601000D8A407820728030B076E061CEF1607A0FB
:1060200002D00650EF12EF5033D8061CEF1607A22D
:1060300002D00650EF12EF502BD829D01E72326AD0
:10604000186A25D0FDEC30F0DCEC59F00CC1E8FF0B
:106050001FD80DC1E8FF1CD8DCEC59F00CC1E8FFDB
:1060600017D80DC1E8FF14D812D0FDEC30F0000EA7
:106070000FD8000E0DD8000E0BD8000E09D807D08F
:106080001E90D8905034466E030EEDEF24F01200AF
:10609000EF6E94EC3EF0EE50120010CBE8FFE8B249
:1060A00015D0E8B00CD00BEE00F0B00E48B2A00E48
:1060B00048B0900E45B0D00F5624E92612000BEEE2
:1060C000B0F0565045B0B00FE9261200E8B00BD042
:1060D0000BEE60F05650E92646500A0DF350E926C3
:1060E000F450EA2212000BEE60F05650E9264650BA
:1060F000300DF350E926F450EA22120010CBE8FFED
:10610000E8B20BD0E8B008D00BEE00F05A0E45B064
:10611000540E5624E9261200F7D7E8B001D0F4D780
:10612000F3D710CBE8FFE8B211D0E8B008D00BEEFF
:10613000C0F04A50050DF3505624E9261200BFDF87
:106140004A50010B070DF350E9261200E8B001D0C8
:106150001200C9DF4A50010B070DF350E926120067
:1061600010CBE8FFE8B20BD0E8B008D00BEEE0F0BF
:106170004B50100DF3505624E9261200A0D7E8B07A
:1061800001D01200B0D70CEE00F04D50080DF350C6
:106190005624E92612000CEE00F04D50080DF35085
:1061A000040FE92612000CEE40F05050030DF3509E
:1061B00056B6010F56B8020FE92612000BEE18F082
:1061C0005150050DF3505624E926120010CBE8FF7C
:1061D000E8B20BD0E8B008D00CEE6CF05250050DD0
:1061E000F3505624E92612006AD7E8B005D00BEE2A
:1061F00000F056C0E9FF120076D710CBE8FFE8B2F6
:1062000015D0E8B00AD05650030B050D1CEE6CF00B
:10621000F350E126F450E22228D00CEE00F02D38A5
:10622000700BE9262C500F0BE9261200E8B00CD0B9
:106230000CEE00F02D50200DF350E9265050070BC6
:10624000040DF350E926120056C0F5FF46C0E1FFE9
:1062500056C046F02B0E566E46DFF5CF56F0E1CF16
:1062600046F0E9CFE1FFEACFE2FF020EE3507F0BF9
:10627000F36E030EE3507F0BF46E2C507F0BF3266E
:10628000F428F36009D00BEE00F0F350800FE96EB4
:10629000010EEA22FF091200000B120000EE80F04E
:1062A0005650E926120000EE80F0030EE926120097
:1062B000F5DF4650080DF350100FE9261200040DCB
:1062C00003D0040D020EF32609EC37F0C3D0C2D080
:1062D000C2D0C5D0C7D0CCD0D0D0D1D0D4D0F6D0B9
:1062E000F7D0FAD0FBD0FDD0FFD017D126D129D1DD
:1062F0002BD12DD12FD132D133D139D13CD142D173
:1063000045D14BD14ED150D152D15BD160D168D162
:106310006FD176D17AD17CD17ED184D187D189D108
:106320008BD18DD18FD191D193D195D197D19CD152
:106330009FD1A6D1AAD1B0D1B3D1B5D1B7D1B9D15E
:10634000BBD1BDD1BFD1C1D1C3D1C5D1C7D1C9D1B5
:10635000CBD1CDD1CDD1CFD1CFD1D3D1D5D1DBD12F
:10636000DED1E0D1E2D1E4D1E4D1EAD1F8D103D257
:1063700009D20CD207D20AD2E7D1EDD10CD20ED27B
:1063800010D212D20ED210D212D213D214D21ED2E6
:1063900024D22DD236D238D23BD23DD240D242D2B4
:1063A00045D246D248D24ED252D258D25CD25ED2D8
:1063B0004ED254D25FD261D263D26CD271D277D234
:1063C0007BD27ED281D284D287D287D287D287D223
:1063D00087D291D291D296D296D29BD29BD29CD286
:1063E0009DD29ED29FD2A0D2A1D2A9D2AFD2B8D2F2
:1063F000BFD2CBD2D2D2D6D2D8D2DCD2DED2EFD25A
:10640000FCD2FFD202D306D308D310D317D31ED3A6
:1064100022D325D328D32BD32ED335D339D341D36D
:1064200046D346D34BD34FD353D353D353D358D35D
:106430005BD360D363D36FD377D377D377D37DD355
:1064400082D38BD38FD399D3A7D3B6D3C1D3C8D399
:10645000CED3D3D3120018C0EFFF4AEF36F0EF507F
:106460000AEF36F018C0EEFF19C0EDFF4AEF36F024
:10647000EECF18F0EDCF19F0120006EF36F002EC77
:1064800036F00AEF36F009C6F3FF335018640CD02B
:106490001850C6EC16F0F31412E11828030B186E0E
:1064A000F2E13350186E0BD01850C6EC16F0F3140E
:1064B00006E11804030B186E030AE5E1F2D7185041
:1064C000C6EC16F0F009446E1D8212003350A2D3C0
:1064D00018C047F0E5EF2DF047509CD31828456EC3
:1064E00012004504030B96D34EEC31F045B007D8AB
:1064F000040E56264EEC31F045B201D81200183881
:10650000F00BEE6E18380F0BEF6E1938F00BED1222
:10651000ABEC3EF0E92AABEF3EF04EEC31F0000E72
:1065200045A0040FE926EE380F0B186EEF38F00B7C
:106530001812EF380F0B196E1200325018C0EBFF13
:1065400012003250EB5066D31EB275D396D71EB2EE
:10655000120095D7C5DB18C0EFFF9CD39EDD7FD717
:10656000BFDB0F0EEF161838F00BEF1293D395DD4B
:10657000EF380F0B4FD3B4DBF00EEF1618500F0BA4
:10658000EF1288D38ADDEF500F0B44D3A9DBFC0E4A
:10659000EF161850030BEF127DD37FDDEF50030B86
:1065A00039D39EDB020E78D378DD020E3DD398DB23
:1065B00018C0EFFF6FDBEE5019C0EFFF6BDBED5043
:1065C00012006BDDEECF18F0EDCF19F0120088DB72
:1065D000E00EEF161850EF121850D8B4EF885AD3C7
:1065E0005CDDEF50070BEFB6080EEFB8000E12D3CC
:1065F00077DB1F0EEF161838E834600BEF124AD322
:106600004CDDEF38E830030B05D36ADB000E44D3D2
:1066100044DD000E09D364DBF10EEF1618340E0BC7
:10662000EF1238D33ADDEF30070BF4D259DB040E0A
:1066300033D333DD040EF8D253DB050E2DD32DDD1D
:10664000050EF2D24DDB060E27D327DD060EECD267
:1066500047DB070E21D321DD070EE6D241DBE00E3A
:10666000EF161850EF1216D318DDEF501F0BD2D2D1
:1066700037DB1F0EEF161838E834E00BEF120AD3A1
:106680000CDDEF38E830070BC5D22ADBC00EEF1661
:1066900018503F0BEF12FED200DDEF503F0BBAD285
:1066A0001FDB070EF9D2F9DC070EBED219DB040E90
:1066B000F3D2F3DC040EB8D213DB030EEDD2EDDC23
:1066C000030EB2D20DDB000EE7D2E7DC000EACD237
:1066D00007DB010EE1D2E1DC010EA6D201DB020EE6
:1066E000DBD2DBDC020EA0D235DFF4EF3FF036D791
:1066F00031DF02EF3FF032D7F3DA050EEF12010E71
:10670000CBD2CBDC010E90D2EBDAC00EEF161850D4
:106710003F0BEF12BFD2C1DCEF503F0B7BD2E0DA70
:10672000070EBAD2BADC070E7FD21ADFF4EF3FF0C1
:106730001ED7BCDAF80EEF161850070BEF12AAD2CC
:10674000DDDCEF50070B66D2B1DA8F0EEF1618388A
:10675000700BEF129FD2D2DCEF38070B5BD2A6DAB8
:1067600018C0EFFF97DAEE50F00EEF161950EF1247
:1067700091DAED501200C2DCEECF18F0ED500F0BA5
:10678000196E120093DA1850EF6E84D2B7DCEFCF97
:1067900018F0196A12008ADA030E7ED2AFDC030EFB
:1067A00043D284DA070E78D2A9DC070E3DD2E3DAB1
:1067B00052D6B7DC54D6DFDA0E0EEF161804E838DE
:1067C000F00BEF121850D8A4EF8064D2AADCEF3897
:1067D0000F0B010FEFA0000E1DD2CDDA4A50562646
:1067E00050C00AF0506A42DB0AC050F012004A5012
:1067F000562650C00AF0506A45EC37F00AC050F0F7
:106800001200B9DA010E48D291EC30F0010E0CD230
:10681000B2DA030E41D291EC30F0030E05D2ABDABE
:10682000020E3AD291EC30F0020EFED1D0DA13D63D
:10683000B0EC30F014D6CBDAF80EEF161850070B88
:10684000EF1228D2B0EC30F0EF50070BE3D1BFDAF3
:106850008F0EEF161838700BEF121CD2B0EC30F020
:10686000EF38070BD7D1B3DA070E16D2B0EC30F001
:10687000070EDAD1C3EC30F0EED5C3EC30F0EFD533
:10688000C3EC30F01850E10FE8BE03D0800FEF6E7C
:1068900001D2E1D5C3EC30F0EF50EFBE9E0FBAD17C
:1068A000C3EC30F0F00EEF161850EF12F3D1C3EC3A
:1068B00030F0EF500F0BAED1C3EC30F0060EECD140
:1068C000C3EC30F0060EB0D1C3EC30F0070EE4D1CB
:1068D000C3EC30F0070EA8D1A3D2B7D2C7D2D5D21D
:1068E00003D9465007E110EE3CF03350030BE1268C
:1068F00018C0E7FF1200FED0EDD836EC3FF018C00C
:10690000E7FF8BD9EDD0E6D82FEC3FF018C0E7FFBA
:1069100084D9E6D0000EC0D1000E86D1010EBCD1C4
:10692000010E82D1020EB8D1020E7ED14EEC31F0B2
:106930001850320FD8B0FF0EEF6EABEF3EF04EECBA
:1069400031F0EF50CE0FD8A0000E64D14EEC31F0F4
:10695000FC0EEF1618B0EF8018B2EF82ABEF3EF0EE
:106960004EEC31F0000EEFB00109EFB2020952D146
:106970005650BEEC8CF0E150020FE96EE250040F6D
:10698000EA6E18C0EFFFB5EF3EF05650BEEC8CF04B
:10699000040EE226020EE3503DD1DEEC30F05BDD6A
:1069A000FAEF3EF0DEEC30F05AD5DEEC30F053DD9D
:1069B00002EF3FF0DEEC30F052D51938F00BF46EF8
:1069C00018380F0BF4121838F00BF36EF3CFEFFFFB
:1069D00061D9EE50F4CFEFFF5DD9ED501200EECF4C
:1069E000F3FFEDCFF4FFF4380F0B196EF438F00B12
:1069F000186EF3380F0B18121200140EE96E565071
:106A00004BD1140EE96E56500FD1E6EC30F023DD79
:106A100002EF3FF0E6EC30F022D5E6EC30F0EF9CF0
:106A2000EF9E18B0EF8C18B2EF8E34D1E6EC30F058
:106A3000000EEFBC010EEFBE0209ECD0E6EC30F028
:106A4000C00EEF1618503F0BEF1224D1E6EC30F0D9
:106A5000EF503F0BDFD0E6EC30F0060E1DD1E6EC38
:106A600030F0060EE1D0E6EC30F0070E15D1E6EC82
:106A700030F0070ED9D0E6EC30F0800EEF1618504B
:106A80007F0BEF1207D1E6EC30F0EF507F0BC2D056
:106A9000E6EC30F018047F0B1852D8B4800EEF6E7D
:106AA000F9D0E6EC30F0EF28EFBE000EB3D0FAD10B
:106AB000FDEC30F0D8A42FEF32F0ACD0A3D8EF909B
:106AC00018B0EF8012009ED8000EEFB0010EA2D0D9
:106AD00000D237D24EEC31F01850EF6EABEF3EF0F3
:106AE0004EEC31F0EF5096D058EC31F01850EF6E7C
:106AF000ABEF3EF058EC31F0EF508CD053EC31F06E
:106B00005650C6EC16F018B003D0FF0AEF1601D0AD
:106B1000EF12ABEF3EF053EC31F05650C6EC16F0EE
:106B2000EF14D8A4010E76D0120012004EEC31F012
:106B3000EF9C18B0EF8CABEF3EF04EEC31F0000E56
:106B4000EFBC010E67D04EEC31F0F80EEF16185086
:106B5000EF12ABEC3EF0FAEF3FF04EEC31F0EF50BD
:106B6000070B58D012D85650C4EC16F0EF16FF0A97
:106B70001852D8A4EF12ABEF3EF007D85650C6EC2F
:106B800016F0EF14D8A4010E45D04EEC31F0E950C8
:106B9000F00B070FE96E120089D81850200DF3CFC3
:106BA000EFFF78D8EE501850200DF00EEF16F4508D
:106BB000EF1270D8ED5012007EEC30F0EE38E83075
:106BC000070B186EED38E830780B1812196A1200AE
:106BD000B0EC30F01850800FE8AE800EEF6E5AD057
:106BE000B0EC30F0EF50800FE8BE000E13D0B0ECE8
:106BF00030F0D8901834EF6E4DD0B0EC30F0D89023
:106C0000EF3008D0EA6AE99EEF501200FBDF18C0AF
:106C1000EFFF1200186E196A12002FEC3FF0E79E8A
:106C2000E7CF18F062EF2DF0C6EC16F0EF14000E6F
:106C3000D8A4010EEFD7FDEC30F0EECF06F0EECF8A
:106C400008F0EECF07F0EFCF09F0FD0EE92658AEC1
:106C50000BD0D89007320632D8B0078ED8900932C0
:106C60000832D8B0098E0AD0D89006360736D8B088
:106C70000680D89008360936D8B0088006C0EFFFE5
:106C800009D808C0ECFF06D807C0ECFF03D809C03C
:106C9000ECFF00D094EF3EF018B004D0C4EC16F036
:106CA000EF16F8D7C6EC16F0EF12F4D7FDCFF6FFCB
:106CB000FECFF7FFFFCFF8FF10CBE8FFE8B20DD013
:106CC000E8B00AD0540EE92645B04BD8060EE926A6
:106CD00045B247D806001200F5D7E8B000D0F2D789
:106CE000FDCFF6FFFECFF7FFFFCFF8FF10CBE8FF99
:106CF000E8B230D0E8B020D045A00DD0600E5624C8
:106D0000E96E48B02ED8100EE92648B22AD8100EE7
:106D1000E92648B426D845A20DD0900E5624E96E37
:106D200048B01FD8100EE92648B21BD8100EE9262D
:106D300048B417D80600120045A004D0600E5624AF
:106D4000E96E0FD845A204D0B00E5624E96E09D8DA
:106D500006001200E8B000D04DEC30F002D806007A
:106D60001200F29E0500F650FD6EF750FE6EF850D0
:106D7000FF6EF28E1200FDCFF6FFFECFF7FFFFCFC2
:106D8000F8FF10CBE8FFE8B21FD0E8B005D091ECD7
:106D900030F0E7DF0600120045A009D0600E56244F
:106DA000E96E4A50010B070DF350E926DADF45A2E0
:106DB00009D0B00E5624E96E4A50010B070DF3506E
:106DC000E926CFDF06001200E8B000D0E0D7FDCF03
:106DD000F6FFFECFF7FFFFCFF8FF10CBE8FFE8B2DA
:106DE00015D0E8B005D0B0EC30F0BBDF06001200E3
:106DF00045A004D0600E5624E96EB3DF45A204D04E
:106E0000B00E5624E96EADDF06001200E8B000D0E7
:106E1000EAD7F350FD26F450FE22000EFF221200A6
:106E2000CBEC30F05650C6EC16F0066E5650C4EC63
:106E300016F0076EEF16065018B0EF122BDF075052
:106E4000EC16065018B2EF1225D7CBEC30F05650A6
:106E5000C6EC16F0066E186A196AEE500614D8A42D
:106E60001880ED500614D8A418821200D3EC30F02C
:106E70005650C6EC16F0066E5650C4EC16F0076E6F
:106E8000EF16065018B0EF1205D7D3EC30F056507D
:106E9000C6EC16F0066E186A196AEF500614D8A4EC
:106EA00018801200FDEC30F0D8B412002C50800A8B
:106EB00003E018C0EFFFEED62C6AFDEC30F006E0E0
:106EC00018C0EFFFE7DE2C2A2CAEF7D7800E2C6E11
:106ED00012002C50F00B06E02C6A04D82C2A2CA8A7
:106EE000FCD71200FDEC30F0565007E0FF0F0BE02E
:106EF000FF0F11E0FF0F17E01CD0F00EEF16185037
:106F00000F0BEF12C7D6CF0EEF161838300BE8BABA
:106F1000E878EF12BFD63F0EEF161838E834E834A1
:106F2000C00BEF12B7D6800EE926EF9E18B0EF8E99
:106F3000B1D6800EE926800EEF1618507F0BEF12A7
:106F4000A9D6FDEC30F0565007E0FF0F08E0FF0F28
:106F50000BE0FF0F0EE013D0EF500F0B5BD6EF38B6
:106F6000030BE8B2E87056D6EF38E830E830030B90
:106F700051D6800EE926000EEFBE010E4BD6800ED4
:106F8000E926EF507F0B46D6880FD8B0880E780FD1
:106F9000C8EC16F077D079D07BD07DD07FD081D06F
:106FA00087D08FD09FD0A3D0A7D0A9D0ABD0CAD044
:106FB000ACD0CCD0CED0DAD0CED0EAD0EBD0EED0A0
:106FC000F0D0F2D006D108D108D109D110D111D119
:106FD00012D131D143D145D14ED150D152D154D11A
:106FE00056D159D15DD160D162D16BD16DD16FD104
:106FF00071D173D175D175D17ED198D1A0D1A3D1E2
:10700000A6D1C0D1C5D1C4D1C9D1D5D1E4D1E6D1A1
:10701000E8D1F0D1F2D1F4D1F6D1F7D1F8D102D242
:1070200005D207D210D21BD223D244D229D22BD2DE
:107030002DD242D252D255D258D26BD272D279D2FC
:107040007CD27FD28ED291D294D297D2A2D2A6D223
:10705000A9D2ADD2B9D2C4D23DD346D34BD351D3AA
:107060005DD360D363D3A2D3A4D3A9D3C0D3C0D3F9
:10707000C8D3D8D3D9D3E3D3E5D3E6D3E9D3E9D37F
:10708000ECD3FAD3030E53EF4FF0EF5070EF3CF018
:10709000EF2870EF3CF0EF507BEF3CF0EF5086EFC5
:1070A0003CF0EC5096EC16F0ED50EF5098EF16F0E7
:1070B00010EE3CF03350030BE126E7287F0B70EF16
:1070C0003CF0200E5BEC3CF02FEC3FF0136E36EC06
:1070D0003FF0146E410FEFDBACEC5EF0200ED8A455
:1070E0002A0EE9D32FEC3FF0010F72EF3CF044EC95
:1070F0003CF0010F72EF3CF0000E9DEF3CF0010EF2
:107100009DEF3CF0020E9DEF3CF044EC3CF0066E2F
:1071100009C607F02D0E06B0310E07A02A0ECBDBF4
:107120002D0E06B2320E07A22A0EC5DB2D0E06B4B6
:10713000330E07A42A0EBFDB2D0E06B6340E07A6AB
:107140002A0EB9D344EC3CF0BAEF3CF09DDB70EF73
:107150003CF09ADBC4D398DB200EADDB2D0EEFB0F4
:107160004C0EA9DB2D0EEFB2520EA5D34EEC31F032
:10717000000E45A0040FE926EF50EC3896EC16F00F
:10718000ED38F00BF36EEF380F0BF31098EF16F0AD
:1071900082DBA6D380DBE8380F0BA2D37CDB0F0B9E
:1071A0009FD379DB7F0B9BD376DBC20EF66E710E1D
:1071B000F76E000EF86E000EEFB0010EEFB2020E89
:1071C000CED34E6F722043544720476C73203F3F0D
:1071D0003F2061DB020EB1D312005DDB6ED35BDBBF
:1071E000EC5096EC16F0ED50EF5098EF16F053DBA4
:1071F00082D351DB8BD34FDB120EF66E720EF76E1D
:10720000000EF86EEF50070BEFB6080EEFB8000E49
:10721000A6D36F6666205472692053617720542B81
:10722000532050756C20502B5420502B532050531A
:1072300054204E6F69202FDB4C0EF66E720EF76EE7
:10724000000EF86EEF30E838030B89D32D2D2D207A
:1072500053796E2052696E20522653201CDB000E9B
:107260006CD319DB340EF66E7A0EF76E000EF86EE4
:10727000EF30070B74D30FDB040E5FD30CDB050E6E
:107280005CD309DB060E59D306DB070E56D303DBAE
:10729000EF501F0B24D3FFDAEF38E830070B1FD372
:1072A000FADAEF503F0B1BD3F6DA070E46D3F3DAC8
:1072B000100EF66E7A0EF76E000EF86EEF500F0B92
:1072C0004ED3E9DA040E39D3E6DA030E36D3E3DA25
:1072D000000E33D3E0DA010E30D3DDDA020E2DD307
:1072E00057D7D9DA100EF66E7A0EF76E000EF86EDA
:1072F000EF380F0B34D30C0EF66E730EF76E000ED4
:10730000F86E7EEC30F0EF50070B29D32D2D2D2099
:10731000312D2D202D322D2031322D202D2D3320B9
:10732000312D33202D323320313233207EEC30F0BA
:10733000EC5096EC16F0ED50EF5098EF16F07EEC16
:1073400030F0EF50CDD27EEC30F0EF50C9D2640E69
:10735000F66E730EF76E000EF86E7EEC30F0EF38BE
:10736000070BFDD22D2D2D204C2D2D202D422D2013
:107370004C422D202D2D48204C2D48202D424820B8
:107380004C4248207EEC30F0EFCF03F0030ED7D212
:107390007EEC30F0EFCF03F0070ED1D2540EF66E34
:1073A0007A0EF76E000EF86E7ADAE8380F0B010FDE
:1073B000EFA0000ED4D273DA7C0EF66E7A0EF76E62
:1073C000000EF86EFE0EEBA404D0EF500B0F01E39D
:1073D000C6D2EF5085D24FEC3CF082D24FEC3CF05D
:1073E00095D24A50562650C00AF0506A76D80AC044
:1073F00050F0120054DA010EA0D251DA030E9DD2E1
:107400004EDA020E9AD24FDA6BD24DDA7FD24BDAD5
:10741000070BF36EA80EF66E7A0EF76E000EF86E7E
:10742000F3509DD240DAEF38070BF3D73CDA070E62
:1074300084D2C80EF66E7A0EF76E000EF86E33DA4E
:10744000EF38070B8CD2E80EF66E7A0EF76E000E50
:10745000F86E2DDAE8AE02D07F0B42D280D2640EF5
:10746000F66E7B0EF76E000EF86E21DA0F0B77D2F8
:10747000A40EF66E7B0EF76E000EF86E18DA6FD261
:1074800016DA060E5AD213DA070E57D2CBEC30F0CA
:107490005650C6EC16F0066EEE5006144C0ED8B4DC
:1074A0002D0E09DA2F0E07DAED500614520ED8B45D
:1074B0002D0E01D2FCD92AD2480EF66E7C0EF76E44
:1074C000000EF86E5034E834FC0BF626000EF7225E
:1074D000000EF822030E9CEF16F0D3EC30F056505D
:1074E0002CD24EEC31F0EF50FBD1060EF66E750E3D
:1074F000F76E000EF86E4EEC31F0000EEFB0010E9C
:10750000EFB2020E2CD24D73742E536C762E417551
:10751000746F800EF66E7C0EF76E000EF86EB4D9A6
:107520001ED25650BEEC8CF0040EE226020EE35042
:10753000D7D1DEEC30F0EF50D3D1DEEC30F0EF50AD
:10754000CFD1EECFF3FFEDCFF4FFF4380F0B96EC75
:1075500016F0F438F00BF46EF3380F0BF41098EFCC
:1075600016F0140EE96E5650E8D1E6EC30F0EF500C
:10757000B7D1E6EC30F0EF50B2D1E6EC30F02D0EA2
:10758000EFBC4C0E98D92F0E96D92D0EEFBE520E91
:1075900092D1E6EC30F0EF503F0BA1D1E6EC30F0A9
:1075A000070ECBD1E6EC30F0EF507F0B26D2E6ECA5
:1075B00030F0EFBE03D0EF507F0B1FD22D0E7BD9E2
:1075C0002D0E79D92D0E77D15FD97F0E2C6406D080
:1075D000410E71D96C0E6FD96C0E6DD1EF500DD27A
:1075E000FDEC30F007E12E0E66D92E0E64D92E0E7A
:1075F00062D94BD0EFAE47D010CBE8FFE8B20ED047
:10760000E8B00BD01CEE6DF05650030B050DF35097
:10761000E126E750FC0BFC0A10D0F4D7E8B001D00B
:10762000F1D71BEE8CF05650070B300DF350E126CE
:10763000F450E222E750F80BF80A21E1EF50FC0B7E
:10764000FC0A0AE14B0E37D9790E35D9EF50030BFE
:10765000010F8EEC16F019D0EF507F0B06E0FF0FF4
:1076600006E0010F5BEC9EF010D02D0E01D02B0E2A
:10767000F56E21D9F5501FD9F5501DD906D0EF5020
:107680007F0BBBD902D0EF50BBD910CBE8FFE8B2DB
:1076900009D0E8B006D01CEE70F05650030B050D73
:1076A00009D0F9D7E8B001D0F6D71BEE64F05650F8
:1076B000070B300DF350E126F450E222E7BE120032
:1076C000E7507F0BF36EE950800FF3183C0ED8B4EF
:1076D000F2D81200480E1DB0440EEDD8650EEBD85E
:1076E000780E1DB0630EE7D0470EE5D86F0EE3D8D5
:1076F000210EE1D0C9D80F0E2C6401D069D7EF500C
:10770000EED0E6EC30F0EF50F80B02E1EF50E7D0AE
:10771000200ED1D8200ECFD82D0ECDD0E6EC30F0F3
:10772000070E0BD1E6EC30F0060E07D1FDEC30F081
:10773000565007E0FF0F16E0FF0F25E0FF0F2DE08A
:1077400030D0200EB8D8EF500F0B020DA00EF3244E
:10775000F66E7C0EF420F76EF86A000EF822020E28
:107760009CEF16F0760EF66E770EF76E000EF86E42
:10777000EF38030BF4D0202D2020205570204477C3
:107780006E20557032202D0EEFBC2A0E94D8200E9C
:1077900092D82D0EEFBE2A0E8ED0800EE926070E4F
:1077A000CCD0800EE926EF507F0B9AD074D8EF50E2
:1077B000EED0470E80D8650E7ED86E0E7CD030C0DD
:1077C00014F02FC013F0ACEC5EF00BE0145009E0A5
:1077D0003050410F70D8200E6ED82D0E6CD82D0E63
:1077E0006AD030C0F3FF2FC0F4FF66EF4FF01200F5
:1077F000450E88EC16F02FC013F030C014F0D4EF13
:107800004FF007EC5FF00AE02E5008E0450E53D829
:107810002D0E51D82D0E4FD82D0E4DD02EC0F3FF6A
:1078200059EF4FF034D85BD032D8F00B02E1EF5073
:1078300056D0200E40D82D0E3ED82D0E3CD027D845
:107840005BEF9EF024D857D053EC31F0565075D0F2
:1078500012004EEC31F0060E70D04EEC31F0EF50CD
:10786000070B04E090EC16F0200E25D06F0E23D805
:10787000660E21D8660E1FD04EEC31F0E950F00BA9
:10788000070FE96E565059D0EA6AEF50120058ECD3
:1078900031F0EF5012004DEC30F0EF50120091EC4F
:1078A00030F0EF501200B0EC30F0EF501200C3ECAB
:1078B00030F0EF50120094EF16F0066E200EFBDF52
:1078C000065098EF16F0066E2B0E06AC2D0EF3DF69
:1078D00006507F0B4008E8BEE86C98EF16F0010FE9
:1078E00092EF16F0036AF4EC16F0045096EC16F0E2
:1078F000035098EF16F0066E200E06AC2D0EDBDF5F
:1079000006504008E8BEE86C90EF16F0E8AE03D0F1
:107910007F0B92EF16F08008066E9C0F05E22D0E8D
:10792000CADF065090EF16F0060EC5DF06509C0F1A
:10793000036AF4EC16F098EF16F0EFCF03F0C6EC04
:1079400016F0031406E1200EB6DF6F0EB4DF200E32
:10795000B2D7200EB0DF2A0EAEDF200EACD7E8364D
:10796000E834FC0BF626000EF722000EF822040E77
:107970009CEF16F0066E2D0E06B0310E9CDF2D0E1C
:1079800006B2320E98DF2D0E06B4330E94D7020DD8
:10799000600EF324F66E3F0EF420F76EF86A010EC7
:1079A000F8220900F5CFF3FF0900F5CFF7FFF3CF79
:1079B000F6FF040E9CEF16F0FDEC30F0EECF06F073
:1079C000EECF08F0EECF07F0EECF09F0100EF36E19
:1079D00006B006D008B002D0A50E07D0410E05D0E3
:1079E00008B002D02A0E01D0530E65DF07320632EE
:1079F00009320832F32EECD712001DA05ED770D7E3
:107A00001DA061D7066E2B0E06AC2D0E54DF78D765
:107A1000204C5220204C2D20202D5220204F312050
:107A2000204F3220204F3320204F3420204F35204C
:107A3000204F36205570202044776E205526442054
:107A4000442655205544322044553220526E64203D
:107A5000722E37206F66662053696E20547269203B
:107A60005361772050756C2052616E2050536E2008
:107A7000505472205053772050506C2036342F31A0
:107A800033322F3131362F31382F3120342F3120FE
:107A9000322F3120312F3120312F3220312F34201D
:107AA000312F3820312F31362D2D2D2041743120AA
:107AB000417432204465312044653220537573206F
:107AC00052653120526532202D2D2D20412D2D2043
:107AD0002D442D2041442D202D2D5220412D52206A
:107AE0002D445220414452202D2D2D204547312038
:107AF000454732204C4631204C4632204C463320FC
:107B00004C4634204C4635204C4636204D503120D2
:107B10004D5032204D5033204D5034204D503520A3
:107B20004D5036204D5037204D5038204D64572051
:107B30004B6579204B2331204B2332204B233320BC
:107B40004B2334204B2335204B2356204B235020EE
:107B50004B2341205754312057543220575433205F
:107B6000575434202D2D2D20537231205372322042
:107B7000312B3220312D3220312A3220584F5220E1
:107B80004F522020414E44204D494E204D41582017
:107B9000313C3220313E3220313D322053264820C4
:107BA000722E32202D2D2D20507431205074322011
:107BB0005074332050743420507435205074362063
:107BC00050573120505732205057332050573420CF
:107BD0005057352050573620466C3120466C3220A5
:107BE000566C3120566C32204C4431204C443220AB
:107BF0004C4433204C4434204C4435204C443620F3
:107C00004C5231204C5232204C5233204C523420B2
:107C10004C5235204C523620457831204578322060
:107C2000457833204578342045783520457836200E
:107C30004578372045783820575431205754322022
:107C400057543320575434204E4F6E204E4F6620E9
:107C500045315320453253204C3150204C32502076
:107C60004C3350204C3450204C3550204C36502052
:107C7000436C6B20436C3620433234204D537420C8
:107C80004B2331204B2332204B2333204B233420F2
:107C90004B2335204B2356204B2350204B23412090
:107CA00043204323442044234520462046234720A5
:107CB0004723412041234220432B030E44B4020EAC
:107CC00044B2010E44B0000E336EFF0B12005F5041
:107CD00008E012005DEC3EF05F18D8B4120033C02B
:107CE0005FF05FC033F0335010E10BEE00F017EEA1
:107CF00000F0F36AF46AE6CFEEFFF32AD8B4F42A70
:107D0000F4A2F9D7FCEC51F004D0DBEC42F01CEC0F
:107D100043F01C841FBE1C8212005F50336E02E1D0
:107D2000FCEF51F01CEF43F033500CE1E9CFE1FFE1
:107D3000EA50FC0FE26EEFCFE7FF020EE226EFCF34
:107D4000E7FF1200E9CF03F0EA50F50F046EEF50A1
:107D500044EC42F01200335002E186EF51F0800E05
:107D6000E924036EEF505DEF42F0335006E1EFCFB0
:107D700003F0565037EC8CF005D056C003F0EF50AE
:107D80008DEC42F02BA2120010EE3CF03350E126B5
:107D90005650070BC8EC16F007D014D015D016D0EB
:107DA00017D018D018D025D0010EF36EE7500F0B66
:107DB000B00924EC16F0F35024EC16F0EF307F0BF2
:107DC00024EF16F0100EF1D7110EEFD7120EEDD7EB
:107DD000130EEBD71200E7500F0BE00924EC16F05E
:107DE000000EEFB0400E24EC16F0EF307F0B24EFC6
:107DF00016F01200036E335003E15150B0EF8CF0D7
:107E0000A5EF42F0335002E10FEF54F050EF43F092
:107E100091D81C841FBE1C82120033B20CD033B028
:107E200005D034C013F038C014F011D035C013F0B1
:107E300039C014F00CD033B005D036C013F03AC0BE
:107E400014F005D037C013F03BC014F000D0139EDF
:107E5000120034C013F038C014F0139E120010EE5C
:107E600034F03350E126E7507F0B120010EE38F06B
:107E70003350E126E750070B12000101F36A00EED0
:107E80003CF0F350E926EF5003190F0B0EE1F80E0A
:107E9000E9260451EF187F0B08E004C1EFFF0C0E38
:107EA000E926EFBE02D0810EEF6EF32AF3A4E7D7E6
:107EB00012000101F36A00EE3CF0F350E926EF50A6
:107EC00003190F0B12E1FC0EE9260551EF18070B01
:107ED0000CE00551070BEF6EFC0EE926EF9E0C0E31
:107EE000E926EFBE02D0810EEF6EF32AF3A4E3D7AA
:107EF0001200335012E10BEE00F017EE00F029EE05
:107F000000F0020EF36EEFCFE6FFEECFDEFFE9509A
:107F1000FAE1F32EF8D7F7EF52F0FBEF43F0336AB4
:107F20003350C6EC16F0441401E0E3DF332A33A4E7
:107F3000F7D7C3D610EE40F03350E126E750D8A46F
:107F40001DD033500CE1010EE76E34BE16D034C0A4
:107F500013F038C014F0348E3BEC54F00ED0060E03
:107F6000E76E10EE34F03350E3BE07D0E38E52ECF0
:107F700043F00DEC3FF06FEC43F0120010EE40F0D8
:107F80003350E126800EE76E1200336A10EE40F0A7
:107F90003350E126E7AE05D0E7507F0B02E1E79EC4
:107FA00037DF332A33A4F2D71200336EC6EC16F053
:107FB000E838F00B076EF29E1D5007181D6EF28E0A
:107FC0003350C6EC16F0E8381D1401E001D006D09D
:107FD000335002E18DEF53F054EF43F0335002E1A0
:107FE000DFEF53F069EF43F0335002E194EF58F0C4
:107FF0006BEF43F0335002E1DEEF58F06DEF43F0EA
:1080000000145349443120452E20506C7920496E8C
:108010006920446D70200C0E00A684EC16F0000E52
:10802000F66E800EF76E000EF86E9EEC16F0030EE4
:1080300088EC16F05DEC3EF0010F8EEF16F05074F8
:108040002E20456E7320400E88EC16F044D84C0E5E
:1080500045A02D0E41D8520E45A22D0E3DD83BD83D
:10806000200E94EC16F010CBE8FF030B73EC4FF0EE
:10807000200E94EC16F02FD85DEC3EF0C6EC16F016
:10808000E8381D146F0ED8A42A0E26D824D823D879
:10809000FDD8066EE8BC010E040D3E0EF324F66E0C
:1080A000800EF420F76EF86A000EF822040E9CECA5
:1080B00016F006BC0BD05DEC3EF036EC3FF0146ED3
:1080C0002FEC3FF0136E66EC4FF002D057EC4FF000
:1080D000140EDEEF2DF0200E94EF16F0066EFBDF8F
:1080E0006F0EFADF660E06B06E0EF6DF660E06B095
:1080F000200EF2DFF0D79EEC16F0400EFAEF16F0ED
:10810000070BC8EC16F007D00DD06FD03BD09DD038
:108110001200120012004528030BD8B4010F456E5F
:108120001C8412000BEE10F0EF50010F030BF36EE6
:10813000EF50FC0BF310EF6E4CEC54F08FEC3FF073
:10814000466A476AE5EC2DF04A6A4B6A4D6A506A06
:10815000516A526ADBEF29F0401420506174636861
:1081600020496E697469616C6973656420204014EC
:10817000456E73656D626C6520496E697469616CEA
:108180006973656483D8E8BC0ED04CEC54F08FEC76
:108190003FF0580EF66E810EF76E000EF86EABDFF4
:1081A000140EDEEF2DF05CEC52F06E0EF66E810ECA
:1081B000F76E000EF86E9FDF140EDEEF2DF0401408
:1081C0002D2D20416C6C204E6F746573204F6666B8
:1081D000202D2D2040142D2D20506C6179696E6763
:1081E000205061746368202D2D2001EC23F05DEC9C
:1081F0003EF0C6EC16F0E8381D1407E0D40EF66E1B
:10820000810EF76E000EF86E06D0BE0EF66E810E71
:10821000F76E000EF86E6FDF140EDEEF2DF04014D7
:108220002D2D2050617463682044756D7020736536
:108230006E74202D40142D2D20456E732E20447514
:108240006D702073656E74202D2020D80809E8CF4A
:1082500015F1146A136A33C012F0E8BC10D01E0E78
:10826000F66E820EF76E000EF86E45DF140EDEEC31
:108270002DF0A8EC8AF004EC16F0126E1200340E09
:10828000F66E820EF76E000EF86EEFD7000E1FBC72
:10829000700E1200C2DDD8EF5EF0BFDDEAEF5EF0D7
:1082A0003104D8A41200316A3DEF51F00014534953
:1082B0004478206E6F7420636F6D70617469626CB6
:1082C0006520001453494478206E6F7420617661F4
:1082D000696C61626C6520204014284E6F204D420D
:1082E0004E657420526573706F6E7365292040145B
:1082F0002843414E20427573204572726F72732974
:108300002020202040142843414E2064697361627C
:108310006C6564212920202020205DEC3EF0C6EC15
:1083200016F0060109153BE11C9000BB14D0335038
:10833000C6EC16F006010A150EE0AC0EF66E820EC3
:10834000F76E000EF86E9EEC16F0400E88EC16F0FC
:10835000335041D81DD0C20EF66E820EF76E000E5D
:10836000F86E9EEC16F0060100BB01D007D0040E9B
:10837000F66E830EF76E000EF86E08D000A906D0D8
:10838000EE0EF66E820EF76E000EF86E9EEC16F094
:10839000030E88EC16F033288EEC16F01200120053
:1083A0005DEC3EF0C6EC16F00601091503E1335012
:1083B00049EC20F01200336E030B10EE34F0E39E14
:1083C000BEEC3FF03350B9EC51F022EC44F08DECB0
:1083D0003EF01C82120006EE20F0E834E834E83467
:1083E000380BE926500E94EC16F0EE50036AF4ECCC
:1083F00016F0045096EC16F0035098EC16F0200E90
:1084000094EC16F0040EF36EEE50D8B43F0E94ECDC
:1084100016F0F32EF9D7200E94EC16F0560E94ECCD
:1084200016F0EE50036AF4EC16F0045096EC16F0D9
:10843000035098EC16F02E0E94EC16F0EE50EECFA2
:1084400003F0F4EC16F0055096EC16F0045098EC9E
:1084500016F0035098EC16F0120033C005F6060132
:10846000060E076F086B000EA7EC1FF00CE1030E61
:10847000E66E03C0E6FF04C0E6FF05C0E6FFCCECF5
:108480001FF0D8A402D21200056E33C005F6060113
:10849000120E076F086B000EA7EC1FF00DE1040E23
:1084A000E66E03C0E6FF04C0E6FF05C0E6FFE66A2D
:1084B000CCEC1FF0D8A4E9D11200056E33C005F64C
:1084C0000601110E076F086B000EA7EC1FF00CE100
:1084D000040EE66E03C0E6FFE66A05C0E6FFE66A44
:1084E000CCEC1FF0D8A4D1D11200056E33C005F634
:1084F00006011C0E076F086B000EA7EC1FF00CE1C5
:10850000040EE66E03C0E6FFE66A05C0E6FFE66A13
:10851000CCEC1FF0D8A4B9D11200056E33C005F61B
:108520000601130E076F086B000EA7EC1FF00CE19D
:10853000040EE66E03C0E6FFE66A05C0E6FFE66AE3
:10854000CCEC1FF0D8A4A1D1120033C005F606016F
:10855000140E076F086B000EA7EC1FF008E1010E68
:10856000E66E03C0E6FFCCEC1FF0D8A48ED112005B
:108570000601076F086B33C005F6000EA7EC1FF06D
:1085800006E1000EE66ECCEC1FF0D8A47ED11200FE
:10859000000EEED7010EECD7100EEAD7170EE8D773
:1085A000335004E1596A5A6A000B120059505A10AC
:1085B00004E1000B1200596A5A6AC8EC42F036E135
:1085C00059C007F65AC008F6010EA7EC1FF032E1B9
:1085D000000EE66ECCEC1FF0D8A457D11EEE75F05D
:1085E000E650080AD8A451D159C0E9FF5A50010BEE
:1085F0000B0FEA6EE6CFEEFFE6CFEEFFE6CFEEFF23
:10860000E6CFEEFFE6CFEEFFE6CFEEFFE6CFEEFFE2
:10861000E6CFEEFF080E5926D8B45A2A59501F0B40
:10862000CFE1595005E15A50FE0B02E0596A5A6AEF
:10863000CAEC42F0FF091200C8EC42F02EE1A96A30
:10864000A9CF07F6FF0EE8CF08F6010EA7EC1FF042
:1086500026E1000EE66ECCEC1FF0D8A416D11EEE7B
:1086600075F0E650080AD8A410D100EE80F0A950A9
:10867000E926E6CFEEFFE6CFEEFFE6CFEEFFE6CF50
:10868000EEFFE6CFEEFFE6CFEEFFE6CFEEFFE6CF62
:10869000EEFF080EA926A9ACD3D7CAEC42F012000F
:1086A000150E66D7160E64D733C005F60601180EF0
:1086B000076F086B000EA7EC1FF00AE1020EE66ED2
:1086C00046C0E6FF45C0E6FFCCEC1FF0D8A4DDD0E5
:1086D0001200190E4DD71A0E4BD71B0E49D7C8ECF6
:1086E00042F05AE1ACEC5EF05AE1135058E0A96A4E
:1086F000AA6AA0EC5EF002EC17F001340E0BA009A0
:1087000006EC17F0045006EC17F0035006EC17F0D7
:1087100002EC17F001340E0BA10906EC17F00BEE7A
:1087200000F0A9CF07F6AACF08F6020EA7EC1FF0BB
:1087300035E1080EE66E08EC17F0E66EF36E5F505A
:108740003318D8B4F3CFEEFFA92AD8B4AA2AA95077
:1087500006E1AA50FE0B03E00CEC17F002D00AEC85
:1087600017F0A950070BE7E1AA5003E1A950080A46
:1087700004E0D3EC1FF0D8A488D0C2EC1FF0A950BD
:10878000D0E1AA50FE0BCDE0D3EC1FF0D8A47DD0F1
:1087900004EC17F0CCEC42F0CAEC42F01200A96AEB
:1087A000AA6A0BEE00F0A9CF07F6AACF08F6020ED0
:1087B000A7EC1FF0F3E1080EE66EB0EC16F0E66EE3
:1087C000F36EA950D8B4AA2A5F503318D8B4F3CFA7
:1087D000EEFFA950070BF1E1CCEC1FF0D8A455D067
:1087E000A950E1E1AA50FE0BDEE0CCEC42F0D4D778
:1087F00007EE00F002D00BEE00F0C8EC42F01FE1F3
:10880000A96AAA6AA9CF07F6AACF08F6020EA7ECB2
:108810001FF017E1080EE66EEECFE6FFA92AD8B4E6
:10882000AA2AA950070BF8E1CCEC1FF0D8A42DD050
:10883000A950E8E1AA50FE0BE5E0CCEC42F0CAEC0E
:1088400042F01200C8EC42F01DE100EE80F0A96A8F
:10885000A9CF07F6FF0EE8CF08F6020EA7EC1FF02F
:1088600013E1080EE66EEECFE6FFA92AA950070B2A
:10887000FAE1CCEC1FF0D8A408D0A9503F0BE8E1F6
:10888000CEEC42F0CAEC42F012001C82FF0912004A
:1088900001030301020404020305000304060004AB
:1088A000050000000B0906090E0C090C0A89BE8997
:1088B0005A8AD28AB6886E8BF055B2532D2D2D115F
:1088C0007F098A8D5C56C2532D2D2D000000BE8D70
:1088D0005C56C2532D2D2D000000DE8D5C56C25318
:1088E0002D2D2D000000088E5C56C253494E534674
:1088F0000510468E5C56C2532D2D2D000000D48EDF
:108900005C56C2532D2D2D000000AC8BF055B25398
:108910002D2D2D137F08EA8E5C56B6534F534347D7
:10892000020D4A915C56B653414368450312E491E7
:108930005C56B6534C464F4A05103E935C56B653B0
:10894000454E564B0110DE945C56B6534D4F444D88
:1089500007108A955C56B653545247500D4F869671
:108960005C56B65341436845031254975C56B65360
:108970004F534347020D4E9A5C56B65357542052FC
:108980000310969B5C56B653506F732C8060A4986E
:108990005C56B6534B4E42510753AC995C56B65396
:1089A0002D2D2D000000F29C5C56B6532D2D2D0070
:1089B0000000769E5C56B6532D2D2D0000003A8C9B
:1089C000F055B2532D2D2D137F083A9C5C56B653AB
:1089D000506F732C0F64069B5C56B6534143684539
:1089E00003122E905C56B653414368450312929190
:1089F0005C56B653414368450312BA925C56B6536F
:108A000041436845031264945C56B653414368453C
:108A1000031234985C56B6534143684503122097BD
:108A20005C56B65341436845031228995C56B653C9
:108A30004B4E42510753AC995C56B6532D2D2D0029
:108A40000000BE9D5C56B6532D2D2D000000769E75
:108A50005C56B6532D2D2D000000B48CF055B2534A
:108A60002D2D2D137F08AA9C5C56B65354726B5063
:108A70000710589B5C56B6532D2D2D000000C69054
:108A80005C56B653496E73460F104A915C56B65306
:108A900041436845031220975C56B65341436845ED
:108AA0000312A4985C56B6534B4E42510753AC99EF
:108AB0005C56B6532D2D2D000000389E5C56B653E3
:108AC0002D2D2D000000769E5C56B6532D2D2D00C9
:108AD0000000108DF055B2532D2D2D137F08968F69
:108AE0005C56B653496E734605104A915C56B653B0
:108AF00041436845031240925C56B653496E734633
:108B00000510FE935C56B653496E73460510BA962F
:108B10005C56B653496E73460510C4975C56B653FF
:108B2000496E73460510B49A5C56B653496E734647
:108B30000510DE9B5C56B653506F732C8060A49872
:108B40005C56B6534B4E42510753AC995C56B653E4
:108B50002D2D2D000000629D5C56B6532D2D2D004D
:108B60000000769E5C56B6532D2D2D0000000600A9
:108B70004153494400000001000042434C4B0000B7
:108B8000000100004346494C000000010000444938
:108B90004E530000000100004545585400000001FC
:108BA0000000465341560000000300000E00014F34
:108BB00053430000000100000246494C0000000140
:108BC0000000034C464F00000001000004454E56D3
:108BD000000000010000054D4F44000000010000AE
:108BE00006545247000000010000074346470000BA
:108BF0000001000008415250000000010000095728
:108C000054430000000100000A57544500000001D1
:108C100000000B4B4E420000000100000C45585470
:108C20000000000100000D524E4400000001000051
:108C30000E5341560000000200000C000153455144
:108C40000000000100000253514300000001000039
:108C5000034F53430000000100000446494C00004C
:108C600000010000054C464F0000000100000645D1
:108C70004E56000000010000074152500000000164
:108C8000000008434647000000010000094B4E4227
:108C90000000000100000A455854000000010000D7
:108CA0000B524E440000000100000C5341560000DE
:108CB00000020000090001534551000000010000BE
:108CC000025351430000000100000344524D0000D4
:108CD000000100000446494C00000001000005436B
:108CE0004647000000010000064B4E420000000114
:108CF00000000745585400000001000008524E448F
:108D0000000000010000095341560000000200006D
:108D10000C00014F53430000000100000246494C83
:108D2000000000010000034C464F0000000100005D
:108D300004454E5600000001000005434647000070
:108D400000010000064152500000000100000757DA
:108D50005443000000010000085754450000000182
:108D60000000094B4E420000000100000A45585423
:108D70000000000100000B524E4400000001000002
:108D80000C534156000000020000050044534944C2
:108D900003000E04040000426E6B07000706420049
:108DA000015061747F0008074300024D6F6E01009F
:108DB00075085C0006535056040076045D000300FD
:108DC0004453494403000E0404000542504DCD00B5
:108DD00051044700024D6F6402005208480004002D
:108DE0004453494403000E04040045414368020013
:108DF00012080600084D696EFF0F110407000A4DA6
:108E00006178FF0F11040700060044534944030032
:108E10000E04040046496E7305001004030000436D
:108E2000686E1000700441000153704C7F007104A3
:108E30005900025370557F00710459000354726E3B
:108E40007F00720459000E004453494403000E048D
:108E5000040000463241010073085A0001563241B5
:108E6000010073085A0002503241010073085A0091
:108E7000034B3241010073085A00044F3241010094
:108E800073085A0000497631010077085E000149F5
:108E90007632010077085E000249763301007708D8
:108EA0005E0003497634010077085E000449763598
:108EB000010077085E0005497636010077085E00FC
:108EC00006497637010077085E00074976380100C9
:108ED00077085E0002002E4523207F006E04030009
:108EE00000646F210000000C00001100484F534344
:108EF00006000D0405000157617608001E041000ED
:108F000001532F5203001F0811000744656CFF0036
:108F100013040A000241746B0F0014040B00024496
:108F200065630F0015040C00035375730F001404E0
:108F30000B000352656C0F0015040C000A50526EB2
:108F40007F0013040A000854726E7F001C040A009C
:108F50000946696EFF001D040A000B506F72FF0086
:108F600013040A0053506873FF0001040100045009
:108F70005720FF0F1B040F0000504D64020017081C
:108F80000D0000475341010018080E00514465745C
:108F9000FF00010401000F0046496E730500100434
:108FA00003000157617608001E04100001532F5280
:108FB00003001F0811000744656CFF0013040A003A
:108FC0000241746B0F0014040B00024465630F0030
:108FD00015040C00035375730F0014040B000352A7
:108FE000656C0F0015040C000A50526E7F001304CC
:108FF0000A000854726E7F001C040A000946696E5C
:10900000FF001D040A000B506F72FF0013040A00DA
:109010001050687301002B081C0004505720FF0FEC
:109020001B040F0000504D64020017080D000F00D4
:1090300045414368020012080600015761760800A6
:109040001E04100001532F5203001F081100074493
:10905000656CFF0013040A000241746B0F001404D6
:109060000B00024465630F0015040C000353757375
:109070000F0014040B000352656C0F0015040C0064
:109080000A50526E7F0013040A000854726E7F006B
:109090001C040A000946696EFF001D040A000B50FB
:1090A0006F72FF0013040A001050687301002B0850
:1090B0001C0004505720FF0F1B040F0000504D648C
:1090C000020017080D000D0046496E730F001004D2
:1090D0000300014D646C130069040A000241746BC3
:1090E0000F0014040B00024465630F0015040C000C
:1090F000035375730F0014040B000352656C0F00CB
:1091000015040C000454756EFF001D040A00054789
:109110004C2EFF001D040A0006537064FF001D045E
:109120000A0007504152FF001D040A000056417317
:1091300008003104260008566541FF003005220072
:1091400000526E640000630A000007000043686E6E
:1091500007003204270001437574FF0F3304280011
:1091600003526573FF0034042900004D6F6407004B
:1091700036042B0000457874010037082C000033BA
:109180004F66010038082D00024649500100390899
:109190002E0008000043686E0700320427000143D8
:1091A0007574FF0F3304280003526573FF00340405
:1091B0002900004D6F64070036042B00044B5472E5
:1091C000FF0035042A0000457874010037082C00A0
:1091D00000334F66010038082D0002464950010057
:1091E00039082E0009004A4C464F050010040300C0
:1091F0000057617609003A04300002527465FF009E
:109200003B042F000043536E010041083400014429
:109210006570FF003D042F000A536E6301003E0895
:1092200031000344656CFF003C042F000450687358
:10923000FF003C042F00004F6E6501004008330022
:109240000C0046496E730500100403004A4C464F5B
:109250000100100403001457617609003A0430003D
:1092600016527465FF003B042F001443536E010037
:109270004108340015442E50FF003D042F001944CE
:109280005057FF003D042F001A442E46FF003D04B6
:109290002F0014536E6301003F0832001744656CC1
:1092A000FF003C042F0018506873FF003C042F009F
:1092B000144F6E650100400833000D0045414368BE
:1092C0000200120806004A4C464F01001004030039
:1092D0001457617609003A04300016527465FF0095
:1092E0003B042F001443536E010041083400154421
:1092F0002E50FF003D042F0019445057FF003D043D
:109300002F001A442E46FF003D042F0014536E63B5
:1093100001003F0832001744656CFF003C042F0039
:1093200018506873FF003C042F00144F6E65010055
:1093300040083300064163637F0013040A001300F2
:109340004B454E5601001004030001446570FF00B8
:10935000430435000244656CFF00420435000341BC
:109360007431FF004204350004414C76FF00420492
:10937000350005417432FF00420435000644653172
:10938000FF004204350007444C76FF0042043500DC
:1093900008446532FF004204350009537573FF002D
:1093A000420435000A526531FF00420435000B5279
:1093B0004C76FF00420435000C526532FF00420437
:1093C00035000D437541FF00430435000E437544DD
:1093D000FF00430435000F437552FF00430435007E
:1093E000004C7042070044043600004C70450700F2
:1093F000450437000043536E0100460838000A0058
:1094000046496E7305001004030023442E50FF00EC
:109410004304350024445057FF00430435002544DD
:109420002E46FF004304350026417474FF004204B9
:10943000350027446563FF004204350028537573E7
:10944000FF00420435002952656CFF0042043500DC
:109450002A437572FF00430435002243417307001D
:10946000470439000C004541436802001208060019
:1094700023442E50FF004304350024445057FF007E
:109480004304350025442E46FF00430435002641A1
:109490007474FF004204350027446563FF004204F2
:1094A000350028537573FF00420435002952656C5E
:1094B000FF00420435002A437572FF004304350063
:1094C0002243417307004704390030446341FF00E1
:1094D00042043500064163637F0013040A00110053
:1094E0004D4D4F44070010040300005372319E009D
:1094F00048043B00015372329E0048043B00024F77
:10950000702E0E0049043C000654723128004A04B3
:109510003A000754723228004A043A000344657046
:10952000FF004B043A000249763101004C083D002F
:109530000249763201004D083E00005074310300AC
:109540004E083F000150743203004E083F000250A5
:10955000743303004E083F000350573103004E0898
:109560003F000450573203004E083F000550573368
:1095700003004E083F000646696C03004E083F009A
:1095800007566F6C03004E083F00190050545247B5
:109590000D004F040300004F314C01005008400003
:1095A000014F324C010050084000024F334C010083
:1095B00050084000034F3152010050084000044F52
:1095C0003252010050084000054F3352010050084C
:1095D0004000064531410100500840000745324136
:1095E0000100500840000845315201005008400079
:1095F000094532520100500840000A4C3120010058
:10960000500840000B4C32200100500840000C4C28
:1096100033200100500840000D4C34200100500858
:1096200040000E4C35200100500840000F4C362001
:10963000010050084000105731520100500840000E
:1096400011573252010050084000125733520100A6
:10965000500840001357345201005008400014577E
:109660003153010050084000155732530100500893
:109670004000165733530100500840001757345329
:10968000010050084000050052566F6C7F00010435
:109690000100504C656701000A0844005057544FC0
:1096A00001000B0845005053754B01000C084600A3
:1096B0001241425701000A0844000A0046496E73ED
:1096C00005001004030052566F6C7F000104010076
:1096D0001156417308002A04210010506F6C0100DC
:1096E0002C081D00104C656701002D081E00105746
:1096F000544F01002E081F001053754B01002F0816
:10970000200012566541FF003005220013506241CF
:10971000FF00300522001241425701000A084400B0
:1097200005004541436802001208060052566F6C5E
:109730007F0001040100104C656701002D081E0028
:109740001053754B01002F082000124142570100B1
:109750000A0844000B00484F534306000D0405005F
:109760000C4F6E200100200812000C4469720600A4
:10977000210413000C536F720100220814000C48DE
:109780006C640100230815000D5370643F00280429
:109790001A000E474C6E1F00260418000E526E670A
:1097A0000700270419000C536E63010024081600FB
:1097B0000C4341430100250817000D4F6E65010061
:1097C00029081B000B0046496E73050010040300B6
:1097D0000C4F6E200100200812000C446972060034
:1097E000210413000C536F720100220814000C486E
:1097F0006C640100230815000D5370643F002804B9
:109800001A000E474C6E1F00260418000E526E6799
:109810000700270419000C536E630100240816008A
:109820000C4341430100250817000D4F6E650100F0
:1098300029081B000B00454143680200120806007E
:109840000C4F6E200100200812000C4469720600C3
:10985000210413000C536F720100220814000C48FD
:109860006C640100230815000D5370643F00280448
:109870001A000E474C6E1F00260418000E526E6729
:109880000700270419000C536E630100240816001A
:109890000C4341430100250817000D4F6E65010080
:1098A00029081B000D00004B2331FF005404490020
:1098B000014B2332FF0054044900024B2333FF00C5
:1098C00054044900034B2334FF0054044900044B63
:1098D0002335FF0054044900054B2356FF00540470
:1098E0004900064B2350FF0054044900074B234115
:1098F000FF0054044900514B6E62070053040300FB
:1099000000506131FF0055054B0001506132FF00EE
:1099100055054B00034D696EFF0056044A00044D87
:109920006178FF0056044A000D0000437574FF0083
:109930005404490001526573FF0054044900024574
:109940004D64FF005404490003446563FF00540460
:10995000490004416363FF0054044900054B23564A
:10996000FF0054044900064B2350FF0054044900F3
:10997000074B2341FF0054044900514B6E6207001E
:109980005304030000506131FF0055054B000150A6
:109990006132FF0055054B00034D696EFF00560410
:1099A0004A00044D6178FF0056044A00100040410F
:1099B0002331FF0F57044C0042412332FF0F57045D
:1099C0004C0044412333FF0F57044C0046412334DD
:1099D000FF0F57044C0048412335FF0F57044C003C
:1099E0004A412336FF0F57044C004C412337FF0FE9
:1099F00057044C004E412338FF0F57044C000053CE
:109A00002331010058084D0001532332010058084A
:109A10004D0002532333010058084D0003532334F3
:109A2000010058084D0004532335010058084D002B
:109A300005532336010058084D0006532337010013
:109A400058084D0007532338010058084D000A00FC
:109A50005220575403001004030001506172FF00AC
:109A600059054E000053494403005B084F00005362
:109A700070643F005C045000024D4F4401005D08DB
:109A80005200024265677F005E04530003456E6426
:109A90007F005E045300044C6F7080005F0454002C
:109AA0001D56616C0100620856000A5754450000BB
:109AB00063010000080046496E73050010040300AE
:109AC0002C506172FF0059054E002B5370643F000B
:109AD0005C0450002D4265677F005E0453002E45F4
:109AE0006E647F005E0453002F4C6F7080005F0433
:109AF00054001D56616C0100620856000857544519
:109B0000000063010000080045414368020012089C
:109B10000600104F6E2001002E0823002C536571A3
:109B2000080065040A002B5370643F005C042400A5
:109B30002D4C656E0F0016040A002B5331360100C0
:109B4000660825002E506172FF0059054E00015332
:109B500045510000630100000600504F6E200100D7
:109B60006708510051536571080065044E00505359
:109B700070643F005C045000534C656E0F005A0542
:109B80004E005053313601006608520001534551D2
:109B900000006301000007002C506F738000600418
:109BA000030000242121FF0061045500012421212C
:109BB000FF006104550002242121FF0061045500CB
:109BC00003242121FF00610455001D56616C010032
:109BD0006208560009575443000063010000090061
:109BE0002C506F7380006004030000242121FF00CB
:109BF0006104550001242121FF0061045500022465
:109C00002121FF006104550003242121FF0061048C
:109C1000550004242121FF00610455000524212161
:109C2000FF00610455001D56616C0100620856007A
:109C3000075754430000630100000B002D5365716A
:109C40000700100403002C506F731000640403001D
:109C5000004E74650C0068045700014F63740300E4
:109C60006808570002532F47030068085700034154
:109C70006363010068085700045061727F00680444
:109C80005700004370790000000E0000005073740C
:109C90000000000F000000436C7200000010000084
:109CA0000253514300006301000007002D5365710A
:109CB0000700100403005054726B070010040300E7
:109CC000324544540F00630D0900004370790000D1
:109CD000000E0000005073740000000F00000043ED
:109CE0006C72000000100000025351430000630139
:109CF00000000B0000416C6C00006A090000014F7D
:109D0000736300006A0900000246696C00006A097A
:109D10000000034C464F00006A09000004454E56FF
:109D200000006A090000054D6F6400006A09000028
:109D30000654726700006A09000007575443000088
:109D40006A0900000857544500006A090000094BE1
:109D50006E6200006A0900000A45787400006A0912
:109D60000000090000416C6C00006A090000014F0E
:109D7000736300006A0900000246696C00006A090A
:109D80000000034C464F00006A09000004454E568F
:109D900000006A0900000757544300006A090000E8
:109DA0000857544500006A090000094B6E62000024
:109DB0006A0900000A45787400006A0900000C0076
:109DC00000416C6C00006A0900000B4E74650000D5
:109DD0006A0900000C47746500006A0900000D5311
:109DE0006C6400006A0900000E41636300006A09A8
:109DF00000000F50617200006A090000014F736398
:109E000000006A0900000246696C00006A0900004F
:109E1000034C464F00006A09000004454E560000FE
:109E20006A090000094B6E6200006A0900000A45D9
:109E3000787400006A090000060000416C6C0000A4
:109E40006A0900001053657100006A0900000144AE
:109E5000726D00006A0900000246696C00006A0920
:109E60000000094B6E6200006A0900000A45787420
:109E700000006A09000003003042232007006B0441
:109E800003002F5023207F006C04030000646F2127
:109E90007F006D0B080094EF16F0F46EF350FBDFBB
:109EA000F42EFCD71200F46E200EF36EF7D711C01B
:109EB000F3FF450E4BEC4FF0F328036AF4EC16F079
:109EC000045096EC16F0035098EF16F01450410F22
:109ED000E2DF1328036AF4EC16F0045096EC16F057
:109EE000035098EF16F0030B020D020EF324F66EEA
:109EF0009F0EF420F76EF86A000EF822020E9CEF17
:109F000016F04C64427344724D6C36EC3FF0146EA4
:109F10002FEC3FF0136E145002E1135006E0ACEC4E
:109F20005EF003E0020A39E029D00BEE00F0000EEB
:109F3000E926066AEE5011E07F0BD8B4200EABDFA5
:109F4000EE50062A06A8F8D712003C656D707479A9
:109F50003E2020202020202020204A0EF66E9F0E3A
:109F6000F76E000EF86E100E9CEF16F03C4E6F2050
:109F700042616E6B537469636B3E20206C0EF66E0B
:109F80009F0EF76E000EF86EEED73C6F6E6C792068
:109F900033326B2042533E2020208A0EF66E9F0EF5
:109FA000F76E000EF86EDFD7145006E0ACEC5EF0F2
:109FB00003E0020AF2E0E2D7A96AAA6A066AD8ECCC
:109FC0005EF07F0BCAE067DFD8EC5EF07F0BD8B4A1
:109FD000200E062A06A8F7D71200066E92EC16F09D
:109FE0007C0E59DF065010CBF5FF16EC94F00900FB
:109FF000F5CF07F00900F5CF08F00750080D740EF3
:10A00000F324F66E260EF420F76EF86A010EF8229D
:10A01000080E9CEC16F0200E3EDF0850ED0FD8B075
:10A02000ED0E130FC8EC16F012D013D01ED02AD0AC
:10A0300044D052D066D074D082D090D09CD0A4D0DE
:10A04000ACD0B4D0BCD0C4D0CED0D6D0D7D0070EF0
:10A050002AD74F0E20DF530E1EDF430E1CDF040EE7
:10A0600022D746696C7465722000620EF66EA00EEF
:10A07000F76E000EF86E070E9CEF16F03132333497
:10A08000355650414B0E07DF4E0E05DF4F0E03DFF6
:10A09000420E01DF230EFFDE0650070B010D7C0E82
:10A0A000F324F66EA00EF420F76EF86A000EF82284
:10A0B0000900F550F0DE200EEED6450EECDE580E0F
:10A0C000EADE540EE8DE230EE6DE0650070B010F33
:10A0D0008EEC16F0020EE7D64F0EDDDE530EDBDE01
:10A0E000430ED9DE230ED7DE0650030B04E08EECC0
:10A0F00016F0020ED8D6310ECEDE320ECCDE330E86
:10A10000CAD64D0EC8DE4F0EC6DE440EC4DE230E88
:10A11000C2DE0650070B010F8EEC16F0020EC3D6FE
:10A120004C0EB9DE460EB7DE4F0EB5DE230EB3DEA3
:10A130000650070B010F8EEC16F0020EB4D6450E3A
:10A14000AADE4E0EA8DE560EA6DE230EA4DE0638CC
:10A15000010B010F8EEC16F0020EA5D6570E9BDEFA
:10A16000540E99DE230E97DE0650030B010F8EEC82
:10A1700016F0030E98D64F0E8EDE530E8CDE430E75
:10A180008ADE200E88DE42D04C0E85DE460E83DE4F
:10A190004F0E81DE310E7FDE39D04C0E7CDE460E56
:10A1A0007ADE4F0E78DE320E76DE30D0450E73DE6C
:10A1B0004E0E71DE560E6FDE200E6DDE27D0420E83
:10A1C0006ADE4C0E68DE200E66DE200E64DE32D0C3
:10A1D0004C0E61DE460E5FDE4F0E5DDE310E06B4C4
:10A1E000320E59DE27D0450E56DE4E0E54DE560E88
:10A1F00052DE200E50DE1ED038D831D036D8200E98
:10A200004ADE06500F0B010F90EF16F00650070BB9
:10A210000BE0FF0F24E0200E3EDE490E3CDE065030
:10A22000070BFF0F8EEF16F0410E35DE6C0E33DE9E
:10A230006C0E31D60650030B0CE0FF0F10E0200E21
:10A240002ADE2D0E06A04C0E26DE2D0E06B0520E76
:10A2500022D6200E20DE4C0E1EDE520E1CD6430EE1
:10A260001ADE750E18DE720E16D6440E14DE720E4D
:10A2700012DE750E10DE6D0E0ED612503EE1F36A40
:10A28000F46A10EE3CF0F350E126F450100FA96E82
:10A2900023EC5FF00F0BE76E10EE38F0F350E12681
:10A2A000F450000FA96E23EC5FF0070BE76E10EE81
:10A2B00034F0F350E126F450010FA96E23EC5FF067
:10A2C000E76E10EE40F0F350E126810EE76EF32AC0
:10A2D000400EF426D6E1010E336EB9EC51F022ECBB
:10A2E00044F0020E336EB9EC51F022EC44F0030E50
:10A2F000336EB9EC51F022EC44F0000E3AD806D897
:10A30000125003E18DEC3EF01C84120010EE80F040
:10A3100020EEC0F0F56AE6CFDEFFF52AF5A8FBD700
:10A3200042EC52F010EE90F026EE60F0F56A000E6E
:10A33000E3CFF3FF000EF3CFDBFF010EE3CFF3FF1C
:10A34000010EF3CFDBFF020EE3CFF3FF020EF3CFDC
:10A35000DBFF030EE3CFF3FF030EF3CFDBFF080EAB
:10A36000E126180ED926F52A050EF564E0D789EF07
:10A370001CF0E838E834E834C00BA96E10EE80F029
:10A3800032EC5FF085C0F3FF320EF36003D0780E3D
:10A39000E8CF85F01200E838E834E834C00BA96E45
:10A3A00010EE80F010EF5FF0F46EE838E834E83437
:10A3B000C00BEE0FF66EF76AA40EF722F86A000ED5
:10A3C000F82210EE80F0400EF36E0900F5CFE6FFA4
:10A3D000F32EFBD700EE3CF0F45090C0EBFF00EE04
:10A3E00038F0F450EBCF80F000EE34F0F450EB5046
:10A3F0007F0BE8CF81F0120010EE80F0F36AE66A7E
:10A40000F32AF3ACFCD710EE80F020EEC0F0F56A32
:10A41000DECFE6FFF52AF5A8FBD710EE90F026EE8A
:10A4200060F0F56A000EDBCFF3FF000EF3CFE3FF21
:10A43000010EDBCFF3FF010EF3CFE3FF020EDBCF04
:10A44000F3FF020EF3CFE3FF030EDBCFF3FF030EA8
:10A45000F3CFE3FF080EE126180ED926F52A050EE4
:10A46000F564E0D71200000EA96E030EAA6E11501B
:10A47000B2EF16F0000EA96E030EAA6EB0EC16F045
:10A48000116E12002F0EF56EAF0EF46E080EF36E05
:10A49000066AC5C007F035EC1DF0F2CFF5FFF29E5D
:10A4A000F31CE8CF7AF0F41CE8CF7BF0F5CFF2FF95
:10A4B000F29A800ED56E1200000E336ED4EC51F07D
:10A4C00025DF010E336ED4EC51F022EC44F0020E85
:10A4D000336ED4EC51F022EC44F0030E336ED4EC26
:10A4E00051F022EC44F05DEC3EF08DEF3EF00000C8
:10A4F0000200027800000000006000000060000020
:10A500007F400000000010007F40000000001000AD
:10A510007F400000000010007F400000000010009D
:10A520007F400000000010007F400000000000009D
:10A5300000000278000000000060000000600100E0
:10A540007F400000000010007F400000000010006D
:10A550007F400000000010007F400000000010005D
:10A560007F400000000010007F400000000000005D
:10A57000000002780000000000600000006002009F
:10A580007F400000000010007F400000000010002D
:10A590007F400000000010007F400000000010001D
:10A5A0007F400000000010007F400000000000001D
:10A5B000000002780000000000600000006003005E
:10A5C0007F400000000010007F40000000001000ED
:10A5D0007F400000000010007F40000000001000DD
:10A5E0007F400000000010007F400000000010804D
:10A5F000050EF56E01EE00F0EE6AE9507F0BFCE10E
:10A60000F52EFAD726EE70F054EC81F026EE88F0A5
:10A6100054EC81F026EEA0F054EC81F026EEB8F078
:10A6200054EC81F026EED0F054EC81F026EEE8F008
:10A6300054EC81F0F56A06EE60F0F550180DF35019
:10A64000040FE926070EF36EEE6AF32EFDD707011D
:10A65000105109011019030B06E0076B090EF36E88
:10A66000EE6AF32EFDD7F52A050EF564E4D7010155
:10A6700007EE00F019EE00F0020EF36EEECFE6FFEB
:10A68000E950FCE1F32EFAD7F29E1F6B09EE54F06D
:10A6900011EEA4F023EE00F03DEC68F01F2B09EE64
:10A6A0005AF011EEA7F023EE40F03DEC68F0F28E88
:10A6B000BFEC5FF07BEC58F010C9E8FF030B1DE125
:10A6C000C6C0E8FF070B19E1010106EE60F00F0EAE
:10A6D000EB5013E012EE00F0016B100EEB507F0B0D
:10A6E000046F640E056FF1EC82F0180EE926180E67
:10A6F000E126012B050E0165F0D712EEA0F00C0E3D
:10A70000F56EDCEC59F00CC1E6FF0DC1E5FF040E5F
:10A71000E126F52EF6D71090120010C9E8FFE8B236
:10A720000BD0E8B002D0000E0DD0000E45B00AD814
:10A73000010E45B207D81200E8B003D0000E02D8CF
:10A7400012004650056E16EE60F0180DF350E1262B
:10A75000000EE350036EF00B31E1900E03123C0E3D
:10A76000046E010EE3500464046E10C9E8FFE8B201
:10A7700012D0E8B001D01ED070C9E8FF05B0C0C942
:10A78000E8FFE8A217D08CC9E8FF05B0DCC9E8FFF4
:10A79000070B04260FD0E8B00DD050C9E8FFE8AC95
:10A7A00005D051C9E8FF070B042604D046500C0F12
:10A7B000042600D0400E056EEFEC7FF01200F29EF2
:10A7C00010C9E8FF030B020A04E1006B12EC79F0F8
:10A7D0000ED0010112EE00F0016B010EE390E39642
:10A7E000E388180EE126012B050E0165F6D7F56A00
:10A7F00006EE60F0F550180DF350040FE926140E24
:10A80000F36EEE6AF32EFDD7F52A050EF564F0D748
:10A81000076B0201EC99FF990101F28E1200020E02
:10A82000F36E07EE00F019EE00F0EECFE6FFE95010
:10A83000FCE1F32EFAD70601646B7C6B946BAC6B76
:10A84000C46BDC6B0201086B206B386B506B686B60
:10A85000806BB6EF8CF05F5033620CD0020EF36E5B
:10A8600007EE00F01BEE00F0EECFE6FFE950FCE152
:10A87000F32EFAD71200A96AAA6A17EE00F0EAECE2
:10A880005EF0400EE126000EE222A950F8E1010E32
:10A89000AA64F5D7E0DFABD610CBE8FFE8B210D062
:10A8A000E8B007D0F60EF66EA80EF76E000EF86E42
:10A8B00016D0F60EF66EAA0EF76E000EF86E0FD0DA
:10A8C000E8B007D0F60EF66EAC0EF76E000EF86E1E
:10A8D00006D0F60EF66EAE0EF76E000EF86E0BEEAC
:10A8E00000F0020EF36E0900F5CFEEFFE950FBE138
:10A8F000F32EF9D712004C656164205061746368CF
:10A900002020202020200000000000000000000087
:10A910008000FF00008000FF00008000FF0000803A
:10A9200000FF00008000FF00008000FF500080005A
:10A93000FF00008000FF0080008000800080008019
:10A9400000800080008000007F00100002000000F6
:10A95000100002000000000400F000080000408029
:10A960000200001F0500001400F0000800004080F5
:10A970000200001F0500001400F0000800004080E5
:10A980000200001F0500000400F0000800004080E5
:10A990000200001F0500001400F0000800004080C5
:10A9A0000200001F0500001400F0000800004080B5
:10A9B0000200001F0500018000000001800000006F
:10A9C0000180000000018000000001800000000103
:10A9D00080000000000000C00030FF0000FF304099
:10A9E00020000080808000400050FF0000FF5010D9
:10A9F000300000808080010003C0000000000200E1
:10AA000003C000000000030003C0000000000400B9
:10AA100003C000000000050003C0000000000600A5
:10AA200003C000000000070003C000000000080091
:10AA300003C000000000FF000F3F03000000000003
:10AA40000000000000000000000000000000000006
:10AA5000000000000000F000000000000000000006
:10AA60000000CB00001F80CB00203FA0CB00405F48
:10AA7000C0CB00607FE0404040404040404040400C
:10AA800040404040404040404040404040404040C6
:10AA900040404040404040404040404040404040B6
:10AAA00040404040404040404040404040404040A6
:10AAB0004040404040404040404040404040404096
:10AAC0004040404040404040404040404040404086
:10AAD0004040404040404040404040404040404076
:10AAE0004040404040404040404040404040404066
:10AAF000404040404040426173736C696E65205035
:10AB00006174636820200100000000000000610003
:10AB10000800FF6500FF00FF69006000FF6D003066
:10AB200000FF71002000FF00008000FF5100800046
:10AB3000FF00008000FF0080008000800080008017
:10AB400000800080008000007F00170800F00000F7
:10AB5000170800F00000010400C000091000288060
:10AB60000228001F05000700000003800600008087
:10AB70008003801600008080008080A004382010B0
:10AB80008003000F0000280000000000000000000B
:10AB900000000000000000000000000000000000B5
:10ABA000000000000000010200C000091000288021
:10ABB0000228001F05000700000003800600008037
:10ABC0008003801600008080008080A00438201060
:10ABD0008003080F000028000000000000000000B3
:10ABE0000000000000000000000000000000000065
:10ABF0000000000000008080808080808080808055
:10AC00008080808080808080808080808080808044
:10AC10008080808080808080808080808080808034
:10AC20008080808080808080808080808080808024
:10AC30008080808080808080808080808080808014
:10AC40008080808080808080808080808080808004
:10AC500080808080808080808080808080808080F4
:10AC600080808080808080808080808080808080E4
:10AC70008080808080804040404040404040404054
:10AC800040404040404040404040404040404040C4
:10AC900040404040404040404040404040404040B4
:10ACA00040404040404040404040404040404040A4
:10ACB0004040404040404040404040404040404094
:10ACC0004040404040404040404040404040404084
:10ACD0004040404040404040404040404040404074
:10ACE0004040404040404040404040404040404064
:10ACF0004040404040404472756D204B69742020B4
:10AD00002020202020200200010000000000000080
:10AD10008000FF00008000FF00008000FF00008036
:10AD200000FF00008000FF00008000FF00008000A6
:10AD3000FF00008000FF0080008000800080008015
:10AD400000800080008003087F0F100002000000D8
:10AD5000100002000000000009C98080808000000F
:10AD6000000109C9808080800000000209C980803C
:10AD700080800000000309C9FF808080000000047B
:10AD800009C9808080800000000509C9808080801A
:10AD90000000000609C9808080800000000709C902
:10ADA000808080800000000809C9808080800000C9
:10ADB000000909C9808080800000000A09C98080DC
:10ADC00080800000000B09C9808080800000000C9A
:10ADD00009C9808080800000000D09C980808080C2
:10ADE0000000000E09C9808080800000000F09C9A2
:10ADF0008080808000001100110000000000000031
:10AE00000000000000000000000000000000000042
:10AE10000000000000001100110000000000000010
:10AE20000000000000000000000000000000000022
:10AE300000000000000011001100000000000000F0
:10AE40000000000000000000000000000000000002
:10AE500000000000000011001100000000000000D0
:10AE600000000000000000000000000000000000E2
:10AE700000000000000011001100000000000000B0
:10AE800000000000000000000000000000000000C2
:10AE90000000000000001100110000000000000090
:10AEA00000000000000000000000000000000000A2
:10AEB0000000000000001100110000000000000070
:10AEC0000000000000000000000000000000000082
:10AED0000000000000001100110000000000000050
:10AEE0000000000000000000000000000000000062
:10AEF0000000000000004D756C746920506174639F
:10AF00006820202020200300000000000000000036
:10AF10008000FF00008000FF00008000FF00008034
:10AF200000FF00008000FF00008000FF00008000A4
:10AF3000FF00008000FF0080008000800080008013
:10AF400000800080008000007F00100002000000F0
:10AF5000100002000000000400FA00080000408019
:10AF60000200001F0500080000790180060000C0F3
:10AF7000800180160000908000808080303040206A
:10AF800080C700000FD0000400FA000800004080D5
:10AF90000200001F0500080000790180060000C0C3
:10AFA000800180160000908000808080303040203A
:10AFB00080C700101FD0000400FA00080000408085
:10AFC0000200001F0500080000790180060000C093
:10AFD000800180160000908000808080303040200A
:10AFE00080C700202FD0000400FA00080000408035
:10AFF0000200001F0500080000790180060000C063
:10B0000080018016000090800080808030304020D9
:10B0100080C700303FD0000400FA000800004080E4
:10B020000200001F0500080000790180060000C032
:10B0300080018016000090800080808030304020A9
:10B0400080C700404FD0000400FA00080000408094
:10B050000200001F0500080000790180060000C002
:10B060008001801600009080008080803030402079
:10B0700080C700505FD0404040404040404040408A
:10B0800040404040404040404040404040404040C0
:10B0900040404040404040404040404040404040B0
:10B0A00040404040404040404040404040404040A0
:10B0B0004040404040404040404040404040404090
:10B0C0004040404040404040404040404040404080
:10B0D0004040404040404040404040404040404070
:10B0E0004040404040404040404040404040404060
:10B0F00040404040404016EEF0F0F36AF3CFE6FFE8
:10B10000F32A050EF364FAD716EEF6F0F36AE66852
:10B11000F32A050EF364FBD707D810EEFCF0E66ABD
:10B12000E66AE66AE66A1200F29E16EEF6F0F36A46
:10B13000E68CF32A050EF364FBD710C9E8FFE8B2EA
:10B1400001D028D0E8B012D019EE60F0F36A000EFA
:10B15000E3380F0BFD0FF46E060EF46001D01CD81F
:10B160000A0EE126F32AF3A8F2D714D019EE60F004
:10B17000F36A110EE3500F0BFD0FF46E060EF46030
:10B1800001D00AD8300EE126000EE222F32A050E85
:10B19000F364EFD7F28E120006EEF0F0F56AF55088
:10B1A000EB507F0BF41806E0F52A050EF564F7D78F
:10B1B000D2EF16F0F550060FEB9C120010C9E8FF15
:10B1C000030B01E198DF120001010239070BF56E54
:10B1D00002510F0B20E0FF0F1BE0FF0F4DE0FF0FB0
:10B1E000F46EF504F46406D0E81C010FF426F55063
:10B1F000F460F46A16EEF0F0F36AF350E3507F0B5C
:10B20000F4186EE0F32A050EF364F7D7D2EF16F0C8
:10B21000030EF560F56E16EEF0F0F36AF350E3CF2F
:10B22000F4FFF4BE07D0F350060FE3AC03D0F504EF
:10B23000F46456D0F32A050EF364F0D7F36AF350A2
:10B24000060FE3AC07D0F350E3507F0BF46EF50428
:10B25000F46446D0F32A050EF364F1D7F36AF35091
:10B26000E3507F0BF46EF504F4643AD0F32A050E34
:10B27000F364F5D7D2EF16F0030EF564CCD716EED3
:10B28000F0F0F36AF350E3CFF4FFF4BE07D0F350CD
:10B29000060FE3AC03D0030EF46022D0F32A050EB0
:10B2A000F364F0D7F36AF350060FE3AC07D0F35022
:10B2B000E3507F0BF46E030EF46012D0F32A050EF8
:10B2C000F364F1D7F36AF350E3507F0BF46E030E8F
:10B2D000F46006D0F32A050EF364F5D7D2EF16F02A
:10B2E000F350E38EE3CFF4FFF350050A1CE0F35074
:10B2F000060FE3CF01F1F328E3CFF5FFFF0FF5CF02
:10B30000E3FFF328060FE3CFF5FFFF0FF5CFE3FFD1
:10B31000F32A040EF364EFD7050EF36EF4CFE3FFC8
:10B320000B0E01C1E3FFF350060FE350400B001179
:10B33000F56EF350060FF5CFE3FFF4507F0BE8CF27
:10B3400001F112EE00F0180DF350E126F450E22264
:10B350001200F46E010116EEF0F0F36AF350E350C0
:10B360007F0BF41805E0F32A050EF364F7D72CD70A
:10B37000F350060FE3503F0B0019F9E10239070BB8
:10B38000F460F5D7ADD716EEF0F0F36AF350E35062
:10B390007F0B011906E0F32A050EF364F7D7D2EF0D
:10B3A00016F0F350E39E12EE00F00151180DF35029
:10B3B000E126F450E222120001010C510D03D65097
:10B3C000F3240C6F690ECE20F4200D6F1200F4DF11
:10B3D00001010D310C19F46E0350045C010F01E002
:10B3E000F402F45003241200FF0E056E036A046891
:10B3F000EEDF0514F36E051CE714F310E66EE15062
:10B40000E962F6D7E250EA62F3D71200036A080E47
:10B41000046EDDDFF56E030E046ED9DFE838E83424
:10B42000600BF5101200036A0F0E046ED0DFF56E8C
:10B43000080E046ECCDFE838F5101200010E036E22
:10B440001F0E046EC4DFF56EE10F05E17F0E046E82
:10B45000BEDF80091200F5501200010E036E0C0EC3
:10B46000046EB5DFF56E0F0E046EB1DFE838F5102F
:10B470001200070E036E280E046EA9D7EF0FD8B086
:10B48000EF0E110FC8EC16F0C3D20FD0D3D0E9D015
:10B4900052D19FD1EBD102D258D25CD260D264D2C9
:10B4A0007CD287D292D29DD2A8D210CBE8FFE8B24C
:10B4B0003FD0E8B01ED01BEE60F00BEEC0F094DF82
:10B4C0000B01536B1F0E511701011BEE60F0030EB1
:10B4D000066E58D8100EE126062EFBD70BEE60F054
:10B4E0001BEE90F0300E066EEECFE6FF062EFCD778
:10B4F00012000101066A1BEE60F00650500DF35079
:10B50000E126F450E222100EE124E96E000EE22062
:10B51000EA6E6ADF1BEE60F00650500DF350E12634
:10B52000F450E2262FD8062A010E0664E4D7120052
:10B53000E8B009D00101066A065054D8062A0F0E59
:10B540000664FAD712000101066A1BEE60F006508D
:10B55000300DF350E126F450E222100EE124E96EA2
:10B56000000EE220EA6E40DF1BEE60F00650300D68
:10B57000F350E126F450E22605D8062A050E0664AB
:10B58000E4D71200F36A070EF3CFE3FF036A030E5A
:10B59000046E1DDF0C0D340EF326080EF3CFE3FF0F
:10B5A000760E036E8A0E046E12DFF36E090EF3CF71
:10B5B000E3FF020EF36E0A0EF3CFE3FF27DFF36E15
:10B5C000010EF3CFE3FF036A0F0E046E00DFF36E8C
:10B5D0000B0EF3CFE3FFF36A0C0EF3CFE3FF000E85
:10B5E000E39412000A6E1BEE60F00A500A0DF3504D
:10B5F000E1260A0EE124E96E000EE220EA6EF4DE96
:10B600001BEE60F00A500A0DF350E126000EE36ACB
:10B61000020EE3500F0BF36E020EF3CFE3FF036A4B
:10B62000130E046ED4DEF36E010EF3CFE3FF080EAB
:10B63000E36A12001BEE54F00BEE60F0D5DE040E50
:10B64000E8CF56FBE8CF5CFB54CBE8FF770BE8CFA5
:10B6500054FBE8CF5AFB000E58CBE8FF5ECBE8FF67
:10B66000120010CBE8FFE8B233D0E8B00FD01BEEE9
:10B67000C0F00BEEDEF0B8DE1BEEC0F0060E066E7C
:10B680004CD8050EE126062EFBD712000101066AF2
:10B690001BEE74F00650500DF350E126F450E222F8
:10B6A0000E0EE124E96E000EE220EA6E9DDE1BEE36
:10B6B00074F00650500DF350E126F450E2262DD8D8
:10B6C000070EE1262AD8062A010E0664E1D71200E9
:10B6D000E8B001D012000101066A1BEE74F00650BA
:10B6E000300DF350E126F450E2220E0EE124E96E13
:10B6F000000EE220EA6E78DE1BEE74F00650300D8C
:10B70000F350E126F450E22608D8070EE12605D8CA
:10B71000062A050E0664E1D7120085DEF36E000EE0
:10B72000F3CFE3FF036A1F0E046E51DEF36E030EC8
:10B73000F3CFE3FF120010CBE8FFE8B231D0E8B05E
:10B7400019D01BEEE0F00CEE00F04EDE1BEEE0F048
:10B75000020E066E000EF3CFE3FF036A1F0E046EA7
:10B7600036DEF36E020EF3CFE3FF100EE126062E57
:10B77000F1D712000101066A1BEE82F00650500D4F
:10B78000F350E126F450E222090EE124E96E000EA6
:10B79000E220EA6E29DE062A010E0664EDD71200C9
:10B7A000E8B001D012000101066A1BEE82F00650DB
:10B7B000300DF350E126F450E222090EE124E96E47
:10B7C000000EE220EA6E10DE062A050E0664EDD7B2
:10B7D000120010CBE8FF030BD8A412001CEE00F0FF
:10B7E0000CEE40F001DE1CEE00F0080E066E26DEC8
:10B7F000F36E000EF3CFE3FF21DEF36E010EF3CF05
:10B80000E3FF2BDEF36E020EF3CFE3FF036A010EBC
:10B81000046EDDDD12E02DDEF36E060EF3CFE3FFE6
:10B8200028DEF36E070EF3CFE3FFF36A040EF3CFC7
:10B83000E3FF050EF3CFE3FF14D0F36A060EF3CF58
:10B84000E3FF070EF3CFE3FF036A070E046EBFDDCD
:10B85000C6EC16F0F36E040EF3CFE3FF050EF3CF44
:10B86000E3FF080EE126062EC2D7120010CBE8FF38
:10B87000030BD8A412001CEE40F00CEE6AF0B4DD0D
:10B88000FF0EE8CF40FC43CCE8FF3F09E8CF43FC84
:10B8900067CCE8FF3F0BE8CF67FC120010CBE8FF56
:10B8A000E8B212D0E8B00FD01CEE6CF00CEEB2F0A3
:10B8B0009BDD1CEE6CF0066A29D8050EE126062AEF
:10B8C00006A4FAD712001200E8B001D0120001015C
:10B8D000066A1BEE8BF00650300DF350E126F45053
:10B8E000E222050EE124E96E000EE220EA6E7CDD24
:10B8F0001BEE8BF00650300DF350E126F450E2269B
:10B9000005D8062A050E0664E4D71200036A0F0E56
:10B91000046E5DDDC009F36E000EF3CFE3FF065049
:10B92000200D020EF3CFE3FF1F0EF326030EF3CF1D
:10B93000E3FF040EE3509F0BF56E0650200DF5500B
:10B94000F326040EF3CFE3FF12001CEE80F00DEEA1
:10B9500000F04AD51BEE18F00BEE40F045D51BEE7B
:10B9600040F00BEE50F040D510CBE8FF030B010A7E
:10B9700013E11CEE00F00CEE80F03F0E36DD1CEE05
:10B9800000F0E7500F0BF36E0C0EF36402D0F70ECD
:10B99000E716E650E1AEF5D7120010CBE8FF030B37
:10B9A000010A06E11CEE00F00CEE80F0800E1DDDB9
:10B9B000120010CBE8FF030B010A06E11CEE00F0B9
:10B9C0000CEE80F0400E11DD120010CBE8FF030BEF
:10B9D000010A06E11CEE80F00DEE00F0800E05DDA0
:10B9E000120010CBE8FF030B010A06E11CEE80F009
:10B9F0000DEE00F07F0EF9DC120010CBE8FF030B18
:10BA0000020A05E11CEE00F00DEE00F0EDDC120084
:10BA10004CEC54F04ADD0EDE24DE8DDEDADE26DF6D
:10BA20003DDF93DF97DF9BDF9FD7B7D7C2D7CDD757
:10BA3000D8D7E3D71BEE00F010CBE8FF030B100DB7
:10BA4000600EF324F66EBA0EF420F76EF86A000E5C
:10BA5000F8220900F5CFE6FF0F0EE164FAD71200D5
:10BA600052616E646F6D204C65616420202020203F
:10BA700052616E646F6D20426173736C696E6520F4
:10BA800052616E646F6D204472756D7320202020AA
:10BA900052616E646F6D204D756C7469202020209A
:10BAA0001528070B156E5CD8B8EC16F016C006F01A
:10BAB00002B005D01550C4EC16F0161604D015507F
:10BAC000C6EC16F016121650061849E01550C6ECD2
:10BAD00016F0161413E115504CEC5FF0070E151814
:10BAE00004E1116A0A0E316E3AD060C6E8FF0F0B0E
:10BAF000C009036E046AA1EC80F031D0155044EC0B
:10BB00005FF00A0E316E320ECEEC16F0070E1518ED
:10BB10000AE126D8B8EC16F0A90A1EE1B8EC16F036
:10BB20004E0A1AE109D01CD8B8EC16F0F30A14E159
:10BB3000B8EC16F08B0A10E11550C4EC16F017168D
:10BB4000B8EC16F0400A04E11550C6EC16F01712D6
:10BB500015C014F0F4D803D015C014F028D8120082
:10BB60001550EEEC16F0036A046A120000142A2045
:10BB7000466F726D617474696E672078786B202AE5
:10BB8000202040142A2050617463682078202030DF
:10BB900020202020202A202040142A20456E736572
:10BBA0006D626C65203030302020202A2020145017
:10BBB000EEEC16F0036A800E046EB8EC16F0F36E2D
:10BBC000420F036A046ABAEC16F0036A800E046E30
:10BBD000B8EC16F0F31806E01550C4EC16F0171682
:10BBE000200E05D01550C6EC16F01712400EF36E5D
:10BBF000020E036E046AF350BAEC16F06C0EF66E89
:10BC0000BB0EF76E000EF86E9AEC16F09AEC16F07A
:10BC10000D0E88EC16F0F35090EC16F0070E151888
:10BC200029E19AEC16F0010E116E4B0E88EC16F01D
:10BC3000112892EC16F0A96A020EAA6E040010EE0A
:10BC400080F01AEC17F0C00EA92610EC5FF0A95096
:10BC5000F5E1112A11AEE9D714C015F081DFA90E64
:10BC6000BAEC16F04E0EBAEC16F0010E116E33EC73
:10BC700052F04CD0480E88EC16F01450410F94EC62
:10BC800016F04CEC54F00BEE00F0EE6AE9A8FDD78C
:10BC9000010E136E490E88EC16F0132892EC16F084
:10BCA000135054EC5FF01BEE00F0A96AAA6A04007E
:10BCB000C2EC5EF0400EE126000EE222A950F7E150
:10BCC000010EAA64F4D7132A1450C6EC16F0171408
:10BCD0007F0ED8B43F0E1364DDD7030E036E046AE3
:10BCE0000400000EBAEC16F00350FAE1010E0464F1
:10BCF000F7D714C015F034DFF30EBAEC16F08B0E44
:10BD0000BAEC16F0136A145044EC5FF00A0E316E70
:10BD1000120000142A20466978696E6720202020CE
:10BD200020202020202A202040142A2050617463E3
:10BD300068207820203020202020202A2020120077
:10BD4000A9CF03F01334FE0BAAB00109046E1450FE
:10BD5000070B8009EEEF16F01450070B070A10E0EE
:10BD60001450C6EC16F01614010E0AE013AC06D0FF
:10BD70001450C6EC16F01714020E02E0000B12006D
:10BD8000FF091200C00EA916E7DF0BE1135009E00E
:10BD9000D7DFF2EC16F000E0400EA926000EAA2232
:10BDA00005D01CEC17F0A952D8B4AA2A0101120040
:10BDB000D3DF09E1135007E0C3DFB8EC16F0A92A7E
:10BDC000D8B4AA2A05D0B0EC16F0A952D8B4AA2A41
:10BDD00001011200C00EA916BFDF0AE1135008E0EE
:10BDE000AFDF18EC17F0400EA926000EAA2205D0EE
:10BDF0001AEC17F0A952D8B4AA2A01011200A9CF4F
:10BE000003F011507F0B046E870EEEEF16F0070E55
:10BE1000C6EC16F0161402E1FF091200000B120026
:10BE2000C00EA916F4DF09E1115007E0E8DFF2ECDB
:10BE300016F000E0400EA92604D0020EAA6E1CECFB
:10BE400017F001011200E3DF07E1115005E0D7DF31
:10BE5000B8EC16F0A92A04D0020EAA6EB0EC16F0C7
:10BE600001011200C00EA916D2DF08E1115006E050
:10BE7000C6DF18EC17F0400EA92604D0020EAA6EF9
:10BE80001AEC17F00101120065D819D8F55053D8F3
:10BE90004CD8040E53D829D05DD811D8F5504BD8C2
:10BEA00044D8040E4BD821D00AD8540E44D8480E9A
:10BEB00042D8040E43D839D8020E40D816D010808C
:10BEC00003010F0E186F586F176B576B0B6B4B6B93
:10BED000126B526B880E056B456B066F466F080E32
:10BEE000036F436F026B426B1200F7EF52F0150FB6
:10BEF000E8BE7F0E020D200EF324F66E3D0EF420F8
:10BF0000F76EF86A010EF8220900F5CF00F3F5CFBD
:10BF100040F30900F5CF01F3F5CF41F3410EE8CF2F
:10BF200004F3E8CF44F3E4EF5FF00301400E046F45
:10BF3000446FE4EF5FF0DBDF020E00D0066E04001A
:10BF40000A0ECEEC16F0062EFBD71200393D404506
:10BF5000494C5139010D4C0EF324F66EBF0EF420FE
:10BF6000F76EF86A000EF8220900F550120003EE91
:10BF700020F013EE60F0036A000EF2D904D2F29EB4
:10BF8000190E066E02EEFFF013EE3FF0EC28F36E92
:10BF9000200EF3CFEBFFE428F36E200EF3CFE3FF88
:10BFA000062EF4D7030104870B87128744874B873B
:10BFB00052870AD8030104970B97129744974B971F
:10BFC000529702D010B0120003EE20F013EE60F092
:10BFD000E00E036E0301F29E0051406307D0205132
:10BFE000606304D000512063E1D906D00051206382
:10BFF000B7D940516063C7D9032A0151416307D0C3
:10C000002151616304D001512163D0D906D001517F
:10C010002163A6D941516163B6D9032A0251426313
:10C0200007D02251626304D002512263BFD906D0E7
:10C030000251226395D942516263A5D9032A035163
:10C04000436307D02351636304D003512363AED904
:10C0500006D00351236384D94351636394D9032ADF
:10C06000032A0551456307D02551656304D0055166
:10C0700025639CD906D00551256372D94551656366
:10C0800082D9032A0651466307D02651666304D03D
:10C09000065126638BD906D00651266361D94651D5
:10C0A000666371D9032A0751476307D02751676335
:10C0B00004D0075127637AD906D00751276350D996
:10C0C0004751676360D9032A0851486307D0285154
:10C0D000686304D00851286369D906D008512863E1
:10C0E0003FD9485168634FD9032A0951496307D0A2
:10C0F0002951696304D00951296358D906D00951DF
:10C1000029632ED9495169633ED9032A0A514A63EA
:10C1100007D02A516A6304D00A512A6347D906D04E
:10C120000A512A631DD94A516A632DD9032A032A69
:10C130000C514C6307D02C516C6304D00C512C6310
:10C1400035D906D00C512C630BD94C516C631BD9DB
:10C15000032A0D514D6307D02D516D6304D00D514D
:10C160002D6324D906D00D512D63FAD84D516D633E
:10C170000AD9032A0E514E6307D02E516E6304D0A4
:10C180000E512E6313D906D00E512E63E9D84E51AD
:10C190006E63F9D8032A0F514F6307D02F516F6395
:10C1A00004D00F512F6302D906D00F512F63D8D876
:10C1B0004F516F63E8D8032A1051506307D03051B4
:10C1C000706304D010513063F1D806D01051306341
:10C1D000C7D850517063D7D8032A1151516307D083
:10C1E0003151716304D011513163E0D806D011513F
:10C1F0003163B6D851517163C6D8032A032A13514B
:10C20000536307D03351736304D013513363CED8D3
:10C2100006D013513363A4D853517363B4D8032A9F
:10C220001451546307D03451746304D014513463EF
:10C23000BDD806D01451346393D854517463A3D835
:10C24000032AF28EF29EE40E036E0451446307D07B
:10C250002451646304D004512463A8D806D0045147
:10C2600024637ED8445164638ED8032AEB0E036E98
:10C270000B514B6307D02B516B6304D00B512B63D5
:10C2800095D806D00B512B636BD84B516B637BD881
:10C29000032AF20E036E1251526307D032517263B9
:10C2A00004D01251326382D806D01251326358D86A
:10C2B0005251726368D8032AF50E036E1551556307
:10C2C00007D03551756304D0155135636FD806D04A
:10C2D0001551356345D85551756355D8032A165104
:10C2E000566307D03651766304D0165136635ED854
:10C2F00006D01651366334D85651766344D8032A93
:10C300001751576307D03751776304D017513763FC
:10C310004DD806D01751376323D85751776333D898
:10C32000032A1851586307D03851786304D0185144
:10C3300038633CD806D01851386312D85851786306
:10C3400022D8032A0101385107E010C9E8FF030B86
:10C3500002E198D839D61CD90101396BF28E12004E
:10C36000046E03501F0B04C0EBFF37D882A4FED726
:10C3700082B4FED78B9A00D000D000D000D000D07D
:10C3800000D08B8A1200046E03501F0B04C0E3FF21
:10C3900024D882A4FED782B4FED78C9800D000D0D7
:10C3A00000D000D000D000D08C881200046E035062
:10C3B0001F0B04C0EBFF04C0E3FF0FD882A4FED71D
:10C3C00082B4FED78B9A8C9800D000D000D000D0D9
:10C3D00000D000D08B8A8C8812008C9A8C9C04B080
:10C3E0008C8C8C8A8C9A8C9C04B28C8C8C8A8C9AC7
:10C3F0008C9C04B48C8C8C8A8C9A8C9C04B68C8C0F
:10C400008C8A8C9A8C9C04B88C8C8C8A8C9A8C9C90
:10C4100004BA8C8C8C8A8C9A8C9C04BC8C8C8C8AF4
:10C420008C9A8C9C04BE8C8C8C8A8C9A8C9C03B0CD
:10C430008C8C8C8A8C9A8C9C03B28C8C8C8A8C9A77
:10C440008C9C03B48C8C8C8A8C9A8C9C03B68C8CC0
:10C450008C8A8C9A8C9C03B88C8C8C8A8C9A8C9C41
:10C4600003BA8C8C8C8A8C9A8C9C03BC8C8C8C8AA6
:10C470008C9A8C9C03BE8C8C8C8A8C9A8B888C9C1E
:10C480008B9812000301F28EF29EE00E036EFF0EF7
:10C490008DDF032AFF0E8ADFE70E036EFF0E86DFB5
:10C4A000032AFF0E83DFEE0E036EFF0E7FDF032AEB
:10C4B000FF0E7CDF04970B97129744974B97529788
:10C4C00038C1E8FFE8B00481E8B20B81E8B412811A
:10C4D000E8B64481E8B84B81E8BA5281E40E036EB5
:10C4E0000451446307D02451646304D0045124638D
:10C4F0005DDF06D00451246333DF4451646343DFBE
:10C50000032A53C9E8FF0E0FD8B0FF0E066E0000D5
:10C51000000000000000000000000000062EF7D719
:10C52000EB0E036E0B514B6307D02B516B6304D0A2
:10C530000B512B633BDF06D00B512B6311DF4B51AB
:10C540006B6321DF032A53C9E8FF0E0FD8B0FF0E3B
:10C55000066E000000000000000000000000000067
:10C56000062EF7D7F20E036E1251526307D03251E6
:10C57000726304D01251326319DF06D01251326354
:10C58000EFDE52517263FFDE032A0101386B1200A5
:10C59000030138C1E8FFE8B00497E8B20B97E8B4AC
:10C5A0001297E8B64497E8B84B97E8BA5297E8B0C4
:10C5B0000481E8B20B81E8B41281E8B64481E8B89E
:10C5C0004B81E8BA5281E40E036E0451446307D0F4
:10C5D0002451646304D004512463E8DE06D004517E
:10C5E0002463BEDE44516463CEDE032AEB0E036E89
:10C5F0000B514B6307D02B516B6304D00B512B6352
:10C60000D5DE06D00B512B63ABDE4B516B63BBDE2B
:10C61000032AF20E036E1251526307D03251726335
:10C6200004D012513263C2DE06D01251326398DE5A
:10C6300052517263A8DE032A0101386B1200F29E88
:10C64000C7C0E8FF8DEC1CF07CEC1CF00301EB5143
:10C65000EC1905E0EBC3ECF3EB517BEC1CF0F28E34
:10C660001200010110B0120010B21200E9CF7CF0EC
:10C67000EACF7DF0F3CF7EF0F4CF7FF010C9E8FF72
:10C68000E8B208D0E8B003D090EC6AF00BD0D7EC59
:10C6900071F008D0E8B003D0CBEC74F003D06DECAF
:10C6A00079F000D07CC0E9FF7DC0EAFF7EC0F3FFD7
:10C6B0007FC0F4FF12001E973D29D8A43D2BC2C0B5
:10C6C000E8FFE8B206D0E8B002D0109806D0108893
:10C6D00004D010983D29D8A410883E0709E13F51A5
:10C6E000030A06E03F2B3B2B3C31E8303F0B3E6F0B
:10C6F0001EA90FD0326B10C9E8FF030B01E009D06F
:10C7000067CAE8FF331368CAE8FF341369CAE8FF51
:10C7100035133B5103E03B0710B80FD010B82DD0B4
:10C72000F2A42BD0F2940001D59E7A51D6247B51ED
:10C73000D7227A51D626D58E0101322B32510F0BDA
:10C74000060A04E13251100FF00B326F1E8710C938
:10C75000E8FF030B03E0800E35130FD01AEE5EF0F6
:10C760000DD81AEE61F032510F0BD8B407D81AEE7B
:10C7700064F03251300BD8B401D81200E6503313B4
:10C78000E6503413E650351312001E911E931E9589
:10C790001EB903D0060EDBA411D0090EDB680A0E09
:10C7A000DB68060EDB921E831EB903D00C0EEBBCB9
:10C7B00005D0070EDB68080EDB681E811EA72ED091
:10C7C0000C0EEBAE06D00F0EDB50D8B4010EF36E9C
:10C7D00002D0010EF36E070EDB50F3260D0EEB5068
:10C7E0003F0B010FF46EF404F36407D0F450F35ED2
:10C7F0001E81010EE3A01E85F6D7070EF3CFDBFFE7
:10C80000080EDB2ADB04F36E0E0EEB501F0B010F3C
:10C81000F36001D003D0080EDB6A1E850C0EEBBA64
:10C8200005D0060EDBA604D0DB9605D0060EDB860F
:10C830000C0EEBB023D0060EDBA0FCD0DB900F0E6D
:10C84000F36EF350DB6AF32A170EF364FAD710C9BC
:10C85000E8FF030B05E01F51C6EC16F037130AD0B2
:10C8600043CAE8FFC00B331344CAE8FF341345CA78
:10C87000E8FF3513010EE396E388DCD0060EDB807B
:10C880000C0EEBBA06D00C0EEBBC03D0010EE3A0ED
:10C8900002D01EA518D0010EE3A415D0E396E388BC
:10C8A00010C9E8FF030B05E01F51C6EC16F0371363
:10C8B0000AD043CAE8FFC00B331344CAE8FF34135D
:10C8C00045CAE8FF35131EA1B5D0090EDB50AA0AF0
:10C8D000D8B4B0D0090EDB2A080EDB6A090EDBCF14
:10C8E000F3FF080EF360F36AF350100FDB50D8B477
:10C8F000F36AF350100FDB50D8B49CD0090EF3CF7D
:10C90000DBFF0C0EEB30060B060A2CE00C0EEBB630
:10C9100002D0EBA41BD0F3500EE1060EDB720C0E1E
:10C92000EBB601D0F32AF350100FDB50D8B4F36A02
:10C93000090EF3CFDBFF0C0EEBB204D0060EDBB218
:10C9400018D007D0060EDBB204D013D00C0EEBA229
:10C9500010D00F0EDB5005E0FF0FF46EF350F45CC7
:10C96000F36E07D0DCEC59F00F0EDB500C03F4CF64
:10C97000F3FF0D0EEBAE13D01EB311D0F350100F1A
:10C98000DB5007E0F350090EDB5009E10A0EDB50E3
:10C9900006E1AA0EF36E090EF3CFDBFF4BD0F35086
:10C9A000100FDB507F0BF46E040ED8A4F4CFE3FF1E
:10C9B000F3500DE10A0EDB2ADB04F36E0E0EEB38AA
:10C9C000E830070BF36001D002D00A0EDB6A0A0ED2
:10C9D000DB500EE00C0D040EE350F324F46E6B0EEE
:10C9E000F46403D0F40EF426FAD7040EF4CFE3FF78
:10C9F000010EE3A01FD0010EE398E3B41BD0E38641
:10CA000010C9E8FF030B0CE01F51C6EC16F03613FB
:10CA10001F51020FC6EC16F034133F0E35130AD027
:10CA200040CAE8FFC00B331341CAE8FF341342CABF
:10CA3000E8FF3513060EDB941200010EEBCF0BF06E
:10CA4000D6EC69F0010EE3A207D00BB80AD0010EB4
:10CA5000E392E3B0E38605D00BA803D0010EE38296
:10CA6000E388010EE3A4E398E3B803D0E3B610D063
:10CA700074D0E398040EDB96000EEBB402D0040EE3
:10CA8000DB90010EE3941F51C6EC16F0391365D00C
:10CA90001F51C6EC16F0391560E10BB85CD0110ED1
:10CAA000E126E650E5101FE010C9E8FF030B020A7B
:10CAB00002E10D6A03D0070EEBCF0DF012C9E8FFBB
:10CAC000E8A004D0190E0D26D8B00D68800E97ECA2
:10CAD00069F00350E6260450E52203E2EF0EE1265A
:10CAE0003ED0E66AE56AEF0EE126010EE39612C932
:10CAF000E8FFE8A011D0020EEBCFF3FF050EF3CF55
:10CB0000DBFF030EEBCFF3FF010EE3AC02D0F00E20
:10CB1000F312060EF3CFDBFF10C9E8FFE8B20BD02B
:10CB2000E8B005D053C9E8FFFF0B13E00AD0100EA0
:10CB3000EBA80FD00ED0E8B001D00BD0100EEBA8B0
:10CB400008D0040EDB86DB901F51C6EC16F03813BC
:10CB500002D0040EDB80010EE384FF091200000BFB
:10CB600012000C0EEBA002D0040E01D0030EE3CF96
:10CB700025F126EE60F0000EE350180DF350D92693
:10CB800010C9E8FF030B010A06E1100EEBA207D063
:10CB9000400E0B6E07D0010A02E126EE60F0030E94
:10CBA000DBCF0BF0080EEB500B248008FF0A0B6E56
:10CBB0002525010FE8AE04D00BAE7F0E0BBE000E94
:10CBC000256F070EE350256301D00AD0070E25C15B
:10CBD000E3FF000EEBA204D00F0EE368100EE36833
:10CBE000010EE3AA42D0000EEBA23FD00B0EEB5099
:10CBF000D8B43BD0D890E830020DA00EF324F66EE6
:10CC0000380EF420F76EF86A010EF8220900F5CF0D
:10CC100016F10900F5CF17F10F0EE3501627100E8D
:10CC2000E35017230AE20F0E16C1E3FF100E17C1DF
:10CC3000E3FF060EE3CF25F123D00F0EE36A100EBB
:10CC4000E36A060EE3500B6E256502D00B2A01D075
:10CC50000B060BBE0AD00B50256301D006D00BC0CB
:10CC600025F1060E25C1E3FF0BD0070EE3CF25F11A
:10CC7000060E25C1E3FF000EEBA202D0010EE39ADF
:10CC8000C3C0E8FFE8A805D0236BD8902535246FF2
:10CC900014D02551150FE8BE7F0E020D200EF3248F
:10CCA000F66E3D0EF420F76EF86A010EF8220900C8
:10CCB000F5CF23F10900F5CF24F10A0EEB50D8B4DB
:10CCC00099D0186B196B10C9E8FFE8B205D0E8B02D
:10CCD00003D0080EE35002D0040EDB500B6E07E0C9
:10CCE000D8900B341827000E0BBEFF0E1923090E27
:10CCF000EB500B6E800A07E0D8900B341827000E1B
:10CD00000BAEFF0E192310C9E8FF030B2DE109013B
:10CD10005151010129E00B6E1FB516D01FB30CD085
:10CD20001FB109D0C2C0E8FFE8BC1ED0D8900B32BA
:10CD3000D8900B3215D014D01FB101D009D0D890A3
:10CD40000B32D8900B3204D01FB101D001D008D0E3
:10CD50000B1C010F18270B50D8A4FF0E192304D069
:10CD60000B501827000E19231851191143E019BF51
:10CD700006D00A0EEB502525E8BE7F0E05D00A0E20
:10CD8000EB50255DE8BE000EC3C0F3FFF3A805D04D
:10CD9000036AD890E834046E13D0150FE8BE7F0EF6
:10CDA000020D200EF324F66E3D0EF420F76EF86AA5
:10CDB000010EF8220900F5CF03F00900F5CF04F0C9
:10CDC00019BF0CD02351035C166F24510458176F00
:10CDD00017AF0AD016697F0E176F06D00350235D78
:10CDE000166F04502459176F27EC1DF01B51232791
:10CDF0001C512423090E23C1E3FF0A0E24C1E3FFC3
:10CE000001DBD6EC69F00B0EE350236305D00C0E6A
:10CE1000E350246301D017D00B0E23C1E3FF0C0EA7
:10CE200024C1E3FFDE50DD10D8B48AD00D0EDECF72
:10CE3000E3FF0E0EDDCFE3FF000EEBB204D00F0ECA
:10CE4000E36A100EE36A010EE3AA7AD0000EEBB299
:10CE500077D0020EE3B002D0E38072D00B0EEB501D
:10CE6000D8B46ED0020DA00EF324F66E380EF42066
:10CE7000F76EF86A010EF8220900F5CF16F10900E5
:10CE8000F5CF17F1000EEBA039D00F0EE3501627A7
:10CE9000100EE350172302E3166917690F0E16C12F
:10CEA000E3FF100E17C1E3FF0D0EE350235D0B6E81
:10CEB0000E0EE35024590C6E5DEC69F0040E0B2647
:10CEC000000E0C220BC018F10CC019F10AEC1DF079
:10CED0000DB009D00D0EE3501C25DE6E0E0EE35092
:10CEE0001D21DD6E1ED00D0EE3CFDEFF0E0EE3CF53
:10CEF000DDFF1C51DE5E1D51DD5A1DD0DECF18F165
:10CF0000DDCF19F10AEC1DF01C511D11D8B41C2BFA
:10CF10002351DE5C2451DD580AE21C51DE261D51EE
:10CF2000DD22DE50235DDD50245913E209D01C516F
:10CF3000DE5E1D51DD5A2351DE5C2451DD5809E2CD
:10CF400023C1DEFF24C1DDFF000EEBB202D0010ED3
:10CF5000E39AC3C0E8FFE8A618D0C40E1F25F66EFA
:10CF6000F76ACF0EF722F86A000EF8220900F55092
:10CF70000CE0036AD8902535046EF50493EC1CF0A0
:10CF80000101F504C6EC16F03A13C3C0E8FFE8A8A7
:10CF900018D0CA0E1F25F66EF76ACF0EF722F86A70
:10CFA000000EF8220900F5500CE0DECF03F0DDCFD3
:10CFB00004F0F50493EC1CF00101F504C6EC16F046
:10CFC0003A131200070000080000070000080000E4
:10CFD000040EEBCF0BF0050EEB500F0B0C6E0C3A62
:10CFE0000B380F0B0C120B38F00B0B6EECEC69F0DE
:10CFF0001F51060F030D11EE80F0F350E126E650AD
:10D000000B26E6500C22E7BE06D0E75001E108E30C
:10D010000B680C6805D0E71C01E102E20B6A0C6AA0
:10D020000B380F0B0D6E0C38F00B0D120C380F0B6C
:10D030000E6E0DC0DEFF0EC0DDFFC3C0E8FFE8A42A
:10D0400018D0740E1F25F66EF76AD00EF722F86A14
:10D05000000EF8220900F5500CE00BC003F00CC0E4
:10D0600004F0F50493EC1CF00101F504C6EC16F095
:10D070003A131200050000060000010EEBCF0BF082
:10D08000020EEB500F0B0C6E0C3A0B380F0B0C1200
:10D090000B38F00B0B6EE750E6240D6EE750E620E0
:10D0A0000E6EE750E6200F6E0D500B260E500C2230
:10D0B0000FBE06D00F5001E108E30B680C6805D0E5
:10D0C0000F1C01E102E20B6A0C6A10C9E8FF030BB6
:10D0D000010A12E1040EEB500FE0F36E07C2E8FF05
:10D0E0001FB14FC2E8FF7F0BF302F3500B26F45041
:10D0F0000C2202E30B680C681FB109D0C8C00DF008
:10D10000C9C00EF0CAC0F3FFCBC0F4FF08D0CCC03A
:10D110000DF0CDC00EF0CEC0F3FFCFC0F4FF0D5028
:10D12000F35CE8CF16F10E50F458E8CF17F10BC0BE
:10D1300018F10CC019F10AEC1DF00D501C250B6EF6
:10D140000E501D210C6E020EEBAE07D013EED0F088
:10D150001F51D8A413EED6F080D90B38E830070B56
:10D160000D6E150E0DC0DBFF160E0CC0DBFFC3C02D
:10D17000E8FFE8A01CD00BC003F00CC004F0000EC8
:10D180001FB1020E93EC1CF00101000E010904090D
:10D190003A13030EEBCF04F0036A010E1FB1030E26
:10D1A00093EC1CF00101000E020908093A13000E6D
:10D1B000EB500F0BF36E030EEB50F00BF312170E48
:10D1C000F3CFDBFF0B6A52C90CF0D8900C361F511D
:10D1D0000E0F030D11EE80F0F350E126E6500B2602
:10D1E000E6500C22E7BE06D0E75001E108E30B68E9
:10D1F0000C6805D0E71C01E102E20B6A0C6AC3C0AF
:10D200000DF00C380F0B0DB20F0EF36E000EEB503D
:10D21000F00BF312180EF3CFDBFF0DA20ED00BC0F4
:10D2200003F00CC004F0040E1FB1050E93EC1CF0CB
:10D230000101000E100920093A1312001F51C6EC1B
:10D2400016F03A1508E1EECF03F0EDCF04F01F51D0
:10D2500093EC1CF00101120013EEEBF014C9E7FF90
:10D260000201E79001B5E780E79249B5E782010145
:10D270001200F56E2CD8D890E834186F196B27EC93
:10D280001DF0F5BE08D01B1F1C1F1D1F1B2BD8B483
:10D290001C2BD8B41D2B12001EAFEBD71B6FE8AEB2
:10D2A00006D0060EEB501B25E8AEFF0EE2D7060EA9
:10D2B000EB1C010FE8BE000EDCD70D6A0CAE06D0E9
:10D2C0000D800B1E0C1E0B2AD8B40C2A1200E8503D
:10D2D000D8B4010FE8AE80087F0B1200010EE350B6
:10D2E0000B6001D011D0E6500326E550042205E280
:10D2F0000350000804500B5805E20BC004F0036A09
:10D30000000B1200FF0912000350E65C036E04508C
:10D31000E558046E05E3000E035C0B50045805E26B
:10D320000BC004F0036A000B1200FF0912000B6E21
:10D33000800A12E10D50020DA00EF324F66E380E95
:10D34000F420F76EF86A010EF8220900F5CF03F019
:10D350000900F5CF04F01200010EE3CF0CF0D890D5
:10D360000D320B50B4DF0BBE7F0A0C020BAE07D0A0
:10D370000D1E0D9EF4500D5CE8BE000E05D00D1C78
:10D380007F0BF424E8BE7F0E7F0B020D200EF324EA
:10D39000F66E3D0EF420F76EF86A010EF8220900D1
:10D3A000F5CF03F00900F5CF04F012001FB50ED041
:10D3B0001FB306D023EE00F01FB123EE07F01200DA
:10D3C00023EE0EF01FB123EE40F0120023EE47F0E3
:10D3D0001FB123EE4EF012001FB50ED01FB306D0C2
:10D3E00023EE02F01FB123EE09F0120023EE10F03D
:10D3F0001FB123EE42F0120023EE49F01FB123EEDD
:10D4000050F012001F51000F030D21EE80F0F35079
:10D41000D926DECFF3FFDECFF4FFDECFF5FFD890C5
:10D42000F5BED880F532F432F332D890F5BED8800C
:10D43000F532F432F332F3502327F4502423F5BEAF
:10D4400006D0F55001E108E32369246905D0F51CF5
:10D4500001E102E2236B246B1200D8900C320B32F4
:10D46000000EE3500B6205D0010EE3500C6201D0B8
:10D4700023D0000E0BC0E3FF010E0CC0E3FF020E31
:10D48000E3500B5C0B6E030EE3500C580C6E0C3229
:10D490000B320C320B320C320B320C501F0BE8B833
:10D4A000E0090C6E0B500C10D8B40B2A040E0BC004
:10D4B000E3FF050E0CC0E3FF020EE3CF0BF0030EFB
:10D4C000E3CF0CF0000EE3500B6205D0010EE350E9
:10D4D0000C6201D01BD0040EE3500B26050EE35066
:10D4E0000C220CBE0AD0000EE3500B5C010EE35080
:10D4F0000C58050EE3BE08D009E3000EE3CF0BF095
:10D50000010EE3CF0CF002D001E2F7D7020E0BC000
:10D51000E3FF030E0CC0E3FFD8900B360C3612006D
:10D52000010110BA6DD0108A3A6B1F6B09EEC0F082
:10D5300012EEA0F0DBEC6DF01F2B09EEC5F012EE41
:10D54000A4F0DBEC6DF01F2B09EECAF012EEA8F090
:10D55000DBEC6DF01F2B09EECFF012EEACF0DBEC44
:10D560006DF01F2B09EED4F012EEB0F0DBEC6DF095
:10D570001F2B09EED9F012EEB4F0DBEC6DF01F2B8F
:10D580001F6B09EEE0F012EED0F01BEC6FF01F2BDA
:10D5900009EEF0F012EED5F01BEC6FF01F2B800EB1
:10D5A0000B6E01EE80F0EE6A0B2EFDD71F6B0AEEBC
:10D5B00000F0DCEC6FF01F2B0AEE08F0DCEC6FF0F3
:10D5C0001F2B0AEE10F0DCEC6FF01F2B0AEE18F0A8
:10D5D000DCEC6FF01F2B0AEE20F0DCEC6FF01F2B61
:10D5E0000AEE28F0DCEC6FF01F2B0AEE30F0DCECDA
:10D5F0006FF01F2B0AEE38F0DCEC6FF01F2BD8D049
:10D60000109A5BEC63F01F6B0AEE6CF022EEEEF00A
:10D6100061D91F2B0AEE71F022EEF0F05BD91F2BBF
:10D620000AEE76F022EEF2F055D91F2B0AEE7BF0CF
:10D6300022EEF4F04FD91F2B356B1F6B09EE60F013
:10D6400012EE00F026EE60F0C5EC63F01F2B09EE41
:10D6500070F012EE18F026EE78F0C5EC63F01F2B98
:10D6600009EE80F012EE30F026EE90F0C5EC63F09B
:10D670001F2BC2C0E8FFE8BC1BD009EE90F012EEF1
:10D6800048F026EEA8F0C5EC63F01F2B09EEA0F0E1
:10D6900012EE60F026EEC0F0C5EC63F01F2B09EE31
:10D6A000B0F012EE78F026EED8F0C5EC63F01F2B48
:10D6B0000DEC6DF01F6B09EE60F012EE00F003D977
:10D6C0001F2B09EE70F012EE18F0FDD81F2B09EE9B
:10D6D00080F012EE30F0F7D81F2BC2C0E8FFE8BC94
:10D6E00012D009EE90F012EE48F0EDD81F2B09EEA3
:10D6F000A0F012EE60F0E7D81F2B09EEB0F012EEAA
:10D7000078F0E1D81F2B1F6B09EE54F011EEA4F056
:10D7100023EE00F03DEC68F0C2C0E8FFE8BC09D0A1
:10D720001F2B09EE5AF011EEA7F023EE40F03DEC6E
:10D7300068F01F6B09EE40F021EED4F0A0EC6DF024
:10D740001F2B09EE42F021EED7F0A0EC6DF01F2B5D
:10D7500009EE44F021EEDAF0A0EC6DF01F2B09EE9B
:10D7600046F021EEDDF0A0EC6DF01F2B09EE48F045
:10D7700021EEE0F0A0EC6DF01F2B09EE4AF021EE57
:10D78000E3F0A0EC6DF01F2B09EE4CF021EEE6F07B
:10D79000A0EC6DF01F2B09EE4EF021EEE9F0A0ECAD
:10D7A0006DF01F2B2CEC69F004D81E991E9B1E9D5A
:10D7B0001200030109EE60F0090E0417010EEB38A8
:10D7C000F60BE8BE8F0B041312C9E8FFE8B006D0D1
:10D7D000020EEBCF05F3030EEBCF06F309EE70F06C
:10D7E000090E0B17010EEB38F60BE8BE8F0B0B136F
:10D7F00012C9E8FFE8B006D0020EEBCF0CF3030E1F
:10D80000EBCF0DF309EE80F0090E1217010EEB3885
:10D81000F60BE8BE8F0B121312C9E8FFE8B006D072
:10D82000020EEBCF13F3030EEBCF14F3C2C0E8FFED
:10D83000E8BC3DD009EE90F0090E4417010EEB381C
:10D84000F60BE8BE8F0B441312C9E8FFE8B006D010
:10D85000020EEBCF45F3030EEBCF46F309EEA0F03B
:10D86000090E4B17010EEB38F60BE8BE8F0B4B136E
:10D8700012C9E8FFE8B006D0020EEBCF4CF3030E5E
:10D88000EBCF4DF309EEB0F0090E5217010EEB3855
:10D89000F60BE8BE8F0B521312C9E8FFE8B006D0B2
:10D8A000020EEBCF53F3030EEBCF54F30AD013EE7B
:10D8B00000F023EE40F0190EF36EE6CFDEFFF32EFC
:10D8C000FCD7010112001DEC65F0D8A4B1EC65F0A5
:10D8D000E8EF67F0020EEBAE39D0030EEB507F0B92
:10D8E0000F6E0F9E020EEB507F0B0E6E0F5E0FAE93
:10D8F00006D00F1E0F2A030EEB507F0B0E6E0F2A61
:10D900001F51240F030D11EE80F0F350E126E6CFF6
:10D910000BF0E6CF0CF0E6CF0DF0800E0C260DBE1E
:10D9200005D00D5001E106E30C6804D00D1C01E1A7
:10D9300001E20C6A0F500C02F4500E26000EDB5070
:10D940000E186AE0000E0EC0DBFF43D01E911F517F
:10D95000000FC6EC16F035150AE0010EDB68020E6A
:10D96000EB507F0BFF0FF36E000EF3CFDBFF1F5169
:10D97000040FC6EC16F035150EE0010EDB28F36E31
:10D9800005E0000EEB503F0BF36402D0F36A1E81FA
:10D99000010EF3CFDBFF1EA13FD0000EDB50AA0A21
:10D9A0003BE0000EDB28F36E030EEB507F0BF364BD
:10D9B0000DD0040EEBAE06D0AA0EF36E000EF3CF20
:10D9C000DBFF2AD0040EEB507F0BF36E000EF3CF7B
:10D9D000DBFF1AEE80F0000EDB507F0BE126E7CF75
:10D9E00003F021EE74F0D8901F35D92603BE06D07F
:10D9F000DE6AD8900334800FDD6E04D0DE6A0350F7
:10DA00007F0BDD6E056A000EEBBC0580EBBE058268
:10DA1000010EEB50E3EC90F0120009EEE0F012EE94
:10DA2000D0F034B1B9EC71F0349133BDA9EC71F0A0
:10DA3000339D09EEF0F012EED5F034B3B9EC71F08D
:10DA4000349333BFA9EC71F0339F1F6B34A507D01B
:10DA500009EEC0F012EEA0F0BFEC6DF034951F2B74
:10DA600034A707D009EEC5F012EEA4F0BFEC6DF0BC
:10DA700034971F2B34A907D009EECAF012EEA8F094
:10DA8000BFEC6DF034991F2B34AB07D009EECFF00B
:10DA900012EEACF0BFEC6DF0349B1F2B34AD07D011
:10DAA00009EED4F012EEB0F0BFEC6DF0349D1F2BF8
:10DAB00034AF07D009EED9F012EEB4F0BFEC6DF040
:10DAC000349F1F2B1F6B33A107D009EE60F012EEBD
:10DAD00000F0BCEC71F033911F2B33A307D009EE9B
:10DAE00070F012EE18F0BCEC71F033931F2B33A5DD
:10DAF00007D009EE80F012EE30F0BCEC71F03395F7
:10DB00001F2B33A707D009EE90F012EE48F0BCECC3
:10DB100071F033971F2B33A907D009EEA0F012EE56
:10DB200060F0BCEC71F033991F2B33AB07D009EEDA
:10DB3000B0F012EE78F0BCEC71F0339B1F2B1200AA
:10DB40001F51C6EC16F03A1519E1EECF03F0EDCFF8
:10DB500004F0DE500326DE500422DFBE06D0DF5084
:10DB600001E108E30368046805D0DF1C01E102E27B
:10DB7000036A046A1F5193EC1CF001011200000EAD
:10DB8000EBA605D01F51C6EC16F0311500E1000ED2
:10DB9000E66E040EEBCFE5FF1F51C4EC16F0311713
:10DBA000030EE36A030EF36AEB50D8A4F32A020EC5
:10DBB000F3CFE3FF85D0000EEBB008D021EE44F0A8
:10DBC000D8901F35D926DE6ADD6A34D1020EE126EF
:10DBD000E650E5100EE0030EEBCF0DF0800E97EC53
:10DBE00069F00350E6260450E52201E223D1E66AFB
:10DBF000E56AFE0EE1261E91000EEBA608D01F512D
:10DC0000C6EC16F0311503E0E668E56859D0000E61
:10DC1000EBA405D01EA754D032510F0B51E1020ED8
:10DC2000EBCF0BF01F51160F030D21EE80F0F350D8
:10DC3000010FD926DE500B26DFBE05D0DF5001E1F3
:10DC400006E30B6804D0DF1C01E101E20B6A000E61
:10DC5000EBA40ED00B500B0F0BE3020DA00EF32420
:10DC6000F66E3C0EF420F76EF86A010EF8220BD027
:10DC70000B50020DA00EF324F66E3A0EF420F76E50
:10DC8000F86A010EF8220900F550E6260900F55061
:10DC9000E52216E31E811F51030D2AEE4CF0F350CE
:10DCA000D926DE503313DE503413DE5035131F51A6
:10DCB000C6EC16F03113000EEBA602D0E668E5685C
:10DCC000E6CF0BF0E5CF0CF0000EEB38E8B682D0D3
:10DCD000E8B449D0E8B235D0E8B01DD00B340C34EC
:10DCE0000CBC7F0A7F0B020D200EF324F66E3E0E55
:10DCF000F420F76EF86A010EF8220900F5CF16F14C
:10DD00000900F5CF17F10CAE05D0161F171F162B03
:10DD1000D8B4172B68D0D8900B34166F0C347F0B07
:10DD2000176F0CAC06D0161F171F162BD8B4172B65
:10DD3000179F0CAE05D0161F171F162BD8B4172B24
:10DD400052D0E8B007D0000E0B5C166F800E0C5856
:10DD5000176F49D0000E0CBEFF0E166F800E0CBE62
:10DD60007F0E176F40D0E8B220D0E8B009D01EA1D6
:10DD700061D0DCEC59F00CC116F10CC117F133D0B5
:10DD80000C500CBE7F0A7F0B020D200EF324F66EA2
:10DD90003E0EF420F76EF86A010EF8220900F5CF66
:10DDA00016F10900F5CF17F11ED0E8B00DD00BC069
:10DDB00016F10CC017F10CAE06D0161F171F162B4C
:10DDC000D8B4172B179F0FD0D8900C30176F0B308B
:10DDD000166F09D0000E0CBEFF0E166F000E0CBEA3
:10DDE0007F0E176F00D0010EEBCF0BF01F51100FFD
:10DDF000030D11EE80F0F350010FE126E6500B26E3
:10DE0000E7BE05D0E75001E106E30B6804D0E71C4C
:10DE100001E101E20B6A0B5039EC69F002D01B6B97
:10DE20001C6B21EE44F0D8901F35D9261BC1DEFFB4
:10DE30001CC1DDFF1200000EEBAE0AD01EA703D0FE
:10DE400032510F0B05E0E6CF03F0E5CF04F094D09C
:10DE5000040EE3BC85D0E3BA73D0E3A0ACD0E3B842
:10DE600068D0E3B648D0E3B436D0E3B225D0020E92
:10DE7000E126E650E5100EE0020EEBCF0DF0800E2D
:10DE800097EC69F00350E6260450E52201E293D0B6
:10DE9000E66AE56AFE0EE126030EEB500D6E0D0EEE
:10DEA000EB5097EC69F0040EEBCF0BF073EC69F0DC
:10DEB00063E1000E21DA60D0050EEBCF0DF00D0E00
:10DEC000EB5097EC69F0FF0E0B6E73EC69F054E1C8
:10DED000010E12DA51D0060EEBCF0DF00E0EEB5004
:10DEE00097EC69F0070EEBCF0BF06EEC69F044E1B4
:10DEF000020E02DA41D0080EEBCF0DF00E0EEB5001
:10DF000097EC69F0090EEBCF0BF06EEC69F034E1A1
:10DF10001F51030D2AEE46F0F350D926DE5033137D
:10DF2000DE503413DE503513030EE6D9040EE3A899
:10DF300023D0090EEBCF04F0036A040EDDD91CD008
:10DF40000A0EEBCF0DF00F0EEB5097EC69F00B0EB5
:10DF5000EBCF0BF06EEC69F00FE1050ECDD90CD0D4
:10DF60000C0EEBCF0DF00F0EEB5097EC69F00B6A37
:10DF700084EC69F0060EC0D903C0E6FF04C0E5FFDB
:10DF8000D8900430176F0330166F0350041008E068
:10DF9000010EEB50800A04E0800A39EC69F002D0EF
:10DFA0001B6B1C6B21EE40F0D8901F35D9261BC18E
:10DFB000DEFF1CC1DDFF1200030EEB50800AD8B457
:10DFC0008CD1000EEB5017E0E8BE0FD021EE40F0F0
:10DFD000FF0FE834FE0B010FD926D890DD30286FF3
:10DFE000DF30276F28BD288F08D0E8303F0B286F1F
:10DFF000276B273302D0276B286B010EEB5017E0FD
:10E00000E8BE0FD021EE40F0FF0FE834FE0B010F09
:10E01000D926D890DD302A6FDF30296F2ABD2A8FAC
:10E0200008D0E8303F0B2A6F296B293302D0296BC7
:10E030002A6B020EEB500F0BC8EC16F00FD011D06C
:10E0400015D019D01FD025D035D03BD041D047D0E6
:10E0500051D05BD065D06FD072D08ED0166B176B5D
:10E0600092D027C116F128C117F18DD029C116F120
:10E070002AC117F188D027512925166F28512A2146
:10E08000176F81D02751295D166F28512A59176FB4
:10E090007AD0D8902735166F2835176FD890293544
:10E0A000186F2A35196F27EC1DF01CC116F11DC120
:10E0B00017F169D027512919166F28512A19176F9E
:10E0C00062D027512911166F28512A11176F5BD082
:10E0D00027512915166F28512A15176F54D02A5128
:10E0E000800A0B6E2851800A0B5C02E12751295DE2
:10E0F000B8E2BCD72A51800A0B6E2851800A0B5C0B
:10E1000002E12751295DB2E2ACD72A51800A0B6E99
:10E110002851800A0B5C02E12751295D2EE231D0A3
:10E120002A51800A0B6E2851800A0B5C02E12751AC
:10E13000295D27E222D02A5128191FE022D01F5141
:10E14000C6EC16F00B6E2AAF000E0C6E26510B14A7
:10E150000C1807E00B1C26170C5026130C5001E17D
:10E1600080D721EE40F0D8901F35100FD926DECF92
:10E1700016F1DECF17F107D071D716697F0E176F32
:10E1800002D0166B176B21EE40F0D8901F35100FA0
:10E19000D92616C1DEFF17C1DEFF16511711D8B4FC
:10E1A0009CD0030EEB5039EC69F01CC103F01F51F9
:10E1B0002FEC27F01B371C371D371BC12BF11CC15F
:10E1C0002CF11DC12DF11BC12EF11CC12FF11DC160
:10E1D00030F1020EEBAC08D02B1F2C1F2D1F2B2B68
:10E1E000D8B42C2BD8B42D2B020EEBAE08D02E1F9A
:10E1F0002F1F301F2E2BD8B42F2BD8B4302B060E48
:10E20000EB500AE021EE80F0FF0F030D21EE80F0CD
:10E21000F3507F0BD92662D8070EEB5008E0FF0FB2
:10E22000030D21EE80F0F3507F0BD9265ED8040E4B
:10E23000EBCF0BF00BA003D021EE80F04FD80BA258
:10E2400003D021EE83F04AD80BA403D021EE86F050
:10E2500045D80BA603D021EE92F040D80BA803D0EE
:10E2600021EE95F03BD80BAA03D021EE98F036D8DA
:10E270000BAC03D021EEA4F031D80BAE03D021EECD
:10E28000AAF02CD8050EEBCF0BF00BA003D021EE9B
:10E2900089F02BD80BA203D021EE8CF026D80BA44A
:10E2A00003D021EE8FF021D80BA603D021EE9BF0F6
:10E2B0001CD80BA803D021EE9EF017D80BAA03D0D0
:10E2C00021EEA1F012D80BAC03D021EEA7F00DD8AF
:10E2D0000BAE03D021EEADF008D812002B51DE2694
:10E2E0002C51DE222D51DE2212002E51DE262F511E
:10E2F000DE223051DE221200F36EF46E000EEB3897
:10E30000070BFF0FF31806E1000EEB50070B02E0BE
:10E31000FE0FF36EF450040A03E1F350040A01E027
:10E32000F32AF3B40AD0F3B204D0010EF3B0030E13
:10E330000BD0070EF3B00F0E07D0F3B204D01F0EB0
:10E34000F3B03F0E01D07F0EF36E040EF3CFE3FF68
:10E350001200010EF36E040EF3CFE3FF030EE36A27
:10E36000020EF36AEB50D8A4F32A020EF3CFE3FFB8
:10E370001200040EE38A1200010EE388E3B0E38684
:10E38000120EE36A070EF36AEB50D8A4F32A12C9FF
:10E39000E8FFE8A008D0010EF36ED6EC69F0050E98
:10E3A000DB6A060EDB6A110EF3CFE3FF12000101F8
:10E3B00010BA58D0108A3A6B800E0B6E01EE80F0C6
:10E3C000EE6A0B2EFDD71F6B09EE74F012EEA0F073
:10E3D000010E026F8CEC7DF01F2B09EE7BF012EE2C
:10E3E000A4F0010E026F8CEC7DF01F2BC2C0E8FF81
:10E3F000E8BC14D0060E1F6F09EEC4F012EEB8F0A0
:10E40000020E026F8CEC7DF01F2B09EECBF012EEAA
:10E41000BCF0020E026F8CEC7DF01F2B1F6B1E9F59
:10E4200001C2E8FF400BD8A41E8F09EE60F012EE87
:10E43000D0F001EC7FF01F2BC2C0E8FFE8BC0FD08A
:10E44000030E1F6F1E9F49C2E8FF400BD8A41E8F0A
:10E4500009EEB0F012EEDFF001EC7FF01F2B62EC62
:10E4600074F08DD0109A5BEC63F01F6B09EE60F0D6
:10E4700012EE00F022EEEAF0D2D81F2BC2C0E8FF65
:10E48000E8BC08D009EEB0F012EE48F022EEFDF044
:10E49000C6D81F2B356B1F6B09EE60F012EE00F033
:10E4A00026EE60F0C5EC63F01F2BC2C0E8FFE8BCAD
:10E4B0000BD0030E1F6F09EEB0F012EE48F026EEFF
:10E4C00078F0C5EC63F01F2B05EC74F01F6B09EEC0
:10E4D00060F012EE00F09CD81F2BC2C0E8FFE8BC31
:10E4E00008D0030E1F6F09EEB0F012EE48F090D87E
:10E4F0001F2B1F6B09EE54F011EEA4F023EE00F079
:10E500003DEC68F0C2C0E8FFE8BC09D01F2B09EE63
:10E510005AF011EEA7F023EE40F03DEC68F01F6BCF
:10E5200009EE40F01EEC69F01F2B09EE42F01EECE4
:10E5300069F01F2B09EE44F01EEC69F01F2B09EE69
:10E5400046F01EEC69F01F2B09EE48F01EEC69F056
:10E550001F2B09EE4AF01EEC69F01F2B09EE4CF060
:10E560001EEC69F01F2B09EE4EF01EEC69F01F2B1C
:10E570002CEC69F0C0EC72F01E991E9B1E9D1200DF
:10E58000030109EE60F012EE00F0090E0417010E0F
:10E59000EB38F60BE8BE8F0B041312C9E8FFE8B0A6
:10E5A0000BD0020EEBCF05F3030EEBCF06F3010EFB
:10E5B000E3AC02D0F00E0613C2C0E8FFE8BC1CD0EA
:10E5C00009EEB0F012EE48F0090E4417010EEB38D8
:10E5D000F60BE8BE8F0B441312C9E8FFE8B00BD06E
:10E5E000020EEBCF45F3030EEBCF46F3010EE3AC87
:10E5F00002D0F00E46130AD013EE00F023EE40F0E6
:10E60000190EF36EE6CFDEFFF32EFCD701011200E8
:10E610001DEC65F0D8A4B1EC65F0E8EF67F01EAD35
:10E6200003D0010EE39007D0100EEBB208D0020E1B
:10E63000DBA61200DB96010EE396E38812000C0EB7
:10E64000EBB012001E91020EDBA607D01EB905D05A
:10E650001F51C6EC16F0351513E0010EDB68020EF3
:10E66000DB500709F36E020EF3CFDBFF2C0EEB3805
:10E67000700BFF0FF36E000EF3CFDBFF010EE39E76
:10E680001EBB02D01EA902D0010EE380020EDB8663
:10E6900035AF0ED0010EDB28F36E05E02B0EEB50EC
:10E6A0003F0BF36402D0F36A1E81010EF3CFDBFF50
:10E6B0001EA1AAD0020EDB28070BF36E020EDB5060
:10E6C000F80BF310F46E020EF4CFDBFFF35006E00C
:10E6D000040AD8B48DD0050EF36496D0020EDB5038
:10E6E000F80BF36E020EF3CFDBFF000EDB280F0BEF
:10E6F000F36E06E02B0EEBAE03D0000EDB5002D023
:10E700002C0EEB38700BF312F350700BF46E2D0ED1
:10E71000EB500F0BF410F36403D0700EF414F36E8F
:10E72000000EF3CFDBFF2C0EEB50F80B04E0010ED4
:10E73000E3B461D069D0E1CFF3FFE2CFF4FF1AEE8A
:10E7400000F0000EDB50E126E7CF03F0800EE1265B
:10E75000E7CF04F0F3CFE1FFF4CFE2FF03500F0B5C
:10E760003C0F03B803D003BAF40F03D00C0F03BA65
:10E770000C0FF36E030EF3CFE3FF010EE3BE0DD0DB
:10E78000E39C04BEE38C1F51030DF334FE0BC6EC77
:10E7900016F03413D890E8343413010EE39AE3BE34
:10E7A000E38AE39E03BCE38E03AE15D0010EE3A023
:10E7B00012D0010EE398E3B40ED0E3861F51030D8F
:10E7C000F350C6EC16F036131F51030DF350020F31
:10E7D000C6EC16F034130450800F036E110E1F5355
:10E7E000D8A4220E056E2E0EEB50E3EC90F00CD068
:10E7F000010EE3BE09D0010EE396E3881F51030D1D
:10E80000F350C6EC16F03713120012EED0F037B109
:10E81000B2EC7FF0379136B1A8EC7FF0369112EE72
:10E82000DFF037B7B2EC7FF0379736B7A8EC7FF060
:10E8300036971F6B34A512D0349509EE74F0EFA211
:10E8400004D012EEA0F070EC7DF01F2B09EE7BF0EF
:10E85000EFA204D012EEA4F070EC7DF0C2C0E8FF8D
:10E86000E8BC16D0060E1F6F34AB12D0349B09EEF5
:10E87000C4F0EFA204D012EEB8F070EC7DF01F2BC4
:10E8800009EECBF0EFA204D012EEBCF070EC7DF0FC
:10E890001F6B33A107D012EE00F009EE60F0B5EC6B
:10E8A0007FF033911F2BC2C0E8FFE8BC0AD033A72A
:10E8B00007D012EE48F009EEB0F0B5EC7FF03397D8
:10E8C0001F2B120044A012002BBC4AD01D9610EE44
:10E8D00060F0080E0B6EE66A0B2EFDD7090170A3DF
:10E8E00021D08C51F80B1EE10201EA51E838C6EC48
:10E8F00016F00C6E10EE60F001C2E8FF010B07E1AC
:10E90000080E0B6E0CC0E6FF0B2EFCD70BD0EC51A3
:10E91000070B0B6E050E0B6005D0EA31070BE126E5
:10E920000CC0E7FF0901C0A319D0DC51F80B16E1B8
:10E9300010EE60F00201FD39070BE12649C2E8FF45
:10E94000010B02E1E7680AD0FF51070B0B6E050EC1
:10E950000B6004D0FD31C6EC16F0E7120101120085
:10E960001D8603013F0E04B1E8CFE9F004B1E8CF02
:10E97000EAF0C2C0E8FFE8BC07D03F0E44B1E8CFE0
:10E98000EDF044B1E8CFEEF00001E86BEB6BEC6B1F
:10E99000EF6B01011200010110BA17D0108A3A6B17
:10E9A000800E0B6E01EE80F0EE6A0B2EFDD75BEC55
:10E9B00063F022EEEAF0BFDA01013F0E35173AECC0
:10E9C00079F01E991E9B1E9D90D0109AD2EC76F085
:10E9D0001F6B12EE00F022EEEEF046DA1F2B12EE65
:10E9E00018F022EEF0F040DA1F2B12EE30F022EE9B
:10E9F000F2F03ADA1F2B12EE48F022EEF4F034DA9D
:10EA00001F2B12EE60F022EEF6F02EDA1F2B12EE24
:10EA100078F022EEF8F028DA1F2BC00E35171F6BA6
:10EA200012EE00F063D827D91F2B12EE18F05ED833
:10EA300022D91F2B12EE30F059D81DD91F2BC2C07E
:10EA4000E8FFE8BC0FD012EE48F050D814D91F2BC5
:10EA500012EE60F04BD80FD91F2B12EE78F046D88B
:10EA60000AD91F2B1F6B09EE54F011EEA4F023EE10
:10EA700000F03DEC68F0C2C0E8FFE8BC09D01F2BF5
:10EA800009EE5AF011EEA7F023EE40F03DEC68F0ED
:10EA90001F6B09EE40F01EEC69F01F2B09EE42F0EF
:10EAA0001EEC69F01F2B09EE44F01EEC69F01F2BE1
:10EAB00009EE46F01EEC69F01F2B09EE48F01EEC43
:10EAC00069F01F2B09EE4AF01EEC69F01F2B09EECE
:10EAD0004CF01EEC69F01F2B09EE4EF01EEC69F0B5
:10EAE0001F2B2CEC69F081EC75F01200030EE3048F
:10EAF0000F0B0A0D09EE60F0F350E926F450EA22FC
:10EB00001200030112EE00F0F1DF110EE3500BE1F1
:10EB1000120EE35008E1090E04170B0EE338F60B52
:10EB2000E8BE8F0B0413020EEBCF05F3030EEBCF01
:10EB300006F3010EE3AC02D0F00E061312EE18F04D
:10EB4000D5DF110EE3500BE1120EE35008E1090E80
:10EB50000B170B0EE338F60BE8BE8F0B0B13020EF0
:10EB6000EBCF0CF3030EEBCF0DF3010EE3AC02D0B1
:10EB7000F00E0D1312EE30F0B9DF110EE3500BE181
:10EB8000120EE35008E1090E12170B0EE338F60BD4
:10EB9000E8BE8F0B1213020EEBCF13F3030EEBCF75
:10EBA00014F3010EE3AC02D0F00E1413C2C0E8FF60
:10EBB000E8BC55D012EE48F099DF110EE3500BE19E
:10EBC000120EE35008E1090E44170B0EE338F60B62
:10EBD000E8BE8F0B4413020EEBCF45F3030EEBCFD1
:10EBE00046F3010EE3AC02D0F00E461312EE60F0D5
:10EBF0007DDF110EE3500BE1120EE35008E1090E28
:10EC00004B170B0EE338F60BE8BE8F0B4B13020EBF
:10EC1000EBCF4CF3030EEBCF4DF3010EE3AC02D080
:10EC2000F00E4D1312EE78F061DF110EE3500BE1A0
:10EC3000120EE35008E1090E52170B0EE338F60BE3
:10EC4000E8BE8F0B5213020EEBCF53F3030EEBCF44
:10EC500054F3010EE3AC02D0F00E54130AD013EEBD
:10EC600000F023EE40F0190EF36EE6CFDEFFF32E38
:10EC7000FCD7010112000B6A20EC65F0D8A420D863
:10EC8000010EE3A41AD0130EE126E650E51013E0BE
:10EC9000FD0EE35010E00D6E800E97EC69F003500E
:10ECA000E6260450E52201E206D0E66AE56AEE0EA9
:10ECB000E396E388E390ED0EE126CCEC76F01200CB
:10ECC000050EE3CF25F12551150FE8BE7F0E020D8D
:10ECD000200EF324F66E3D0EF420F76EF86A010E56
:10ECE000F8220900F5CF23F10900F5CF24F1186BC4
:10ECF000196B040EEB500B6E800A3FE0D8900B347A
:10ED00001827000E0BAEFF0E192319BF05D0180EE1
:10ED10002525E8BE7F0E04D0180E255DE8BE000E46
:10ED2000150FE8BE7F0E020D200EF324F66E3D0E89
:10ED3000F420F76EF86A010EF8220900F5CF03F00F
:10ED40000900F5CF04F019BF0CD02351035C166FF6
:10ED500024510458176F17AF0AD016697F0E176F2A
:10ED600006D00350235D166F04502459176F27EC0B
:10ED70001DF01B5123271C512423090E23C1E3FF3F
:10ED80000A0E24C1E3FF02EC6AF0D6EC69F023C15D
:10ED9000DEFF24C1DDFF12000B6A0C0EE3CF0CF086
:10EDA000F6EF67F01F6B33A106D012EE00F09EDE87
:10EDB0000EEC77F033911F2B33A306D012EE18F030
:10EDC00095DE0EEC77F033931F2B33A506D012EEB1
:10EDD00030F08CDE0EEC77F033951F2BC2C0E8FFCD
:10EDE000E8BC1BD033A706D012EE48F07FDE0EEC55
:10EDF00077F033971F2B33A906D012EE60F076DE42
:10EE00000EEC77F033991F2B33AB06D012EE78F06F
:10EE10006DDE0EEC77F0339B1F2B1200010EE388A2
:10EE2000E3B0E386F36AF46A12C9E8FFE8A00DD004
:10EE3000010EF36ED6EC69F0090EF56E040EF5CFF7
:10EE4000DBFF1F51C6EC16F03813110EF3CFE3FFB2
:10EE5000120EF4CFE3FF010EF36E130EF3CFE3FFB8
:10EE6000140EF4CFE3FF12001E911F51C6EC16F0F2
:10EE7000351507E0010EDB68F368000EF3CFDBFF0A
:10EE80001E81010EDB28F36E040EE3507F0BF3644A
:10EE900002D0F36A1E81010EF3CFDBFF1EA14AD020
:10EEA000000EDB50AA0A46E0110EE35043E1120EB9
:10EEB000E35040E1000EDB28F36E060EE350F364EE
:10EEC0000DD0070EE3AE06D0AA0EF36E000EF3CF00
:10EED000DBFF30D0070EE3507F0BF36E000EF3CF55
:10EEE000DBFF0D0EE3CFF6FF0E0EE3CFF7FF000EB4
:10EEF000DB50D890E8340C0FF626000EF722010EF6
:10EF0000F86E0900F5AE0FD0F59E150EE3307F0BBD
:10EF1000C00FF36EF524F3BE03D0E8BE7F0E02D01F
:10EF2000E8BE000EF56E050EF5CFE3FF09000B0EEF
:10EF3000F5CFE3FF12001EAD03D0020EDB98B3D075
:10EF400050C9E8FF400B05E1020EDBA61200DB967C
:10EF5000AAD01E91020EDBA604D01EB902D035AD98
:10EF600012D0010EDB68020EDB500709F36E020EB1
:10EF7000F3CFDBFF51C9E8FFE838700BFF0FF36EEA
:10EF8000000EF3CFDBFF1EBB02D01EA902D0020E83
:10EF9000DB88020EDB8635AF0ED0010EDB28F36E68
:10EFA00005E050C9E8FF3F0BF36402D0F36A1E810D
:10EFB000010EF3CFDBFF1EA179D0020EDB28070B79
:10EFC000F36E020EDB50F80BF310F46E020EF4CF6A
:10EFD000DBFFF35006E0040AD8B465D0050EF364F5
:10EFE00065D0020EDB50F80BF36E020EF3CFDBFFA1
:10EFF000000EDB280F0BF36E07E050C9E8FFE8AE08
:10F0000003D0000EDB5003D051C9E8FFE838700B85
:10F01000F312F350700BF46E53C9E8FF0F0BF410AA
:10F02000F36403D0700EF414F36E000EF3CFDBFF25
:10F03000020EDBA804D051C9E8FFF80B01E033D081
:10F04000010E0B6E0BC000F102010AEE00F0EA3572
:10F05000E00BE9260B04D890E834E926000EEAB765
:10F06000020EE926EA51C6EC16F0F36E0101EE1429
:10F0700006E1ED50F31401E110D0046807D0ED5023
:10F08000F31402E1046A02D0002B046AEE50EF1080
:10F09000F36EF31402E057EC78F00B2A0B2A100EF3
:10F0A0000B64D0D703D0006B12EC79F01200010191
:10F0B000D7D8000EDB380F0B026F0001600EC2BD07
:10F0C000300E0101021312EE00F0016B030EE3504B
:10F0D000006317D002510F0B10E0FF0F04E0FF0F89
:10F0E00006E0FF0F08D0030E01610BD006D0020E20
:10F0F000016507D002D0016304D00151A9EC59F099
:10F100000AD0180EE126012B02390F0BFF0F016503
:10F11000DDD7E4EC58F0030E00C1E3FF010EDBCFB6
:10F12000F3FF140EF360F36AF350020D600EF32444
:10F13000F66E3F0EF420F76EF86A010EF8220D0EFF
:10F140000900F5CFE3FFF5CFF3FF0E0E0900F5CF71
:10F15000E3FFF5CFF4FFF350040FF66EF76AF450B7
:10F16000F72209000F0EF5CFE3FF0900050EF5CFDA
:10F17000E3FF0900F55011E0050EDB30E8303F0BEE
:10F18000E00FF36EF524F3BE03D0E8BE7F0E05D08A
:10F19000E8BE000EFF0BD8B4010FF56E100EF5CFD0
:10F1A000E3FF09000B0EF5CFE3FF09000C0EF5CFCE
:10F1B000E3FF0900060EDB30E8303F0BE00FF36E93
:10F1C000F524F3BE03D0E8BE7F0E02D0E8BE000EE9
:10F1D000F56E040EF5CFE3FF0900060EF5CFE3FF51
:10F1E0000900070EF5CFE3FF070EDBCFF5FF150E85
:10F1F000F5CFE3FF010EE39C04BCE38C010EE3803A
:10F200000151C6EC16F033130151020FC6EC16F093
:10F2100034130151C6EC16F035130151C6EC16F04B
:10F2200036131200010112EE00F0016B005104E0F0
:10F23000030EE35000630DD0C3EC59F0100EE35001
:10F2400008E1010EE390E396E3880151C6EC16F065
:10F250003713180EE126012B050E0165E7D71200C2
:10F2600000050F0B29EE60F00A0DF350D926F4507B
:10F27000DA22120044A012002BBC2DD01D9610EEF5
:10F2800060F0080E0B6EE66A0B2EFDD7090150AD3B
:10F2900020D05151F80B1DE10201EA51E838C6ECCB
:10F2A00016F00C6E10EE60F0EC51100B07E1080E3A
:10F2B0000B6E0CC0E6FF0B2EFCD70BD0EC51070BEE
:10F2C0000B6E050E0B6005D0EA31070BE1260CC072
:10F2D000E7FF01011200D4EF7FF0010110BAFBD06B
:10F2E000108A3A6B800E0B6E01EE80F0EE6A0B2EE8
:10F2F000FDD71F6B12EE00F0BFD9110EEBCF02F15C
:10F30000140EE926000EEA2212EEA0F08CEC7DF03D
:10F310001F2B12EE00F0B0D9110EEBCF02F11B0E35
:10F32000E926000EEA2212EEA4F08CEC7DF01F2BF1
:10F3300012EE18F0A1D9110EEBCF02F1140EE9264E
:10F34000000EEA2212EEA8F08CEC7DF01F2B12EEDC
:10F3500018F092D9110EEBCF02F11B0EE926000E28
:10F36000EA2212EEACF08CEC7DF01F2B12EE30F0A6
:10F3700083D9110EEBCF02F1140EE926000EEA221A
:10F3800012EEB0F08CEC7DF01F2B12EE30F074D941
:10F39000110EEBCF02F11B0EE926000EEA2212EE4F
:10F3A000B4F08CEC7DF01F2BC2C0E8FFE8BC5AD053
:10F3B00012EE48F061D9110EEBCF02F1140EE926DE
:10F3C000000EEA2212EEB8F08CEC7DF01F2B12EE4C
:10F3D00048F052D9110EEBCF02F11B0EE926000EB8
:10F3E000EA2212EEBCF08CEC7DF01F2B12EE60F0E6
:10F3F00043D9110EEBCF02F1140EE926000EEA22DA
:10F4000012EEC0F08CEC7DF01F2B12EE60F034D9C0
:10F41000110EEBCF02F11B0EE926000EEA2212EECE
:10F42000C4F08CEC7DF01F2B12EE78F025D9110E74
:10F43000EBCF02F1140EE926000EEA2212EEC8F01C
:10F440008CEC7DF01F2B12EE78F016D9110EEBCF5D
:10F4500002F11B0EE926000EEA2212EECCF08CEC33
:10F460007DF01F2B1E9F1F6B12EE00F005D912EED0
:10F47000D0F001EC7FF01F2B12EE18F0FDD812EE49
:10F48000D5F001EC7FF01F2B12EE30F0F5D812EE24
:10F49000DAF001EC7FF01F2BC2C0E8FFE8BC18D007
:10F4A00012EE48F0E9D812EEDFF001EC7FF01F2BEE
:10F4B00012EE60F0E1D812EEE4F001EC7FF01F2BC9
:10F4C00012EE78F0D9D812EEE9F001EC7FF01F2BA4
:10F4D000D0EC7FF0D0D0109A5BEC63F01F6B09EE9C
:10F4E00060F022EEEEF07CD91F2B09EE90F022EEB8
:10F4F000F0F076D91F2B09EEC0F022EEF2F070D9B1
:10F500001F2B09EEF0F022EEF4F06AD91F2B0AEE61
:10F5100020F022EEF6F064D91F2B0AEE50F022EE16
:10F52000F8F05ED91F2B356B1F6B206B26EE60F059
:10F53000B8D8ACD803E1A0D8C5EC63F01F2B26EEF9
:10F5400078F0AFD8A3D803E197D8C5EC63F01F2BB0
:10F5500026EE90F0A6D89AD803E18ED8C5EC63F0D9
:10F560001F2BC2C0E8FFE8BC1BD026EEA8F099D83C
:10F570008DD803E181D8C5EC63F01F2B26EEC0F0D7
:10F5800090D884D803E178D8C5EC63F01F2B26EE21
:10F59000D8F087D87BD803E16FD8C5EC63F01F2B78
:10F5A0003FEC7CF01F6B12EE00F066D812D91F2BD7
:10F5B00012EE18F061D80DD91F2B12EE30F05CD886
:10F5C00008D91F2BC2C0E8FFE8BC0FD012EE48F0EC
:10F5D00053D8FFD81F2B12EE60F04ED8FAD81F2B4D
:10F5E00012EE78F049D8F5D81F2B1F6B09EE54F0B6
:10F5F00011EEA4F023EE00F03DEC68F0C2C0E8FF8D
:10F60000E8BC09D01F2B09EE5AF011EEA7F023EE4B
:10F6100040F03DEC68F01F6B09EE40F01EEC69F025
:10F620001F2B09EE42F01EEC69F01F2B09EE44F08F
:10F630001EEC69F01F2B09EE46F01EEC69F01F2B43
:10F6400009EE48F01EEC69F01F2B09EE4AF01EECA3
:10F6500069F01F2B09EE4CF01EEC69F01F2B09EE30
:10F660004EF01EEC69F01F2B2CEC69F059EC7BF08E
:10F670001E991E9B1E9D1200000EE350300D09EED8
:10F6800060F0F350E926F450EA221200000EE35035
:10F69000C6EC16F0F36E201503E1F3502013000BB7
:10F6A0001200050EDB50180D12EE00F0F350E126AB
:10F6B0001200030112EE00F0DFDF090E0417010E45
:10F6C000EB38F60BE8BE8F0B041312C9E8FFE8B065
:10F6D00006D0020EEBCF05F3030EEBCF06F312EECE
:10F6E00018F0CADF090E0B17010EEB38F60BE8BE57
:10F6F0008F0B0B1312C9E8FFE8B006D0020EEBCF58
:10F700000CF3030EEBCF0DF312EE30F0B5DF090E64
:10F710001217010EEB38F60BE8BE8F0B121312C94D
:10F72000E8FFE8B006D0020EEBCF13F3030EEBCFE9
:10F7300014F3C2C0E8FFE8BC40D012EE48F09CDFF2
:10F74000090E4417010EEB38F60BE8BE8F0B44137D
:10F7500012C9E8FFE8B006D0020EEBCF45F3030E66
:10F76000EBCF46F312EE60F087DF090E4B17010E68
:10F77000EB38F60BE8BE8F0B4B1312C9E8FFE8B06D
:10F7800006D0020EEBCF4CF3030EEBCF4DF312EE8F
:10F7900078F072DF090E5217010EEB38F60BE8BE57
:10F7A0008F0B521312C9E8FFE8B006D0020EEBCF60
:10F7B00053F3030EEBCF54F30AD013EE00F023EE15
:10F7C00040F0190EF36EE6CFDEFFF32EFCD70101F9
:10F7D00012001DEC65F0D8A4B1EC65F0E8EF67F01D
:10F7E0001E911F51C6EC16F035150BE0010EDB68BB
:10F7F0002D0EEB507F0BFF0FF36E000EF3CFDBFFF0
:10F800001E8135AF0DD0010EDB28F36E2B0EEB50B1
:10F810003F0BF36402D0F36A1E81010EF3CFDBFFCE
:10F820001EA12CD0000EDB50AA0A28E0000EDB2817
:10F83000F36E2E0EEB507F0BF3640DD02F0EEBAE5C
:10F8400006D0AA0EF36E000EF3CFDBFF17D02F0EFB
:10F85000EB507F0BF36E000EF3CFDBFF1AEE80F060
:10F86000000EDB507F0BE126E7CF03F01F39F00BD2
:10F870000309056E2C0EEB50E3EC90F0120012EE33
:10F88000D0F037B1B2EC7FF0379136B1A8EC7FF011
:10F89000369112EED5F037B3B2EC7FF0379336B332
:10F8A000A8EC7FF0369312EEDAF037B5B2EC7FF0C9
:10F8B000379536B5A8EC7FF0369512EEDFF037B706
:10F8C000B2EC7FF0379736B7A8EC7FF0369712EEA0
:10F8D000E4F037B9B2EC7FF0379936B9A8EC7FF095
:10F8E000369912EEE9F037BBB2EC7FF0379B36BBAE
:10F8F000A8EC7FF0369B1F6B34A51BD0349512EE1D
:10F9000000F0BADE140EEBA207D0E926000EEA22C0
:10F9100012EEA0F070EC7DF012EE00F0ADDE1B0EEA
:10F92000EBA207D0E926000EEA2212EEA4F070EC5A
:10F930007DF01F2B34A71BD0349712EE18F09CDEFD
:10F94000140EEBA207D0E926000EEA2212EEA8F070
:10F9500070EC7DF012EE18F08FDE1B0EEBA207D0DC
:10F96000E926000EEA2212EEACF070EC7DF01F2BBF
:10F9700034A91BD0349912EE30F07EDE140EEBA2C7
:10F9800007D0E926000EEA2212EEB0F070EC7DF00E
:10F9900012EE30F071DE1B0EEBA207D0E926000E4E
:10F9A000EA2212EEB4F070EC7DF01F2BC2C0E8FF2B
:10F9B000E8BC5AD034AB1BD0349B12EE48F05CDE6E
:10F9C000140EEBA207D0E926000EEA2212EEB8F0E0
:10F9D00070EC7DF012EE48F04FDE1B0EEBA207D06C
:10F9E000E926000EEA2212EEBCF070EC7DF01F2B2F
:10F9F00034AD1BD0349D12EE60F03EDE140EEBA24F
:10FA000007D0E926000EEA2212EEC0F070EC7DF07D
:10FA100012EE60F031DE1B0EEBA207D0E926000EDD
:10FA2000EA2212EEC4F070EC7DF01F2B34AF1BD035
:10FA3000349F12EE78F020DE140EEBA207D0E926F8
:10FA4000000EEA2212EEC8F070EC7DF012EE78F0B3
:10FA500013DE1B0EEBA207D0E926000EEA2212EEFF
:10FA6000CCF070EC7DF01F2B1F6B33A106D012EE93
:10FA700000F002DEB5EC7FF033911F2B33A306D0EC
:10FA800012EE18F0F9DDB5EC7FF033931F2B33A5A0
:10FA900006D012EE30F0F0DDB5EC7FF033951F2B81
:10FAA000C2C0E8FFE8BC1BD033A706D012EE48F076
:10FAB000E3DDB5EC7FF033971F2B33A906D012EEB0
:10FAC00060F0DADDB5EC7FF033991F2B33AB06D055
:10FAD00012EE78F0D1DDB5EC7FF0339B1F2B1200D6
:10FAE000000EEBA605D01F51C6EC16F0311500E153
:10FAF000000EE66E040EEBCFE5FF1F51C4EC16F0CE
:10FB00003117030EE36A030EF36AEB50D8A4F32A0D
:10FB1000020EF3CFE3FF5CD0000EEBA05FD1020E2C
:10FB2000E126E650E5100EE0030EEBCF0DF0800E5F
:10FB300097EC69F00350E6260450E52201E24ED12D
:10FB4000E66AE56AFE0EE1261E91000EEBA608D0DD
:10FB50001F51C6EC16F0311503E0E668E56838D0B1
:10FB6000000EEBA405D01EA733D032510F0B30E1AD
:10FB7000020EEBCF0BF0000EEBA40ED00B500B0FD0
:10FB80000BE3020DA00EF324F66E3C0EF420F76E8C
:10FB9000F86A010EF8220BD00B50020DA00EF324D0
:10FBA000F66E3A0EF420F76EF86A010EF82209009C
:10FBB000F550E6260900F550E5220AE31E811F51A3
:10FBC000C6EC16F03113000EEBA602D0E668E5682D
:10FBD000E6CF0BF0E5CF0CF0000EEB38E8B682D0A4
:10FBE000E8B449D0E8B235D0E8B01DD00B340C34BD
:10FBF0000CBC7F0A7F0B020D200EF324F66E3E0E26
:10FC0000F420F76EF86A010EF8220900F5CF16F11C
:10FC10000900F5CF17F10CAE05D0161F171F162BD4
:10FC2000D8B4172B68D0D8900B34166F0C347F0BD8
:10FC3000176F0CAC06D0161F171F162BD8B4172B36
:10FC4000179F0CAE05D0161F171F162BD8B4172BF5
:10FC500052D0E8B007D0000E0B5C166F800E0C5827
:10FC6000176F49D0000E0CBEFF0E166F800E0CBE33
:10FC70007F0E176F40D0E8B220D0E8B009D01EA1A7
:10FC8000ADD0DCEC59F00CC116F10CC117F133D03A
:10FC90000C500CBE7F0A7F0B020D200EF324F66E73
:10FCA0003E0EF420F76EF86A010EF8220900F5CF37
:10FCB00016F10900F5CF17F11ED0E8B00DD00BC03A
:10FCC00016F10CC017F10CAE06D0161F171F162B1D
:10FCD000D8B4172B179F0FD0D8900C30176F0B305C
:10FCE000166F09D0000E0CBEFF0E166F000E0CBE74
:10FCF0007F0E176F00D0010EEB50800A1CE0800AC7
:10FD000039EC69F021EE80F0D8901F31030DF350EB
:10FD1000D926D8901DBFD8801D331C331B33D890F3
:10FD20001DBFD8801D331C331B331B51DE261C51D5
:10FD3000DE221D51DE22050EEB50800A10E0800A03
:10FD400039EC69F021EE92F0D8901F31030DF35099
:10FD5000D9261B51DE261C51DE221D51DE22060E45
:10FD6000EB50800A3BE010C9E8FF030B030A0BE0ED
:10FD7000060EEB5039EC69F0060E1F6102D02FD849
:10FD80002DD036D82BD022EE00F01F317F0BF56E30
:10FD9000180DF350000FD926DF5026EE60F0180D35
:10FDA000F350050FD926DF50F56218D0060EEB5040
:10FDB00039EC69F002510F0B0BE0FF0F0CE0FF0F65
:10FDC0000CE0FF0F08E0FF0F06E0FF0F04E005D096
:10FDD00006D80ED803D003D801D00AD8120021EEDD
:10FDE000A4F01B51DE261C51DE221D51DE22120022
:10FDF00021EEA7F01B51DE261C51DE221D51DE2212
:10FE00001200220EEBAE0AD01EA703D032510F0B08
:10FE100005E0E6CF03F0E5CF04F04CD0040EE3BCE0
:10FE200096D0E3BA35D0E3A092D0E3B82CD0E3B6B5
:10FE300014D0260EEB500D6E220EEBA803D02A0E26
:10FE4000EB5001D0800E97EC69F0FF0E0B6E73EC57
:10FE500069F030E1040EE3862DD0270E1EBF300E70
:10FE6000EBCF0DF0220EEBAA03D02A0EEB5001D0FF
:10FE7000800E97EC69F0280EEBCF0BF06EEC69F07A
:10FE800019E1040EE388280EEBCF04F0036A12D0C8
:10FE9000290EEBCF0DF0220EEBAC03D02A0EEB5067
:10FEA00001D0800E97EC69F00B6A84EC69F002E1F6
:10FEB000040EE38C03C0E6FF04C0E5FF035004100A
:10FEC00046E0D8900430176F0330166F230EEB50C6
:10FED000800A0FE0800A4CEC69F021EE80F01F519F
:10FEE000030DF350D9261B51DE261C51DE221D5175
:10FEF000DE22240EEB50800A0FE0800A4CEC69F001
:10FF000021EE92F01F51030DF350D9261B51DE262E
:10FF10001C51DE221D51DE22250EEB50800A17E017
:10FF2000800A4CEC69F0030E1F6109D021EEA4F0A9
:10FF30001B51DE261C51DE221D51DE2208D021EE8F
:10FF4000A7F01B51DE261C51DE221D51DE221200BD
:10FF5000010EF36E040EF3CFE3FF030EE36A020E0D
:10FF6000E36A1200040EE38A1200010EE388E3B094
:10FF7000E386120EE36A070EF36AEB50D8A4F32A65
:10FF800012C9E8FFE8A008D0010EF36ED6EC69F0C4
:10FF9000050EDB6A060EDB6A110EF3CFE3FF1200DB
:10FFA00044A012002BAC12001D8603013F0E04B1C9
:10FFB000E8CFE9F00BB1E8CFEAF012B1E8CFEBF00F
:10FFC0003F0E44B1E8CFECF04BB1E8CFEDF052B1C9
:10FFD000E8CFEEF00001E86BEF6B01011200035077
:10FFE0000F0BE8CF03F104C004F105C005F1F29E48
:10FFF00002D8F28E12000338070BC8EC16F018D0A6
:020000040001F9
:1000000006D0A7D047D09DD0A1D01FD012000101AB
:100010000551D8B40DD010C9E8FF030BCAEC16F097
:10002000F3EF81F056EF83F0E8EF84F08EEF85F088
:1000300010C9E8FF030BCAEC16F055EF82F0BFEFD2
:1000400083F031EF85F0DBEF85F00101D89004BD3E
:10005000D8800535046F006B06EE60F0000EEB50A3
:1000600003630BD045C006F0010E456E04C103F0DA
:10007000060E37EC8CF006C045F010C9E8FF030B04
:10008000CAEC16F0B6EF82F009EF84F058EF85F075
:100090000EEF86F00101045110E1080E0561120017
:1000A00005C014F0125002E159EF3FF003516063B4
:1000B00012003BEC54F0CBEF1BF0620E046306D051
:1000C00013EEA0F0035105C1E3FF1200630E0463B9
:1000D00006D013EEB0F0035105C1E3FF1200260E67
:1000E000046306D013EEC0F0035105C1E3FF120014
:1000F000006B06EE60F0000EEB50036315D00405B4
:1001000006E1D8900535036E000E37EF8CF00F0E28
:1001100004650AD0140E046107D0D8900535036E2B
:100120000451F10F37EF8CF010C9E8FF030BCAEC54
:1001300016F0B7EF82F01BEF84F05AEF85F02BEF4B
:1001400086F0125002E13DEF3FF0120005C104F1CC
:1001500000D00101006B06EE60F0000EEB5003636F
:1001600006D0D8900435036E070E37EC8CF01200E1
:10017000F36AF350DB5008E00419D8B416D0F32A20
:10018000080EF362F6D702D0FF0EDB2A060EF36EDE
:10019000F350DBCFF4FFF328F4CFDBFFF306F328B3
:1001A000F7E104C1DFFF000B1200FF091200F36A40
:1001B000F350DB50041905E0F32A080EF362F8D778
:1001C00010D0F328DBCFF4FFF350F4CFDBFFF32A9A
:1001D000080EF362F6D7070EDB6AFF0EDB06000B94
:1001E0001200FF091200F36AF350DB50041906E015
:1001F000F32A080EF362F8D7FF091200F350DB8EE2
:10020000000B1200F36AF350DB507F0B08E0041977
:100210007F0B0CE0F32A080EF362F5D707D0F350FA
:1002200004C1DBFFFF0EDB2A000B1200FF091200E6
:10023000F36AF350DB507F0B0BE004197F0B22E0D5
:100240000419045D05E3F32A080EF362F2D71200E5
:10025000FF0EDB2ADB50090AFF0ED8B4DB06F35091
:10026000070A0DE0060EF46EF450DBCFF5FF010F28
:10027000F5CFDBFFF350F41802E0F406F5D7F350A6
:1002800004C1DBFF1200000EF36EDB5009E0F350F7
:10029000DB5006E0800B06E0F32A070EF364F7D785
:1002A000FF091200000B1200000EF36EDB5019E084
:1002B000F350DB5018E0800B0FE0F328DBCFF4FFA6
:1002C000F350F4CFDBFFF32A080EF362F6D7070EE4
:1002D000DB6AFF0EDB06E8D7F32A070EF364E8D7E4
:1002E00002D0FF091200000B1200FF0EDB6AF36A56
:1002F000F350DB6AF32A070EF364FAD71200F5BA5B
:1003000002D0D2DF01D0BFDF03E0060EEB84EDDFC9
:10031000F5B802D077DF01D08BDF010EE380050E48
:1003200004C1E3FF12005FDF06BA04D0ACDF02E0D5
:10033000010EE3901200F36AF350DB50041905E05C
:10034000F32A040EF362F8D70ED0F328DBCFF4FFC4
:10035000F350F4CFDBFFF32A040EF362F6D7030E5B
:10036000DB6A000B1200FF091200F36AF350DB5046
:100370007F0B0BE004197F0B1BE00419045D05E300
:10038000F32A040EF362F2D71200F350030A0DE0D1
:10039000020EF46EF450DBCFF5FF010FF5CFDBFF5B
:1003A000F350F41802E0F406F5D7F35004C1DBFF74
:1003B00012000101000EEB50036313D0010EEBCFCE
:1003C000F3FF020EEBCFF4FFF350F41008E0F3500C
:1003D000046101D006D0F450046501D002D0000BB6
:1003E0001200FF0912000101006B06EE60F0D9EC6B
:1003F00081F05AE1C6C0E8FF070B1CE012601AD07A
:10040000E838026FE4EC58F010EEFCF0015104C142
:10041000E3FF0151126248D006016F6B876B9F6B3F
:10042000B76BCF6BE76B706B886BA06BB86BD06BE7
:10043000E86B01010451C40F636F000E63BFFF0E30
:10044000626FD8900535036E050E37EC8CF050C9FD
:1004500006F106EE60F012EE00F0016B29EE6CF092
:100460000151100DF350D926DFCF06F026EE6BF0C8
:100470000151180DF350D926B5EC81F0050ED9269F
:1004800006B008D0B8EC80F006B302D006A1FBD8C5
:10049000A8D802D07FEC81F0180EE926180EE126CC
:1004A000012B050E0165DAD712000101006B06EE83
:1004B00060F0D9EC81F059E1C6C0E8FF070B13E00A
:1004C000126011D010EEFCF0016BE750041905E04A
:1004D000E650012B01A5F9D748D0E76AC3EC59F0E3
:1004E0000151126242D050C906F106EE60F012EEE0
:1004F00000F0016B29EE6CF00151100DF350D9267C
:10050000DFCF06F026EE6BF00151180DF350D9261F
:1005100007A19BEC81F0050ED926DFCF08F007A1DB
:1005200012D006B00ED0F36AF46AF350DB5202E048
:10053000DBAEF42AF32A070EF364F7D7020EF46059
:1005400002D051DE0AD006B006D031DE085081D884
:10055000E8B047D802D093EC81F0180EE926180EC7
:10056000E126012B050E0165C5D71200120001011D
:1005700060C6E8FF036334D0060E046304D0056A46
:10058000AEEC90F02DD0400E04632AD005BD26D0ED
:10059000076B06EE60F012EE00F0016BEACFDAFFB7
:1005A0000E0EE924D96EDD6ADD6ADD6ADF6A050EAA
:1005B000D9267ADE050EE350046F100EEB500419B5
:1005C00004E0045146D8E8B00CD8180EE926180EFD
:1005D000E126012B050E0165E1D702D0010E076F60
:1005E0001200100EEBCFF3FFF39E06B303D0030E01
:1005F000F3CFE3FF050EF3CFE3FF06A505D0010E11
:10060000E39A0F0EEB0402E0010EE38A06A103D089
:10061000010EE3B01DD034D806A109D8100EEBCFDF
:10062000F3FF0451F36214D0110EEB5011E106B345
:100630000CD00151C6EC16F0C009F36E40CAE8FFB9
:10064000F314331341CAE8FF341342CAE8FF3513E9
:100650001200F56EF550046312D006B101D013D824
:100660000F0EEB50D8A4010C0ED843CAE8FFC00B04
:10067000331344CAE8FF341345CAE8FF3513000CAE
:10068000010EE3801200010EE3A00FD0010EE390F3
:10069000E3960151C6EC16F0F36E0A014315010111
:1006A000010ED8A4E388F31C33171200006B06EE8A
:1006B00060F0D9EC81F05CE145C006F00051C6EC79
:1006C00016F0456ED8900535036E050E37EC8CF0AC
:1006D00006C045F03ED90C0EDBCF06F0100EDBCF86
:1006E00006F12DD906B320D006B00FD026EE6BF060
:1006F0000051180DF350D926B5EC81F0050ED9261E
:1007000037DD06A108D9B7D833D0050E01C1EBFFFC
:10071000000E00C1E3FF26EE70F00051180DF350FB
:10072000D9267FEC81F024D026EE6BF00051180D15
:10073000F350D926B5EC81F0050ED92619DD10B895
:100740000CD001C2E8FFE8B002D0010E351349C257
:10075000E8FFE8B002D0020E351304D9020170C9D7
:10076000E8FFE8B20181C0C9E8FFE8B249810101B0
:10077000180EE926002B010E00659BD7120001011F
:10078000006B016B06EE60F0D9EC81F03BE1E1D843
:100790000C0EDBCF06F0100EDBCF06F126EE6BF071
:1007A0000051180DF350D9269BEC81F0C8D8050EE6
:1007B000D926DFCF08F006B30BD006B006D0F7DCA1
:1007C000085083D8E8B057D81DD093EC81F01AD0E8
:1007D000EEDCBFD80F0EEB50D8A4C4D810B812D09E
:1007E0008CC9E8FFF80B0EE0DCC9E8FFF80B0AE063
:1007F000020170C9E8FFE8B20191C0C9E8FFE8B2A0
:1008000049910101180EE926002B010E0065BCD7A5
:10081000120006EE78F0000EEB5003630BD045C0DB
:1008200006F0020E456E04C103F0060E37EC8CF0A4
:1008300006C045F012000101006B06EE60F0000EEC
:10084000EB5003630BD0060E046305D00039056E30
:10085000AEEC90F003D0400E046300D060C6F3FF0E
:1008600078C6E8FFF31806E0180EE926002B010E03
:100870000065E5D71200100EEBCFF3FF030EF3CFA8
:10088000E3FF050EF3CFE3FF06A505D0010EE39AC3
:100890000F0EEB0402E0010EE38A06A103D0010E65
:1008A000E3B001D01FD806A109D8100EEBCFF3FF9B
:1008B0000451F36203D0110EEB5000E1050E01C1AB
:1008C000EBFF000E00C1E3FF1200F56EF55004636C
:1008D00008D006B101D01FD80F0EEB50D8A4010CE0
:1008E0001AD8000C010EE3800151C6EC16F0331348
:1008F0000151020FC6EC16F034130151010ED8A4B9
:10090000020E35130151C6EC16F03613010EE39CAE
:1009100005BDE38C1200010EE3A010D0050EE350DC
:1009200004630CD0010EE390E3960151C6EC16F07F
:10093000010EE3880151C6EC16F037131200005186
:10094000D8A4030E016F12EE00F0D8A412EE48F006
:10095000120029EE60F00051500DF350D926F450EA
:10096000DA221200100EEBCFF3FF030EEB50C00F94
:10097000E8BE05D0F326F3AE07D0F40FFBD7F3267D
:10098000F3AE02D00C0EFBD7050EF3CFE3FF0B0E38
:10099000F36403D0F40EF326FAD7080EF360F36E77
:1009A00000B10BD0F3CF8CF7F3CF8CF95DEC3EF0B8
:1009B0005F18D8B4F3CF8CFB1200F3CFDCF7F3CF82
:1009C000DCF95DEC3EF05F18D8B4F3CFDCFB12002D
:1009D00006EE60F0D9EC81F043E126EE70F0B8EC61
:1009E00080F0045174D8006F50C9E8FF400B1EE13D
:1009F000110E006135D0D8900535036E050E37EC29
:100A00008CF005C104F0D8900436036A0005E8387C
:100A1000F00B0309056E30EC79F0080EDB509FEC0B
:100A200090F005C104F057EC78F01AD0D890053555
:100A3000036E050E37EC8CF010B806D0ECC2E8FF60
:100A4000E8B802D0400E35130005F36E0B0EF364C8
:100A500002D0F40EF326F35052D80201EC890101C2
:100A60001200010106EE60F0D9EC81F020E126EEE3
:100A700070F0D7EC80F050C9E8FF400B09E1045159
:100A800026D8006F110E006112D012EC79F00FD051
:100A90000F0EEB5003E01BD8FF0F31D810B807D072
:100AA00051C9E8FFF80B03E00201EC9901011200C3
:100AB00001011200010160C6E8FF036307D0060EC2
:100AC000046304D0056AAEEC90F000D01200F36E1F
:100AD000030EEB50C00FE8BE05D0F326F3AE07D0EF
:100AE000F40FFBD7F326F3AE02D00C0EFBD7170E94
:100AF000F36403D0E80EF326FAD7F3281200F36E5E
:100B0000080EF360F36EF3CF51F7F3CF51F95DECBC
:100B10003EF05F18D8B4F3CF51FB1200006B06EE25
:100B200060F0D9EC81F040E1005106E1D890053544
:100B3000036E050E37EC8CF005C104F0D890043636
:100B4000036A0039700B0309056E54D9120EDB508D
:100B50009FEC90F00C0EDBCF06F0100EDBCF06F111
:100B600006B012D026EE6BF00051180DF350D926C6
:100B7000B5EC81F0050ED926B8EC80F006B302D0B2
:100B800006A1D5D882D810D0BAEC86F0050E01C1E6
:100B9000EBFF000E00C1E3FF26EE70F00051180DD0
:100BA000F350D9267FEC81F0180EE926002B050EB4
:100BB0000065B7D712000101006B06EE60F0D9ECBA
:100BC00081F025E117D90C0EDBCF06F0100EDBCF3C
:100BD00006F126EE6BF00051180DF350D9269BEC70
:100BE00081F0050ED926DFCF08F006B007D0D7EC8C
:100BF00080F0085077D8E8B048D809D0050EEB50FF
:100C0000180D12EE00F0F350E12693EC81F0180E6F
:100C1000E926002B050E0065D2D712000101006BFA
:100C200006EE60F0000EEB5003630CD004C104F03C
:100C3000036A0039700B0309056EDCD8130EDB5014
:100C40009FEC90F0180EE926000EEA22002B050E0C
:100C50000065E8D712000101006B06EE60F0000E9F
:100C6000EB5003630BD0060E046305D00039056E0C
:100C7000AEEC90F003D0400E046300D0180EE926CD
:100C8000002B050E0065EBD7120074D8100EEBCFC9
:100C9000F3FF06B303D0030EF3CFE3FF050EF3CF4C
:100CA000E3FF06A505D0010EE39A0F0EEB0402E068
:100CB000010EE38A06A103D0010EE3B001D021D8D2
:100CC00006A109D8100EEBCFF3FF0451F36203D055
:100CD000110EEB5000E1050E01C1EBFF000E00C14B
:100CE000E3FF1200F56E06B70AD0F550046308D092
:100CF00006B101D01CD80F0EEB50D8A4010C17D8A8
:100D0000000C010EE38006B311D00151C6EC16F0C1
:100D100033130151020FC6EC16F034130151C6EC27
:100D200016F035130151C6EC16F03613120012EE10
:100D300000F0016B010EE3A016D0000EE35000633B
:100D400012D0050EE35004630ED0C3EC59F0010E2F
:100D5000E390E3960151C6EC16F0010EE3880151D1
:100D6000C6EC16F03713180EE126012B050E0165AF
:100D7000E1D7120012EE00F0050EEB501F6F180DB8
:100D8000F350E1260B0EE3CF06F00C0EE3CF07F095
:100D9000070EE3CF08F0D6EC69F0DECF09F0DDCF27
:100DA0000AF0110EDB500F0B026F0001600EC2BD86
:100DB000300E010102131ED80C0EDBB005D006A7C1
:100DC00003D0E4EC58F004D0050EEB50A9EC59F038
:100DD0000B0E06C0E3FF0C0E07C0E3FF070E08C0B2
:100DE000E3FF01C11FF1D6EC69F009C0DEFF0AC0C4
:100DF000DDFF120029EE60F00051300DF350D926CE
:100E0000F450DA2212000101106FF80E1061120086
:100E10000EBF20D00E510ED810630AD00E2B0E51EB
:100E2000070B060A06E1800E0E6F28EC16F001D0C3
:100E30000BD01200070BC8EC16F0F00C000C000CE5
:100E40007E0C4B0C1250120001010E6B0F6B2AEC42
:100E500016F0EFD701010EBD05D00E8D10510F0B0E
:100E60000E13E7D710AF04D0F70E1063EDD70E8B3B
:100E70000E510F0BFF0FD8B410D0FF0FD8B42FD0E6
:100E8000FF0FD8B408D1FD0FD8B442D1FA0FD8B4AF
:100E900071D1FD0FD8B4C1D1D7D70EBB16D00FB1C9
:100EA00004D00F8110C115F1C4D70FB304D00F8344
:100EB00010C114F0BED70FB507D00F8510C113F0C5
:100EC00003DBD8A40E89B5D7B4D70FA5AAD10EB924
:100ED000ACD12EDBD8A4B1D116DB3DDBB5D7108267
:100EE0000EBB45D00FB107D00F8110C115F1116BAA
:100EF000136B146B9ED70FB304D00F8310C114F083
:100F000098D70FB507D00F8510C113F0DDDAD8A43C
:100F10000E898FD70FB728D00FB908D00F8910517D
:100F20000F0B126F10517F0B112783D70F991039B8
:100F3000F00B121310517F0B11271551F70B700A8C
:100F400009E0B5D9132BD8B4142B1451020AD8B424
:100F50000F876FD70BEE00F013C1E9FF12C1EFFF4F
:100F6000132BD8B40F8765D710C112F162D70FA722
:100F700058D10EB95AD1DCDAD8A45FD1115180080A
:100F80007F0B1219D8A44FD11551F70B03E0700A4B
:100F900051E080D0125002E06FDB19D0336A0400B8
:100FA00009C6E8FF01090F0BF36E6DC0E8FFF316E9
:100FB0003350C6EC16F0F31407E0335002E15CDB6B
:100FC00003D0F8EC43F00101332A33A4E8D7080E2C
:100FD000F66E100EF76E010EF86E9AEC16F0060E15
:100FE00088EC16F066EC4FF0400E88EC16F007EE39
:100FF00000F0EE5094EC16F0E9500F0BFAE1040EFD
:1010000053EC4FF0010145D0001450617463682027
:10101000412020312075706C6F616465642000147C
:10102000456E73656D626C65207878787820757090
:101030006C642E2015B70BD01BEE00F0A96A0400DB
:1010400010EC5FF0400EE126A950F9E10BD0136BD4
:1010500004001BEE00F013C1E1FFE7CF12F127D926
:10106000132BF6E1010115A73DEC51F01E0EF66EB3
:10107000100EF76E010EF86E9AEC16F0090E88EC61
:1010800016F057EC4FF001018DEC3EF071EC3EF0A4
:101090001090DDD8D9D60EBB11D00FB104D00F817E
:1010A00010C115F1C6D60FB308D00F8310C114F0CC
:1010B000136A0ADAD8A40E89BCD6BBD60FA3B1D066
:1010C0000EB9B3D0155103E0700A12E0B4D0136A20
:1010D000040019DA40DA132A1450C6EC16F017147B
:1010E0007F0ED8B43F0E1364F3D7136A0CDAACD674
:1010F00011C00AF0116A04003DEC51F011C013F068
:101100002ADA112A11AEF7D7116A3DEC51F09CD6BC
:101110000EBB2CD00FB104D00F8110C115F189D6B0
:101120000FB308D00F831031030B146F136B10B182
:10113000138F7FD60FB505D00F8510517F0B13137A
:1011400078D60FB705D00F8710510F0B126F71D6DD
:101150000F970F891039F00B1213A9D8132BD8B49D
:10116000142B15BD8DEC3EF0010163D60FA959D0AB
:101170006ED86AD60EBB0FD00FB106D00F81010119
:10118000126B10C115F155D60FB304D00F8310C1E7
:1011900012F14FD64ED6155105E0F80F0DE0FF0FB6
:1011A0001BE047D00FA33DD01250FBE11251D8B441
:1011B000010EE8CF6DF02FD00FA133D0336A33503A
:1011C000C6EC16F06DC0F3FFF31402E0EEEC3FF056
:1011D000332A33A4F4D71FD00FA123D012C033F089
:1011E00046C015F145C010F112C146F01251D8B4F5
:1011F000030E456E336A3350C6EC16F06DC0F3FF34
:10120000F31402E0E8EC3FF0332A33A4F4D715C11D
:1012100046F010C145F01BD817D60EAB0AD617D82A
:1012200013D6010E0BD0030E09D00A0E07D00B0EF9
:1012300005D00C0E03D0100E01D0110E076E1BD876
:101240000E0E31DA07502FDA010E28D8FDD513D84B
:101250000F0E29DA12500BE1010109C6E8FF01095E
:101260000F0BF36E6DC0E8FFF3147F0B01D0000E7F
:101270001ADA010E13D001010EAF07D012EC16F0EE
:10128000010B03E0050E066E01D0066A0650D2DDA2
:101290000ADA062A060E0662F9D71200E8B005D06F
:1012A00012EC16F0010BD8B41200F70EFCD10101BC
:1012B0001551F00B04E0700AD8B43BD075D007EE9E
:1012C00000F01551F30B2FE014510BE11351F00B0B
:1012D000400AD8B4A2D0530E136503D05F0E136535
:1012E000A4D0100EEB50030B05E0FF0F13E0FF0F2F
:1012F00018E018D0145105E01351FE0B040A01E167
:101300009FD0145106E15F0E136503D0BF0E136525
:101310009FD009D0145104E15F0E136501D0C9D0EC
:1013200002D001D000D01351E9261451EA223ED850
:1013300039D01339E830E830030B336E03E1FCECAD
:1013400051F002D01CEC43F000EE80F013C1E8FF36
:101350003F0BE92612C1EFFFABEC3EF013C1E8FFF3
:101360003F0B100A05E0100A09E0010A0DE018D051
:1013700000EE3CF0335012C1EBFF12D000EE38F01B
:10138000335012C1EBFF05D000EE34F0335012C1E0
:10139000EBFF00EE40F03350E926810EEF6E00D0F7
:1013A000010100D0000B1200FF09120001011250D0
:1013B00023E10E510F0B060A1FE1336A09C6E8FF4D
:1013C00001090F0BF56E6DC0E8FFF5163350C6EC42
:1013D00016F0F5140DE0335002E10ED809D0E9CF34
:1013E00003F0EA50F90F046E125144EC42F001018F
:1013F000332A33A4E3D7120012C1EFFF020EEA260C
:1014000012C1EFFFFE0EEA265F5006E1040EEA2647
:1014100012C1EFFFFC0EEA2612001351FD0BE92664
:10142000C5DF020EE926C2DF83D71351AC0FE8BE39
:10143000060F540FE926BADF060EE926B7DF78D784
:10144000040EE926010EEA22B1DFE92AAFDF70D7E8
:101450001551F30BFF0F05E0FF0F0EE0FF0F1DE02E
:1014600012001351A00FE8BE300F600FE9269EDF77
:10147000300EE9269BDF5CD713510F0B600FE92676
:101480008F0E136502D0300EE92690DF100EE9268C
:101490008DDF100EE9268ADF4BD713510F0B600F3B
:1014A000E926060EF36E82DF100EE926F32EFBD737
:1014B0003FD71351A00FE8BE500F600FE92676DF2B
:1014C000500EE92673DF34D70101080E146019D0DD
:1014D000145004E0C6EC16F0161413E01551F00B8E
:1014E00003E0700A07E00DD013C034F0348E14C04E
:1014F00038F005D0145005E113C011F01200000BB4
:101500001200FF09120001011551F00B03E0700AEF
:1015100009E00DD015B704D05DEC3EF03BEC54F083
:101520001C8205D015B702D03DEC51F000D012005E
:1015300001011551F80B0AE11350C00B07E01450DC
:10154000C6EC16F0171402E1FF091200000B12009E
:101550000BEE00F002D007EE00F08DDE020EA3D8F5
:1015600015C1E8FFA0D814509ED813509CD8010193
:10157000116B04001551F70B700A46E0EA500B0A94
:101580001CE0336A09C6E8FF01090F0BF36E6DC05A
:10159000E8FFF31612E0030EF3B4020EF3B2010EED
:1015A000F3B0000E030B09E0336EDBEC42F0D0EC3D
:1015B00042F0FDE101010BEE00F0A96AAA6AEECF4C
:1015C000F5FF100EA96006D0AA5004E1200EF560C8
:1015D00001D0F56EF5500F0B112724EC16F0010128
:1015E000F5380F0B112724EC16F00101A92AD8B405
:1015F000AA2AA950E4E1010EAA64E1D7335035E0EC
:1016000071EC3EF0010131D0066A06503F0B15E146
:101610000638E830E830030B336E03E1FCEC51F0A0
:101620000CD01CEC43F03350C6EC16F00601091543
:10163000010103E13350B9EC51F000EE80F00650A7
:101640003F0BE926EECFF5FFF5500F0B112724ECE9
:1016500016F00101F5380F0B112724EC16F00101EB
:10166000062A0650D2E18DEC3EF011C1E8FF800859
:101670007F0B19D8010E12D615B710D017EE00F057
:10168000A96AAA6A0400C2EC5EF0400EE126000ED0
:10169000E222A950F7E1010EAA64F4D734DF67EC27
:1016A0003EF01090120024EF16F00601F00F19E042
:1016B000FF0F1AE0FF0F29E0FF0F3EE0FF0F48E0A9
:1016C000FF0F4EE0FF0F4FE0FF0F4FE0FF0F52E024
:1016D000FF0F5CE0FF0F5DE0FF0F5EE0FF0F5FE0DC
:1016E000030CF7EC52F0000C040E0D63030C080E13
:1016F000E3CFF3FF00EE80F0060EE3503F0BE92648
:10170000F3CFEFFF86EC51F0000C040E0D63030CD9
:10171000080EE3CFF3FF060EE3CFE9FFE3CFD9FFD7
:10172000070EE350010B070FEA6E020FDA6EF3CFDC
:10173000EFFFF3CFDFFF000C040E0D63030C080E68
:10174000E3CF03F0060EE350070B37EC8CF0000CF0
:10175000010E0D63030C060EE350B0EC8CF0000C90
:101760000FEC54F0000C1082000C10EE80F086ECB0
:1017700051F0000C020E0D63030C060EE3CF46F091
:10178000070EE3CF45F08DEC53F0000CDFEC53F087
:10179000000C94EC58F0000CDEEC58F0000C040E39
:1017A0000D63030C080EE3CFF3FF060EE350E96E62
:1017B000EA6AF3CFEFFF000C0601030EE350FF0AC5
:1017C00008E0040EE3CFE9FF030EE350070FEA6ED3
:1017D00006D000EE80F0040EE3503F0BE926080E21
:1017E000DE6EEECFDEFFEECFDEFFEECFDEFFEECF22
:1017F000DEFFEECFDEFFEECFDEFFEECFDEFFEECF81
:10180000DEFF12000D51D8B4030C030EE350FF0AA3
:1018100015E0040EE3CFE9FFE3CFD9FF030EE35059
:10182000010B070FEA6E020FDA6E060EE126E7CF14
:10183000EEFFE6CFDEFF0D2FFAD7000C00EE80F0B2
:10184000040EE3503F0BE926060EE126E6CFEEFF3D
:10185000E6CFEEFFE6CFEEFFE6CFEEFFE6CFEEFF00
:10186000E6CFEEFFE6CFEEFFE6CFEEFF000C010184
:10187000096F84D8020E03C0E3FF020EE226020EB7
:1018800003C0E3FF5F5005E1020EE226020E03C033
:10189000E3FF095143D8F3CF0AF1F4CF0BF110C99C
:1018A000E8FF030B0BE111EE64F0D8900935E12657
:1018B000000E0A5DE66E800E0B59E56E0AC103F05C
:1018C0000BC104F011D8095159D8000EE3509FEC18
:1018D00090F00AC103F00BC104F006D809514ED8AC
:1018E000010EE3509FEF90F010C9E8FFE8B20BD073
:1018F000E8B003D0030E056E1200030E056E4538E6
:10190000300B05121200E8B003D0030E056E120072
:10191000030E056E4638800B051212002FD8020EFA
:10192000E3CFF4FF030EE3CF03F0040EE3CF04F0A4
:101930000450036407D003C0F3FF04C003F0F3CFE7
:1019400004F0F41EF36A0350045C010F01E0F4029A
:101950000350F426F450120011D8020EE350120086
:101960000101096FF9DF036E095181D70101096B8C
:101970000951F6DF092B09A7FBD71200070B17EE59
:1019800018F0050DF350E126F450E2221200F2AEF9
:1019900004D0F29E02D8F28E12000101086F10C925
:1019A000F5FF16EC94F0090009000900F5CFF3FFEC
:1019B0000900F5CFE1FF090EE26EF350C60FD8B073
:1019C000C60E3A0FC8EC16F039D039D03CD093D0BF
:1019D000C1D0F2D03BD044D04ED059D064D06FD0DB
:1019E00077D076D075D074D089D0A1D0B9D0D1D0ED
:1019F000E9D003D106D10ED113D112D114D113D114
:101A000015D11BD121D171D224D123D122D121D101
:101A100036D14ED166D17ED196D1BAD1B9D1FBD1D2
:101A2000B7D1B6D1C0D1CDD1DAD1E7D102D20CD263
:101A300019D226D22BD230D235D23AD2120003504C
:101A40007F0BE76E120003C0E7FF12000338F00BB4
:101A5000E66E03380F0BE76E0438F00BE512120048
:101A6000085103B004D0C4EC16F0E7161200C6EC1F
:101A700016F0E712120005B004D805A21200060EF7
:101A8000E126F00EE71603500F0BE712120005B027
:101A900004D805A21200060EE1260F0EE716033841
:101AA000F00BE712120005B004D805A21200060ED2
:101AB000E12603C0E6FF04500F0BE56E120005B0EF
:101AC00004D805A21200060EE12603C0E7FF1200AB
:101AD00005B004D805A21200300EE1260851030B10
:101AE0000AE109D8100EE12606D8100EE12603D827
:101AF000E00EE126120003C0E7FF120005B004D893
:101B000005A21200300EE1260851030B0AE109D8A4
:101B1000100EE12606D8100EE12603D8E00EE126CD
:101B2000120003C0E6FF04500F0BE56E120005B073
:101B300004D805A21200300EE1260851030B0AE179
:101B400009D8100EE12606D8100EE12603D8E00EC3
:101B5000E1261200F00EE71603500F0BE7121200F9
:101B600005B004D805A21200300EE1260851030B7F
:101B70000AE109D8100EE12606D8100EE12603D896
:101B8000E00EE1261200C00EE71603503F0BE712ED
:101B9000120005B004D805A21200300EE12608514B
:101BA000030B0AE109D8100EE12606D8100EE12633
:101BB00003D8E00EE12612000F0EE7160338F00BF3
:101BC000E7121200020EE26E0851030B0AE109D877
:101BD000180EE12606D8180EE12603D8D00EE1260D
:101BE00012000350800AF36E080E05B0F3CFE3FF36
:101BF000500E05B2F3CFE3FF1200E22A03C0E7FF65
:101C00001200E22A3F0EE7160338E834E834C00B2E
:101C1000E71212000F0EE7160338F00BE71212005E
:101C200003C0E7FF120003C0E7FF1200E22AC00E64
:101C3000E71603503F0BE7121200E22A800EE71668
:101C400003507F0BE7121200020EE26E03C0E7FFA3
:101C50001200E6DAF4B010D805DBF4B20DD802DBDE
:101C6000F4B40AD8FFDAF4B607D8FCDAF4B804D82A
:101C7000F9DAF4BA01D8120003C0E7FF1200D0DA93
:101C8000F4B010D8EFDAF4B20DD8ECDAF4B40AD824
:101C9000E9DAF4B607D8E6DAF4B804D8E3DAF4BA45
:101CA00001D8120003C0E6FF04500F0BE56E1200CE
:101CB000B7DAF4B010D8D6DAF4B20DD8D3DAF4B477
:101CC0000AD8D0DAF4B607D8CDDAF4B804D8CADA2C
:101CD000F4BA01D81200F00EE71603500F0BE7120A
:101CE00012009EDAF4B010D8BDDAF4B20DD8BADA28
:101CF000F4B40AD8B7DAF4B607D8B4DAF4B804D82A
:101D0000B1DAF4BA01D81200C00EE71603503F0B47
:101D1000E712120085DAF4B010D8A4DAF4B20DD8C4
:101D2000A1DAF4B40AD89EDAF4B607D89BDAF4B88C
:101D300004D898DAF4BA01D812000F0EE716033867
:101D4000F00BE71212000851070B06E0FF0F06E048
:101D5000FF0FC6EC16F005D03F0E03D00538070B79
:101D6000F8D7F46E0350800AF36EF4B0F3CF64F644
:101D7000F4B2F3CF7CF6F4B4F3CF94F6F4B6F3CF29
:101D8000ACF6F4B8F3CFC4F6F4BAF3CFDCF6120035
:101D90006EDAF4B005D8500EE126F4B201D8120084
:101DA00003C0E7FF120063DAF4B005D8500EE12655
:101DB000F4B201D8120003C0E6FF04500F0BE56E29
:101DC000120055DAF4B005D8500EE126F4B201D86D
:101DD0001200F00EE71603500F0BE712120047DA5D
:101DE000F4B005D8500EE126F4B201D81200C00EAE
:101DF000E71603503F0BE712120039DAF4B005D8AA
:101E0000500EE126F4B201D812000F0EE716033887
:101E1000F00BE71212002BDAF4B005D8500EE126D1
:101E2000F4B201D812000350800FE8AEFF0EE76E47
:101E300012001DDA0350800AF36EF4B0F3CF64F69B
:101E4000F4B2F3CF7CF6120012DAF4B005D8500EDB
:101E5000E126F4B201D8120003C0E6FF04500F0BD4
:101E6000E56E120004DAF4B005D8500EE126F4B2A3
:101E700001D8120003C0E6FF04500F0BE56E1200FC
:101E800005380F0B0A0DF350E126DDD505380F0B91
:101E90000A0DF350E1262FD605380F0B0A0DF3502B
:101EA000E1268AD605380F0B0A0DF350E12652D6EB
:101EB0000592B6D9F4CF16F112EE00F016B124D87F
:101EC00012EE18F016B320D812EE30F016B51CD86A
:101ED00012EE48F016B718D812EE60F016B914D802
:101EE00012EE78F016BB10D81200020EE26E085106
:101EF000030B0AE109D8180EE12606D8180EE126D0
:101F000003D8D00EE1261200030467E003501FE15E
:101F100005A003D0010EE396E38805A203D0490E85
:101F2000E396E38810C9E8FFE8B20BD0E8B008D028
:101F300043CAE8FFC00B331344CAE8FF34134DD043
:101F40004CD0E8B001D049D0030E341346D0010E76
:101F5000E3A01ED0E3B41CD005A002D0010EE3869E
:101F600005A202D0490EE38610C9E8FFE8B20BD003
:101F7000E8B008D040CAE8FFC00B331341CAE8FFFD
:101F8000341306D005D0E8B001D002D0C00E34130F
:101F900003C0F5FF7B0EF56412D0E1CFF3FFE2CF73
:101FA000F4FF16EE6BF0F550840FE350D8B4E35015
:101FB000F56EF3CFE1FFF4CFE2FFF550A9E0030E99
:101FC00005B0F5CFE3FF010E05B0E38A05A205D009
:101FD0004B0EF5CFE3FF490EE38A120010C9F5FF5F
:101FE00016EC94F0090009000900F550C60FD8B0AE
:101FF000C60E3A0FC8EC16F039D073D07ED07DD023
:1020000056D055D084D035D052D051D080D075D054
:1020100068D073D066D071D07AD049D054D047D030
:102020006CD06BD034D043D068D067D066D065D048
:102030004AD057D056D055D054D05FD052D05DD072
:1020400066D035D040D033D058D04BD056D049D0C0
:1020500048D053D05CD02BD036D029D04ED057D0DA
:102060004CD04BD04AD023D022D03BD0036A046A54
:10207000120005B606D0000E04BE010E036E046AFF
:102080001200000E03B0800E046E036A120005B643
:1020900007D00438E830E830030B036E046A1200FE
:1020A0000338E834E834C00B046E036A120005B646
:1020B00005D004380F0B036E046A12000338F00BCE
:1020C000046E036A120005B606D00430E8303F0BF8
:1020D000036E046A12000334E834FC0B046E036AD6
:1020E000120005B605D004307F0B036E046A12009F
:1020F0000334FE0B046E036A120005B604D004C05C
:1021000003F0046A120003C004F0036A120005B66B
:102110000BD00438F36E0F0B046E03380F0B036EF5
:10212000F350F00B031212000338F36EF00B036E42
:102130000438F00B046EF3500F0B04121200F2AED1
:1021400004D0F29E02D8F28E12000101FF0B05E0CE
:10215000086F059643DF085120DC1200010113EEE1
:10216000A0F00351E3CFF3FF13EEB0F00351E350BF
:10217000F46EB80B27E1F450060B060A23E0F45086
:10218000060B060ED8B4F412F430030B0512F4B0AB
:10219000F38E13EEC0F00351E350036EF4BC0AD08B
:1021A00005C104F0D8900336D89003360436F350B6
:1021B000C6DF08D005C104F00432D8A0038EF35066
:1021C000C7EC8CF012000101FF0B29E0086F03BE81
:1021D00020D01C6BD8900334800F1D6F20E0058445
:1021E000085148EC91F008510586F8DE1C51032691
:1021F0001D5104221DBF04D006E30368046803D008
:1022000002E2036A046A08510596E8DE0851C7EF46
:102210008CF0D8900334046E036A085196DF1200E4
:102220000851070B19E0FF0F1AE0FF0FF46A0201D3
:10223000006301D0F480186301D0F482306301D0D0
:10224000F484486301D0F486606301D0F488786335
:1022500001D0F48A010112003F0EF46E120005381D
:10226000070BE4D7300EE126000EE22212000851DF
:10227000030B0BE0FF0F06E0FF0F02E0020E06D09B
:10228000010E04D00538030B01D0030EF46E1200CA
:10229000F46E10C9F5FF16EC94F00900090009006E
:1022A000F5CFF3FF0900F5CFE1FF070E05B4090EE6
:1022B000E26E046AF350C60FD8B0C60E3A0FC8ECEF
:1022C00016F039D03BD03DD07CD08FD0A0D03BD0C1
:1022D00045D04BD053D05BD066D06DD06CD06BD096
:1022E0006AD071D07CD084D08CD094D09FD0A1D033
:1022F000A6D0A8D0A7D0A8D0A7D0A8D0ABD0AED019
:10230000AED1B0D0AFD0AED0ADD0C0D0D7D0EBD062
:10231000FFD013D11ED11DD155D11BD11AD123D13C
:1023200030D13AD144D15BD166D173D180D185D13E
:102330008AD18FD194D1000E036E1200E7507F0B2B
:10234000FBD7E750F9D7E4380F0B046EE538F00BF4
:10235000036EE7380F0B03120350EED7F450C6ECB0
:1023600016F0E714D8A4010EE7D70550030B020AB4
:1023700002E1060EE126E7500F0BDED70550030BF6
:10238000020A02E1060EE126E7380F0BD5D7055009
:10239000030B020A02E1060EE126E4500F0B046E65
:1023A000E550E750C9D70550030B020A02E1060EBB
:1023B000E126E750C1D70550030B020A02E1300EB7
:1023C000E126E750B9D70550030B020A02E1300EAF
:1023D000E126E4500F0B046EE550E750ADD70550F1
:1023E000030B020A02E1300EE126E7500F0BA4D7DF
:1023F0000550030B020A02E1300EE126E7503F0BC5
:102400009BD70550030B020A02E1300EE126E738A4
:102410000F0B92D7020EE26E0550030B020A02E187
:10242000480EE126080EE350800A86D7E22AE750DC
:1024300083D7E22AE738E830E830030B7DD7E73866
:102440000F0B7AD7E75078D7E75076D7E22AE750D4
:102450003F0B72D7E22AE7507F0B6ED7020EE26E77
:10246000E7506AD7F450070B0FE0FF0F01E003D0ED
:102470000538070B03D0F450070BFE0F300DF35255
:10248000E126F452070BE222E75056D7F450070B2F
:102490000FE0FF0F01E003D00538070B03D0F45025
:1024A000070BFE0F300DF352E126F452070BE22228
:1024B000E4500F0B046EE550E7503ED7F450070B85
:1024C0000FE0FF0F01E003D00538070B03D0F450F5
:1024D000070BFE0F300DF352E126F452070BE222F8
:1024E000E7500F0B29D7F450070B0FE0FF0F01E067
:1024F00003D00538070B03D0F450070BFE0F300D47
:10250000F352E126F452070BE222E7503F0B14D7B7
:10251000F450070B0FE0FF0F01E003D00538070B65
:1025200003D0F450070BFE0F300DF352E126F452A6
:10253000070BE222E7380F0BFFD6020EE26E0550C2
:10254000030B020A02E1480EE126080EE350800A5E
:10255000F3D6F4A006D0F4B202D005B802D0500EE3
:10256000E126E750E9D6F4A006D0F4B202D005B8CF
:1025700002D0500EE126E4500F0B046EE550E750F8
:10258000DBD6F4A006D0F4B202D005B802D0500ECB
:10259000E126E7500F0BD0D6F4A006D0F4B202D05B
:1025A00005B802D0500EE126E7503F0BC5D6F4A087
:1025B00006D0F4B202D005B802D0500EE126E738BA
:1025C0000F0BBAD6F4A006D0F4B202D005B802D0F0
:1025D000500EE126E750800FE8BE000EADD6020E89
:1025E000E26E0550030B020A02E1480EE126080ED6
:1025F000E350800AA1D6F4A006D0F4B202D005B808
:1026000002D0060EE126E4500F0B046EE550E750B1
:1026100093D6F4A006D0F4B202D005B802D0060ECC
:10262000E126E4500F0B046EE550E75085D60538DF
:102630000F0B0A0DF350E12684D605380F0B0A0D57
:10264000F350E126BED605380F0B0A0DF350E126F4
:10265000DED605380F0B0A0DF350E126C6D6020E62
:10266000E26E0550030B020A02E1480EE126030E5A
:10267000E35062D62D2D2D2D2D2D2D2D566F6C75E1
:102680006D65202050686173652020204465747555
:102690006E6520204375744F666620205265736F07
:1026A0006E616E2E4368616E6E656C734D6F64650E
:1026B000202020204B6E6F62202020204578742E31
:1026C000414F55544578742E53772E2057617665C7
:1026D000666F726D5472616E73702E2046696E65FE
:1026E00074756E65506F7274616D2E2050756C73C9
:1026F00065772E2044656C617920202041747461D7
:10270000636B2020446563617920202053757374C6
:1027100061696E2052656C6561736520502E42655B
:102720006E6465724172702E5370642E4172702E09
:10273000474C2E2044657074682020204D6F6449FA
:102740006E762020526174652020202041747461CF
:10275000636B3120412E4C6576656C204174746149
:10276000636B32204465636179312020442E4C65CF
:1027700076656C20446563617932202052656C6512
:1027800061736531522E4C6576656C2052656C65BF
:10279000617365324375727665202020412E437542
:1027A00072766520442E437572766520522E4375ED
:1027B00072766520537065656420202053746172C1
:1027C00074202020456E6420202020204C6F6F70E4
:1027D00020202020506F736974696F6E4E6F74658E
:1027E00020202020446570746820502E4465707449
:1027F00068205057446570746820462E456E764DAB
:102800006F642020416363656E74202044656361BA
:102810007920412E442E4D6F64656C2047617465AC
:102820004C6E2E20506172616D2E3320F5B218D09F
:10283000F5B00BD0040D900EF324F66E280EF420A4
:10284000F76EF86A010EF8221200040D900EF324C0
:10285000F66E300EF420F76EF86A010EF8221200C0
:10286000F5B00BD0040DA00EF324F66E340EF42058
:10287000F76EF86A010EF8221200040D900EF32490
:10288000F66E2C0EF420F76EF86A010EF822120094
:102890000000000001000152020102530301025135
:1028A00004020A5505020B57060208540702095490
:1028B0000803021A0803021F08030224080302295E
:1028C0000803022E08030233080302380803023DFE
:1028D00009040640090406420904064409040646A0
:1028E000090406480904064A0904064C0904064E70
:1028F0000A0407140A0407140A0407140A04071434
:102900000A0407140A0407140A0407140A04071423
:102910000B050E610B050E610B050E710B050E818B
:102920000C050C680C050C680C050C780C050C8863
:102930000D050D690D050D690D050D790D050D8947
:102940000E050F6B0E050F6B0E050F7B0E050F8B23
:102950000F0510640F0510640F0510740F05108427
:1029600010050F6710050F6710050F7710050F870B
:1029700011051362110513621105137211051382FB
:1029800012051162120511621205117212051182EF
:1029900013051363130513631305137313051383CF
:1029A00014051163140511631405117314051183C3
:1029B0001605126D1605126D1605127D1605128D7F
:1029C0001705116E1705116E1705117E1705118E6B
:1029D00015051400150514001505141815051430F7
:1029E00000000000000000000000000000000000E7
:1029F00000000000000000000000000000000000D7
:102A000000000000000000000000000000000000C6
:102A1000180615031806150B180615131806151BAE
:102A2000180615231806152B180615331806153B1E
:102A3000190616021906160A190616121906161A8A
:102A4000190616221906162A190616321906163AFA
:102A50000000000000000000000000000000000076
:102A60000000000000000000000000000000000066
:102A70000000000000000000000000000000000056
:102A80000000000000000000000000000000000046
:102A90000B0717C00B0717C50B0717CA0B0717CF74
:102AA0000B0717D40B0717D9000000000000000027
:102AB000180718C1180718C6180718CB180718D018
:102AC000180718D5180718DA0000000000000000E9
:102AD0001A0719C21A0719C71A0719CC1A0719D1E8
:102AE0001A0719D61A0719DB0000000000000000C1
:102AF000100719C3100719C8100719CD100719D2EC
:102B0000100719D7100719DC0000000000000000B2
:102B1000020719C4020719C9020719CE020719D3FF
:102B2000020719D8020719DD0000000000000000AC
:102B30000000000000000000000000000000000095
:102B40000000000000000000000000000000000085
:102B50000000000000000000000000000000000075
:102B60000000000000000000000000000000000065
:102B70000000000000000000000000000000000055
:102B80000000000000000000000000000000000045
:102B900007081BE018081AE110081BE21B081BE3DA
:102BA0001C081BE41D081BE51E081BE61F081BE78D
:102BB00020081BE813081BE921081BEA22081BEB6D
:102BC00023081BEC25081BED26081BEE27081BEF2E
:102BD00007081BF018081AF110081BF21B081BF35A
:102BE0001C081BF41D081BF51E081BF61F081BF70D
:102BF00020081BF813081BF921081BFA22081BFBED
:102C000023081BFC25081BFD26081BFE27081BFFAD
:102C100028091C6C28091C6C28091C6C28091C6CD0
:102C200029091D6E29091D7329091D7829091D7D92
:102C30002A091D6F2A091D742A091D792A091D7E7A
:102C40002B091D702B091D752B091D7A2B091D7F62
:102C50002C091EEE2C091EF02C091EF22C091EF464
:102C60000000000000000000000000000000000064
:102C70000000000000000000000000000000000054
:102C80002D051F002D051F002D051F182D051F30B8
:102C900000000000010001520000000000000000E0
:102CA00004020A5505020B57000000000000000056
:102CB0000803021A0803021F08030224080302295A
:102CC0000803022E08030233080302380803023DFA
:102CD000090406400904064209040644090406469C
:102CE000090406480904064A0904064C0904064E6C
:102CF0000A0407140A0407140A0407140A04071430
:102D00000A0407140A0407140A0407140A0407141F
:102D10000B0A22610B0A22610B0A22610B0A229123
:102D20000B0A22C10B0A22F10B0A22210B0A2251A3
:102D30000C0A20680C0A20680C0A20680C0A2098EB
:102D40000C0A20C80C0A20F80C0A20280C0A20586B
:102D50000D0A21690D0A21690D0A21690D0A2199BF
:102D60000D0A21C90D0A21F90D0A21290D0A21593F
:102D70000E0A236B0E0A236B0E0A236B0E0A239B8B
:102D80000E0A23CB0E0A23FB0E0A232B0E0A235B0B
:102D90000F0A24640F0A24640F0A24640F0A24947F
:102DA0000F0A24C40F0A24F40F0A24240F0A2454FF
:102DB000110A2762110A2762110A2762110A279253
:102DC000110A27C2110A27F2110A2722110A2752D3
:102DD000120A2562120A2562120A2562120A259237
:102DE000120A25C2120A25F2120A2522120A2552B7
:102DF000130A2763130A2763130A2763130A279307
:102E0000130A27C3130A27F3130A2723130A275386
:102E1000140A2563140A2563140A2563140A2593EA
:102E2000140A25C3140A25F3140A2523140A25536A
:102E3000160A266D160A266D160A266D160A269D96
:102E4000160A26CD160A26FD160A262D160A265D16
:102E5000170A256E170A256E170A256E170A259E72
:102E6000170A25CE170A25FE170A252E170A255EF2
:102E7000150A2800150A2800150A2800150A280135
:102E8000150A2802150A2803150A2804150A280518
:102E90002E0B21752E0B21752E0B21752E0B21A5C6
:102EA0002E0B21D52E0B21052E0B21352E0B216546
:102EB0002F0B21792F0B21792F0B21792F0B21A992
:102EC0002F0B21D92F0B21092F0B21392F0B216912
:102ED000300B217A300B217A300B217A300B21AA6A
:102EE000300B21DA300B210A300B213A300B216AEA
:102EF0001A0B21761A0B21761A0B21761A0B21A6B2
:102F00001A0B21D61A0B21061A0B21361A0B216631
:102F10002E0C217C2E0C217C2E0C217C2E0C21AC25
:102F20002E0C21DC2E0C210C2E0C213C2E0C216CA5
:102F30002F0C21802F0C21802F0C21802F0C21B0F1
:102F40002F0C21E02F0C21102F0C21402F0C217071
:102F5000300C2181300C2181300C2181300C21B1C9
:102F6000300C21E1300C2111300C2141300C217149
:102F70001A0C217D1A0C217D1A0C217D1A0C21AD11
:102F80001A0C21DD1A0C210D1A0C213D1A0C216D91
:102F90002E0D21832E0D21832E0D21832E0D21B385
:102FA0002E0D21E32E0D21132E0D21432E0D217305
:102FB0002F0D21842F0D21842F0D21842F0D21B45D
:102FC0002F0D21E42F0D21142F0D21442F0D2174DD
:102FD000300D2185300D2185300D2185300D21B535
:102FE000300D21E5300D2115300D2145300D2175B5
:102FF000110D2386110D2386110D2386110D23B685
:10300000110D23E6110D2316110D2346110D237604
:10301000120D2387120D2387120D2387120D23B75C
:10302000120D23E7120D2317120D2347120D2377DC
:10303000130D2388130D2388130D2388130D23B834
:10304000130D23E8130D2318130D2348130D2378B4
:10305000140D2389140D2389140D2389140D23B90C
:10306000140D23E9140D2319140D2349140D23798C
:103070002D0A39002D0A39002D0A39002D0A39018F
:103080002D0A39022D0A39032D0A39042D0A390572
:1030900000000000010001520000000000000000DC
:1030A00004020A5505020B57060208540702095488
:1030B0000803021A0803021F080302240803022956
:1030C0000803022E08030233080302380803023DF6
:1030D0000904064009040642090406440904064698
:1030E000090406480904064A0904064C0904064E68
:1030F0000A0407140A0407140A0407140A0407142C
:103100000A0407140A0407140A0407140A0407141B
:103110000B0E2C610B0E2C610B0E2C610B0E2C6117
:103120000C0E29680C0E29680C0E29680C0E2968F3
:103130000D0E2A690D0E2A690D0E2A690D0E2A69D7
:103140000E0E2D6B0E0E2D6B0E0E2D6B0E0E2D6BAF
:103150000F0E2E640F0E2E640F0E2E640F0E2E64B3
:10316000100E2D67100E2D67100E2D67100E2D6797
:10317000110E3162110E3162110E3162110E316287
:10318000120E2F62120E2F62120E2F62120E2F627B
:10319000130E3163130E3163130E3163130E31635B
:1031A000140E2F63140E2F63140E2F63140E2F634F
:1031B000160E306D160E306D160E306D160E306D0B
:1031C000170E2F6E170E2F6E170E2F6E170E2F6EF7
:1031D000150E3200150E3200150E3218150E323053
:1031E00000000000000000000000000000000000DF
:1031F00000000000000000000000000000000000CF
:1032000000000000000000000000000000000000BE
:10321000040E3355040E3355040E3355040E335B40
:10322000050E3457050E3457050E3457050E345D20
:10323000310E2B85310E2B85310E2B85310E2B85D2
:10324000120E2D87120E2D87120E2D87120E2D872E
:10325000320E2C66320E2C66320E2C66320E2C6626
:10326000000000000000000000000000000000005E
:1034A00000000000010001520000000000000000C8
:1034B00004020A5505020B5700000000000000003E
:1034C0000803021A0803021F080302240803022942
:1034D0000803022E08030233080302380803023DE2
:1034E0000904064009040642090406440904064684
:1034F000090406480904064A0904064C0904064E54
:103500000A0407140A0407140A0407140A04071417
:103510000A0407140A0407140A0407140A04071407
:10352000341135611111376212113862131137638A
:10353000141138630D11366435113665281136665D
:103540003611366700000000000000000000000097
:10355000000000000000000000000000000000006B
:10356000341202613412026B341202753412027F7B
:1035700034120289341202933412029D341202A7CB
:10358000341202B1341202BB341202C5341202CF1B
:10359000341202D9341202E3341202ED341202F76B
:1035A000111205621112056C1112057611120580B7
:1035B0001112058A111205941112059E111205A807
:1035C000111205B2111205BC111205C6111205D057
:1035D000111205DA111205E4111205EE111205F8A7
:1035E000121204621212046C121204761212048077
:1035F0001212048A121204941212049E121204A8C7
:10360000121204B2121204BC121204C6121204D016
:10361000121204DA121204E4121204EE121204F866
:10362000131205631312056D13120577131205812A
:103630001312058B131205951312059F131205A97A
:10364000131205B3131205BD131205C7131205D1CA
:10365000131205DB131205E5131205EF131205F91A
:10366000141204631412046D1412047714120481EA
:103670001412048B141204951412049F141204A93A
:10368000141204B3141204BD141204C7141204D18A
:10369000141204DB141204E5141204EF141204F9DA
:1036A0000D1203640D12036E0D1203780D120382C6
:1036B0000D12038C0D1203960D1203A00D1203AA16
:1036C0000D1203B40D1203BE0D1203C80D1203D266
:1036D0000D1203DC0D1203E60D1203F00D1203FAB6
:1036E000351203653512036F3512037935120383E2
:1036F0003512038D35120397351203A1351203AB32
:10370000351203B5351203BF351203C9351203D381
:10371000351203DD351203E7351203F1351203FBD1
:1037200028120366281203702812037A28120384D1
:103730002812038E28120398281203A2281203AC21
:10374000281203B6281203C0281203CA281203D471
:10375000281203DE281203E8281203F2281203FCC1
:1037600036120367361203713612037B3612038555
:103770003612038F36120399361203A3361203ADA5
:10378000361203B7361203C1361203CB361203D5F5
:10379000361203DF361203E9361203F3361203FD45
:1037A0000000000000000000000000000000000019
:1037B0000000000000000000000000000000000009
:1037C00000000000000000000000000000000000F9
:1037D00000000000000000000000000000000000E9
:1037E00000000000000000000000000000000000D9
:1037F00000000000000000000000000000000000C9
:1038000000000000000000000000000000000000B8
:1038100000000000000000000000000000000000A8
:103820000000000000000000000000000000000098
:103830000000000000000000000000000000000088
:103840000000000000000000000000000000000078
:103850000000000000000000000000000000000068
:103860000000000000000000000000000000000058
:103870000000000000000000000000000000000048
:103880000000000000000000000000000000000038
:103890000000000000000000000000000000000028
:1038A000FFFF83F9E1E772CFC4B41C9B2B847F70C8
:1038B000FF5F4D52FA46993DCD354A2FD0292F252D
:1038C0003E21DE1DF51A70183E165114A01221116A
:1038D000CC0F9D0E8D0D990CBD0BF60A420A9D0969
:1038E00008097F0801088D072307C106660612062E
:1038F000C4057C053805F904BE0487045304230479
:10390000F503CB03A2037C03580336031603F80226
:10391000DB02C002A6028D02760260024B02360272
:1039200023021102FF01EE01DE01CF01C001B2014D
:10393000A40197018B017F01740168015E015401AC
:103940004A01400137012E0126011E0116010E0118
:1039500007010001F900F200EC00E500DF00DA00E9
:10396000D400CF00C900C400BF00BA00B600B10047
:10397000AD00A800A400A0009C0098009500910054
:103980008E008A008700840081007E007B00780022
:10399000750072006F006D006A00680065006300CA
:1039A00061005F005C005A0058005600540052004D
:1039B00050004F004D004B004900480046004500B4
:1039C0004300410040003F003D003C003A00390008
:1039D0003800370035003400330032003100300049
:1039E0002F002D002C002B002A0029002900280080
:1039F00027002600250024002300230022002100A8
:103A000020001F001F001E001D001D001C001B00C9
:103A10001B001A00190019001800180017001700E1
:103A200016001600150015001400140013001300F2
:103A300012001200110011001100100010000F0000
:103A40000F000F000E000E000E000D000D000D0007
:103A50000C000C000C000B000B000B000A000A000D
:103A60000A000A000900090009000900080008000E
:103A7000080008000800070007000700070007000B
:103A80000600060006000600060006000500050008
:103A90000500050005000500050004000400040001
:103AA000000001000300060008000A000C000E00E0
:103AB000100012001500170019001C001E00210044
:103AC0002300260028002B002D0030003300360094
:103AD00038003B003E004100440047004A004D00D2
:103AE0005000530057005A005D00610064006800F8
:103AF0006B006F00730076007A007E008200860003
:103B00008A008E00920096009A009F00A300A800F1
:103B1000AC00B100B500BA00BF00C400C900CE00BF
:103B2000D300D800DD00E300E800ED00F300F90069
:103B3000FE0004010A01100116011C0123012901E4
:103B4000300136013D0144014B0151015901600131
:103B500067016F0176017E0185018D0195019D014F
:103B6000A601AE01B601BF01C801D101DA01E3012E
:103B7000EC01F601FF01090213021D0227023102C6
:103B80003C02460251025C02670272027E028A0215
:103B90009502A102AE02BA02C602D302E002ED0211
:103BA000FA02080316032403320340034F035D03A4
:103BB0006C037C038B039B03AB03BB03CB03DC03D2
:103BC000ED03FE03100421043304450458046B0480
:103BD0007E049104A504B904CD04E204F7040C05A5
:103BE000210537054D0564057B059205A905C1052D
:103BF000D905F2050B0624063E06580673068E0606
:103C0000A906C506E106FE061B0738075607750715
:103C10009307B307D207F307130835085608790846
:103C20009B08BF08E20807092C09510977099E097A
:103C3000C509ED09150A3E0A680A920ABD0AE90A91
:103C4000150B420B6F0B9D0BCC0BFC0B2C0C5D0C66
:103C50008F0CC20CF50C290D5E0D940DCA0D020ED1
:103C60003A0E730EAD0EE80E230F600F9D0FDC0FA2
:103C70001B105B109D10DF1022116611AC11F211A8
:103C800039128212CC1216136213AF13FD134D14A6
:103C90009D14EF1442159615EB1542169A16F4165C
:103CA0001000200040008000000100020004000815
:103CB000001000200040F36EF46A0B0EF36404D091
:103CC000F40EF326F42AF9D7F334FE0B080FF66E40
:103CD000F76A3D0EF722010EF8220900010EF46486
:103CE00005D0E00EF526FE0EF42604D0020EF4B048
:103CF000010EF46EF55094EC16F00900F55094ECBA
:103D000016F0F4508EEF16F0632D6323642D6423B8
:103D1000652D662D6623672D6723612D6123622D36
:103D200028002B002D0030003300360039003D0004
:103D30004000440048004C00510056005B00600009
:103D400066006C0073007A00810089009100990080
:103D5000A300AC00B700C100CD00D900E600F4001C
:103D60000201120122013301460159016E01830152
:103D70009B01B301CD01E80105022402450267025F
:103D80008C02B302DA020703360366039A03D103F7
:103D90000B0449048A04CF0418056605B8050F060C
:103DA0006C06CD063507A3071708920815099F0969
:103DB000310ACD0A710B1F0CD80C9B0D6A0E460FF1
:103DC0002E1025112A123E1363149A15E3163F187C
:103DD000B019371BD51C8C1E5D204A2254247D2629
:103DE000C728342BC62D7E3061336F36AB39193D71
:103DF000BC409544A848FC4C8F5168568C5BFE60D3
:103E0000C266DE6C5773347A77812A895391F699AA
:103E10001EA3D1AC18B7FCC185CDBCD9AFE667F401
:103E2000000092012403B6044706D9076A09FB0A79
:103E30008B0C1B0EAB0F3911C8125514E2156D1700
:103E4000F818821A0B1C931D191F9F202322A623EA
:103E50002825A8262628A3291F2B982C112E872F2A
:103E6000FB306E32DE334D35BA3624388C39F23AB7
:103E7000563CB83D173F7340CE4125437A44CD456B
:103E80001C476948B449FB4A3F4C814DBF4EFB4F2C
:103E9000335169529B53CA54F5551D5742586459C2
:103EA000825A9D5BB45CC75DD75EE35FEC60F161F5
:103EB000F262EF63E864DD65CF66BD67A6688C6972
:103EC0006D6A4A6B246CF96CCA6D966E5F6F2370D5
:103ED000E2709E7155720773B5735F740475A575B2
:103EE0004176D9766C77FA77847809798A79057A78
:103EF0007D7AEF7A5D7BC57B297C897CE37C397D8B
:103F00008A7DD67D1D7E5F7E9D7ED57E097F387F32
:103F1000627F877FA77FC27FD87FE97FF67FFD7FA3
:103F20000001020304050607080A0C0E11121314FF
:103F3000151618181B1C1E20222426282B2D303362
:103F400036393D4044484D51565B61666C737A8109
:103F5000899199A3ACB7C2CDD9E6F4FFFFFFFFFF6B
:103F6000883FA43FBA3FD63FEC3F0E401E402C4056
:103F70003E4068409240A640B440C840D640004110
:103F80002A4142415841764142443120003C2001BF
:103F9000800A07FFBC013A013801340130012C01CD
:103FA0002801200142443220006B2008800A04FFCF
:103FB000EB083C04370432042A044244332000480E
:103FC0002001800A07FFC8014E08C501B5044E084C
:103FD000400847083B0853443120006B2008800A02
:103FE00004FF6B08BC046B08BB046B08534432200D
:103FF00000502008800A0AFF5008BC04BA04500888
:104000005108520853085408550856085708534495
:104010003320004B2008800A01004B08BC014848AF
:104020003120006C2008800A00FFEC08484832204C
:10403000006C2008800A02FFEC083304EC08544F9F
:104040003120003C2004800A0DFFBC043B04BA046C
:104050003804B7043404B3043104AF042D04AA04B3
:104060002604A2041C049304544F3220003C200474
:10407000800A0D0CBC043B01BA043801B7043401BA
:10408000B3043101AF042D01AA042601A2041C01CE
:104090009304434C5020003C2008800A04013C0853
:1040A000F0083008BC0846583120003C2001800A46
:1040B00000FFBC0146583220003C2001800A03006A
:1040C000BC013001BC01480146583320003C20416E
:1040D000800A00FFBC4146583420003C2041800A41
:1040E0000DFFBC413B41BA413841B7413441B34176
:1040F0003141AF412D41AA412641A2411C4193418A
:104100004658352000542004800A0D0AD4043B018F
:10411000E0043801D4043401E0043101D4042D0159
:10412000E0042601D4041C01E0044658362000189F
:104130002001800A050098012401B0013C01C8015A
:1041400054014658372000182002800A04009802C3
:104150003C0224023C02B00246583820007020087D
:10416000800A0800F00868086004D804500848086D
:10417000C004380830044658392000182004800A4A
:104180001100980454012404C80130043C01BC040B
:1041900030014804980154042401C80430013C044F
:1041A000BC01300448010001F06BF16B10941096D3
:1041B000120010841086F5ECA0F010EE60F0F36AA7
:1041C000E66AF32AF3A6FCD71200109410961C821C
:1041D000F7EF52F00014534944706C617965722016
:1041E0004D6F6465202020202020D40EF66E410EF5
:1041F000F76E010EF86E9EEC16F0400E88EC16F08D
:10420000140E53EC4FF0400E88EF16F0401250722F
:10421000657373204D454E5520746F206578697421
:104220000C0EF66E420EF76E010EF86E9EEC16F056
:10423000400EFAEF16F0036EF80E0360C2D00001D4
:1042400003BEF06BF051030BC8EC16F003D004D0A2
:104250000AD016D0F00E01D02D0E036202D0F02B42
:10426000B0D0F06BAED0F02BF26B0350F16F4C0A74
:1042700012E0010A13E0030A21E0010A12E0A1D0D2
:10428000F22BF1514C0A09E0010A0AE0030A1AE094
:10429000010A10E096D08DDF94D093D096DF91D0B4
:1042A00090D0400E88EC16F010B402D082DF01D01E
:1042B000A4DF87D0035094EC16F083D0F36B10A4E6
:1042C00078DF7FD0090EF26106D000EEF4F0F2053F
:1042D00003C0EBFF76D01C0EF36173D0F4B102D0B3
:1042E00052D8F9D703C004F0F351010DC40EF324E2
:1042F000F66E430EF420F76EF86A010EF8220900FC
:10430000F550E009036EF8B1048E170EF56202D085
:10431000F70E041610A62CD003501F0B040A0CE154
:1043200024C3E8FF010B08E104A006D03F0EE8CF4C
:10433000E8F0E8CFE9F01CD00F0A0CE12BC3E8FF4E
:10434000010B08E104A006D03F0EE8CFEBF0E8CF68
:10435000ECF00ED0190A0CE132C3E8FF010B08E1C2
:1043600004A006D03F0EE8CFEEF0E8CFEFF000D08B
:1043700003EE20F013EE60F0F29E0450D6EC61F0F4
:10438000F28E01D81ED0D890F733D8B0F68FD890DF
:10439000F633D8B0F58FD890F533D8B0F48FD890E5
:1043A000F433D890FB33D8B0FA8FD890FA33D8B022
:1043B000F98FD890F933D8B0F88FD890F833F32B21
:1043C000120012000001020305060708090A0C0D7D
:1043D0000E0F1011131415161718040B12040B12DC
:0200000400F00A
:100000004C656164205061746368202020202020AA
:10001000000000000000000000008000FF000080E1
:1000200000FF00008000FF00008000FF0000800053
:10003000FF00008000FF50008000FF00008000FFF4
:1000400000800080008000800080008000800080B0
:1000500000007F00100002000000100002000000FD
:10006000000400F00008000040800200001F0500AE
:10007000001400F00008000040800200001F05008E
:10008000001400F00008000040800200001F05007E
:10009000000400F00008000040800200001F05007E
:1000A000001400F00008000040800200001F05005E
:1000B000001400F00008000040800200001F05004E
:1000C00001800000000180000000018000000001AC
:1000D000800000000180000000018000000000009E
:1000E00000C00030FF0000FF304020000080808012
:1000F00000400050FF0000FF501030000080808062
:10010000010003C000000000020003C00000000066
:10011000030003C000000000040003C00000000052
:10012000050003C000000000060003C0000000003E
:10013000070003C000000000080003C0000000002A
:10014000FF000F3F0300000000000000000000005F
:10015000000000000000000000000000000000009F
:10016000F00000000000000000000000CB00001FB5
:1001700080CB00203FA0CB00405FC0CB00607FE081
:10018000404040404040404040404040404040406F
:10019000404040404040404040404040404040405F
:1001A000404040404040404040404040404040404F
:1001B000404040404040404040404040404040403F
:1001C000404040404040404040404040404040402F
:1001D000404040404040404040404040404040401F
:1001E000404040404040404040404040404040400F
:1001F00040404040404040404040404040404040FF
:1002000000000200027800000000006000000060B2
:1002100000007F400000000010007F400000000050
:1002200010007F400000000010007F400000000030
:1002300010007F400000000010007F400000000020
:100240000000000002780000000000600000006074
:1002500001007F400000000010007F40000000000F
:1002600010007F400000000010007F4000000000F0
:1002700010007F400000000010007F4000000000E0
:100280000000000002780000000000600000006034
:1002900002007F400000000010007F4000000000CE
:1002A00010007F400000000010007F4000000000B0
:1002B00010007F400000000010007F4000000000A0
:1002C00000000000027800000000006000000060F4
:1002D00003007F400000000010007F40000000008D
:1002E00010007F400000000010007F400000000070
:1002F00010007F400000000010007F400000000060
:020300000100FA
:00000001FF
